:020000040800F2
:10000000002000109DEC020805ED02086164000864
:1000100005ED020805ED020805ED020800000000EC
:1000200000000000000000000000000005ED0208D4
:1000300005ED02080000000005ED020855790008F2
:1000400005ED020805ED020805ED020805ED0208C0
:1000500005ED020805ED02080545000831460008D7
:10006000F5450008B94500087D450008D959000844
:10007000C9590008B9590008A95900089959000838
:10008000855900087159000805ED020805ED0208C0
:1000900005ED020805ED020805ED020841450008DE
:1000A000B16A0008F16A0008A16A0008196B00082B
:1000B000E16A0008D16A0008C16A000805ED02087B
:1000C00005ED020805ED020805ED020805ED020840
:1000D00005ED0208D97A00085D7A0008E179000888
:1000E000C944000805ED020805ED020805ED020807
:1000F00005ED020805ED020805ED020805ED020810
:1001000000000000000000000000000005ED0208F3
:1001100005ED020805ED020895AC020879AC02086D
:100120005D5900084959000835590008215900084F
:100130000D59000805ED0208000000000000000055
:1001400005ED020805ED020805ED020800000000BB
:10015000000000000000000000000000000000009F
:10016000000000000000000005ED020805ED020897
:1001700005ED020800000000000000000000000083
:080180000000000005ED02087B
:100188002DE9F04F2DED028B97B00646B0F9080027
:100198000881C5B200AF28460C46924605F07EFE9F
:1001A80048B101231A4618465C376281BD46BDEC4A
:1001B800028BBDE8F08FA5F10A02E72A00F2EA8077
:1001C800DFE812F0FA04E800E800E800E800E800D8
:1001D800E800E800E800E800E800E800E800E800D7
:1001E800E800E800E800E800E800E800E800E800C7
:1001F800E800E8000D05E800E800E8002C05E80044
:10020800E800E800C203E800E403E8002404E8008A
:100218003D04E8009903E8009D03E8008503E80031
:10022800E800E800FE010502E8000D02E800E80029
:100238001B02E8002302E800E800E8004C02E8009E
:10024800E800E800E8007E02E8009902E800ED0115
:10025800BC02E800E800E800E800E800E800E80080
:10026800E202E8002803E8005503E8005605E80024
:10027800AC05E800E800E800E800BC05E1051F0659
:1002880054062806E800E8003B068606E8009406BF
:100298002007E800E800E800E8003D07E800E8007B
:1002A800FE06E800E800E80073074907620749040A
:1002B800E800E800E8008C04E800E8009D04E80095
:1002C800E800E800E800E800E800E800E800E800E6
:1002D800E800E800E800E800E800E800BC05E800FD
:1002E800E800E800E800E800E800E800E800E800C6
:1002F800E800E800E800E800E800E800E800E800B6
:10030800E800E800E800E800E800E800E800E800A5
:10031800E800E800E800E800E800E800E800E80095
:10032800E800E800E800E800E800E800E800E80085
:10033800E800E800E800E800E800E800E800E80075
:10034800E800E800E800E800E800E800E800E80065
:10035800E800E800E800E800E800E800E800E80055
:10036800E800E800E800E800E800E800E800E80045
:10037800E800E800E800E800E800E800E800E80035
:10038800E800E800E800E800E800E800E800E80025
:10039800C204CF04742D35D0772D25D0F52D00F06B
:1003A8009586472D3CD0392D326800F0E78700F25A
:1003B800F186212D01F09487292D41F02380531CCB
:1003C800336013780A2B02F04280502B41F01686D6
:1003D800304604F04EFCB04D2880304604F049FC0D
:1003E800012368801A46DEE6336872689A421EBFA7
:1003F8005A1C32601978A94A08BF0021204628F003
:10040800AFFCCEE6336872689A421EBF5A1C32604F
:100418001978A34A08BF0021204628F0A1FCC0E6AD
:100428007268356878623046551B04F00BFC052D60
:1004380038627B6A01F2D8878026B346012594E8A2
:100448000600521A103AB242B8BF1FFA82FB954A08
:10045800396A92683A61521A9345396A7B62204632
:10046800FA6088BF1FFA82FB04F02AFC7B6A002B23
:1004780001F07D87002D41F053872368C7F800D02D
:100488005D71C0B00533C7F808D0FB61BBF1000F40
:1004980002F0EF803B6A3A69934282F0E680AA460E
:1004A8003E6A7D627C6080255446FB681C1B7D4B40
:1004B800B4F5807F28BF4FF480749B6832199A4244
:1004C80088BF9C1B04F04AFF2246BC683046214680
:1004D80004F0C4FFF969B86104EB000C0B787B6188
:1004E800644530D2DFF8D4910CF1FF3C04F1FF3EB3
:1004F8001EF8013F09EB830219F823405688FCB126
:1005080000234FF4004204F1FF3816424FEA52022A
:1005180002D00878284308706D0806D10AF1010A4C
:100528004D701FFA8AFA01318025D34505D8E64572
:10053800C0F029864345C0F2268601339C42E4D1A7
:10054800F445D5D1F9617B6ABA6913449BB2D345A6
:100558007B6206D97B6A3A6A1C46D6183B699E427A
:10056800A3D37C68802D1CBF0AF101031FFA83FA0C
:100578000AF1020189B2204604F0B9FB2368796ABE
:1005880001255A19226020461D7004F0B0FB22682C
:10059800524422602B462A46D7F800D003E6236847
:1005A80000255A1C22601D7023685A1C22601D7089
:1005B80023685A1C226029461D70204604F080FBDF
:1005C8000021204604F07CFB01231A46EBE5216854
:1005D80001200A182260034602460870E3E5324B00
:1005E80022689978501C20601170216858784A1C3C
:1005F800012322601A460870D5E508222B492046B7
:1006080004F047FB01231A46CDE52368284A294D03
:100618001178294A581C206019701168204604F086
:100628004FFB2368214A591C127A21601A702988C5
:10063800204604F05CFBA988204604F058FB298971
:10064800204604F054FB0021204604F050FB002112
:10065800204604F04CFB01231A46A4E504F070FD83
:100668002368104D002803F101010CBF0222032268
:1006780021601A702988204604F022FBA9682046C8
:1006880004F01EFB04F034FD0146204604F018FB7C
:1006980001231A4687E500BF2C2A00209982020808
:1006A800158C0208581C00204C35002020680020BA
:1006B8007035002088310020A8440020381803082D
:1006C8002368A34D591C2A7921601A7023686A7916
:1006D800591C21601A702988204604F008FB2368F9
:1006E800AA79591C21601A706988204604F0FFFA1B
:1006F8002168E8797BE7974D2B78002B3FF451ADC3
:10070800954E4FF00008B146236816F81820591C7A
:1007180021601A7099F8011001EB810101EB810148
:1007280001F2EE2189B2204604F0E1FA2B7808F1B3
:100738000108984509F10209E6DB32E52368874E8E
:1007480001255A1C22601D702368B278591921604E
:100758001A7013F017FC2368814A824903EB050ECF
:10076800C4F800E01870B1F90010B2F9000004F004
:1007780047FC23685A19226018703188204604F013
:10078800B6FA2B462A460EE521F028F8FF28064639
:1007980001F0388607F15801002501F82E5D07F1B0
:1007A800290087F8295020F0F9FF07F1580000F8D0
:1007B8002D5D20F0E7FF07F1580000F82C5D20F0D0
:1007C800D5FF07F1580020F8245D20F0C3FF236807
:1007D8005A1C22601E70236897F82920591C216032
:1007E8001A70236897F82A20591C21601A70236808
:1007F80097F82B20591C21601A70236897F82C2031
:10080800591C21601A70B98E204604F070FA012331
:100818001A46C8E4DFF8548198F80330002B01F039
:10082800D18523680822591C21601A702368012287
:10083800991821601A7023684B4D591C2A79216038
:100848001A702368AA78591C21601A7029882046D2
:1008580004F04DFAE989204604F049FA236898F82B
:100868000720591C21601A702168E878BFE63F4EBE
:10087800236872793E4D591C21601A702B682046F6
:10088800198C04F034FA2B682046D98B04F02FFA1F
:100898007189204604F02BFAB189204604F027FA22
:1008A8002B682046598C04F022FA2B682046998C34
:1008B80004F01DFAF189204604F019FA318A20461D
:1008C80004F015FA2B68216893F826008FE6294D65
:1008D800294E05F1280895F90210284B93F90620AE
:1008E8008A4203F1080300F060849E42F6D108357D
:1008F8004545F0D155E4224B2168587D77E6214BD8
:1009080003F15A0522685979501C20601170226839
:100918001978501C2060117022685978501C20608A
:10092800117022689978501C206011702268D9785B
:10093800501C20601170226819790633501C9D42A2
:1009480020601170DED12CE40F4B2268197849E63B
:10095800C049002030540020A06A0020A47600205E
:10096800A0330020A2330020BC600020EC630020EC
:100978003C42002094700020FC670020D4670020CF
:10098800206800205C47002070350020AC4D2368AB
:100998002A7A591C21601A70A98B204604F0A7F9FD
:1009A800298B204604F0A3F9698B204604F09FF9AF
:1009B8002368EA7C591C21601A70A98C204604F02F
:1009C80096F9E98C204604F092F92368AA7F591C0D
:1009D80021601A70236895F82020591C21601A702C
:1009E800698C204604F083F92368EA7A591C21604F
:1009F8001A70E968204604F063F923682A7C591CB8
:100A080021601A70216895F82100F0E58D4D05F1F7
:100A18004006B5F88010204604F069F9236895F877
:100A28008220591C21601A70236895F883200435A8
:100A3800591CB54221601A70EBD1FFF7B2BB824D49
:100A480005F1800655F8041F204604F039F9B5422F
:100A5800F8D1FFF7A6BBDFF810C24FF0000E5FFA1F
:100A68008EF6614600232268501C206016702268AA
:100A7800501C20601370226811F8010F0133551CB7
:100A8800062B25601070EED10EF1010EBEF1060F97
:100A98000CF1060CE3D16D4900232268501C20603C
:100AA80082F800E02268501C20601370226811F858
:100AB800010F0133551C0B2B25601070EDD12368F5
:100AC800604A581C07212060197023680021581CAF
:100AD80020601970216892F8F00088E55C4D204686
:100AE800298A04F004F9698A204604F000F9A98AE1
:100AF800204604F0FCF801231A46FFF754BB23688C
:100B0800DFF86881591C98F8002021601A7098F85D
:100B18000030002B3FF445AB0025EEB230461FF005
:100B2800A5FC23684278591C216030461A701FF0D2
:100B38009DFC0189204604F0DAF898F80030013568
:100B48009D42EADBFFF72DBB424D2046E98904F0C0
:100B5800CEF8A989204604F0CAF801231A46FFF7FF
:100B680022BB3D4B03F1700522681978501C2060A8
:100B7800117022685978501C206011702268997889
:100B8800501C206011702268D978501C20601170A8
:100B980022681979501C2060117022685979501CFC
:100BA80020601170226899790733501C9D4220609B
:100BB8001170D9D1FFF7F5BA284D28462DF0CCF998
:100BC80000287FF7EEAA2B460544226813F8011B7C
:100BD800501C9D4220601170F7D1FFF7E2BA204DFA
:100BE80005F15006287828F00FF92368027A591C75
:100BF80021601A7023686A78591C21601A7023686A
:100C0800AA78591C21601A702368EA780435591C9F
:100C1800AE4221601A70E5D1FFF7C3BA114D2046E4
:100C2800298804F064F8A988204604F060F8298926
:100C3800204604F05CF801231A46FFF7B4BA00BF57
:100C480020680020E4400020E0400020C741002048
:100C5800BC60002030350020743800202442002079
:100C68007435002088310020A3410020194E00204F
:100C78000021204604F03BF80021204604F037F814
:100C88000021204604F033F82368B54D00265A1C8D
:100C980022601E7023682A68591C92F82C20216053
:100CA8001A7023682A68591C92F8362021601A7035
:100CB80023682A68591C92F8372021601A70236823
:100CC8005A1C22601E7023685A1C22601E702368FA
:100CD8005A1C22601E702B682046598F04F007F8B2
:100CE8002B682046198F04F002F823682A68591CDB
:100CF80092F82E2021601A7023685A1C22601E70F8
:100D08002B682046598E03F0F2FF2B682046998EF7
:100D180003F0EDFF01231A46FFF745BA2368914A0D
:100D28009149D078914A5D1C2560187023684979EB
:100D3800581C206019702168D07858E4002607F103
:100D480034037B62DFF860B2894A7E63FE623E63E9
:100D5800BE6301214FF6FF7A05E001360B2E00F045
:100D680042821BF9011F481C4AFA06F3F5D0DB073B
:100D7800F3D513883341D807EFD5786A3A6204F07F
:100D88009BF93A6AE9E77B4B9B8AB3F5006F01F25E
:100D98002783B3F5806F01F26083B3F5007F34BF1A
:100DA8004FF001084FF00208734D05F10C0655F895
:100DB800041B91FBF8F1204689B203F098FFB54275
:100DC800F5D16E4DDFF8E48105F10C06B5EC010AAA
:100DD800D8ED087A80EE270A2EF04AFB81B2204629
:100DE80003F085FFB542F1D1654D05F10C0655F8C4
:100DF800041B204689B203F07AFFAE42F7D1FFF711
:100E0800D0B910225F49204603F043FF01231A4658
:100E1800FFF7C9B95C4D2B78002B3FF4C2A9DFF866
:100E28009081002638F8021F204603F060FF2B78D7
:100E380001369E42F6DBFFF7B4B9544D20462988A7
:100E480003F055FF6988204603F051FFB5F90430D7
:100E58004F49DA1781FB0313C2EBA30399B220466B
:100E680003F045FF01231A46FFF79DB9494DDFF806
:100E780044A1DFF84481DFF844919FED478A05F1EA
:100E880020060DE0FCEEE77AC7ED097AB98C20461A
:100E9800043503F02CFFAE420AF1180A3FF481A989
:100EA8009AF811100029F2D098F80030D5ED007AA0
:100EB800012BE7D1D9F80030DB0441F17982F5EE56
:100EC800407AF1EE10FA41F0078340F2DC51DEE798
:100ED800324B2046196803F0F3FE314B204619883F
:100EE80003F005FF01231A46FFF75DB92D4D23686E
:100EF8002A68591C127821601A702B682268997820
:100F0800531C2360002311702A6821681A44013396
:100F18005279481C032B20600A70F5D123682A688F
:100F2800591C127A21601A7023682A68591CD278D1
:100F380021601A7023682A68591C127921601A7076
:100F48002B682046598903F0D2FE23682A68591C69
:100F5800527A21601A702B6821685878FFF747BBCE
:100F68003C42002030350020F47500204035002038
:100F78000C42002094530020CC53002088660020A7
:100F88001C4A002060330020305400201C420020FE
:100F9800676666667033002000004042B076002025
:100FA8004C4200204C7700202C18030800640020D5
:100FB800465F0020FC5F0020E0600020946600206F
:100FC800AB4D05F16006A988204603F090FEE9883C
:100FD800204603F08CFE2989204603F088FE23680A
:100FE800AA7A591C21601A702368EA7A591C216070
:100FF8001A7055F80C1B204603F062FEB542E2D188
:10100800FFF7CFB89B4D00212368286801EB410208
:101018005E1C805C266018702B6820681344461C90
:101028005B78266003702B682068134401319B7835
:10103800421C0A2922600370E6D1FFF7B2B88E4934
:1010480052232268501C2060137011F8013F002BB6
:10105800F7D1FFF7A6B82268884B89491878551C3C
:101068002560107022685878551C25601070226819
:101078009B78501C20601370C988204603F037FE07
:1010880001231A46FFF78FB823687E4A7E491078F5
:101098007E4A5D1C2560187023688978581C20607A
:1010A800197021689078FFF7A2BA754D20462988F3
:1010B80003F01DFE6988204603F019FEA988204622
:1010C80003F015FE01231A46FFF76DB833687268FE
:1010D8009A4241F021826E4BFF221A704FF00009AC
:1010E8006C4D29F055FB494620226B4885F8009045
:1010F80030F0CBFA87F8349097F83430072B01F2A8
:10110800B182DFF8A081644E4A4697F8343003EB89
:10111800430308EBC3035B7CE3B197F8343003EB7C
:10112800430308EBC30320215B699BB197F8343074
:1011380003EB430308EBC303586946F8220002F0A7
:1011480048FF2B7856F8230003F004F92A78013277
:10115800D2B22A7097F834300133DBB287F83430D2
:1011680097F83430072BD0D92368591C21601A709E
:10117800BAF1000F3FF415A8484BCAF80030012314
:101188001A46FFF710B8FB697C681A463B7D137056
:10119800FFF7E8B9552D00F00481572D40F0328152
:1011A8004FF0FF331A46FEF7FEBF23685A1C226031
:1011B80019702988204603F09AFD2368EA78591C9B
:1011C80021601A7023682A79591C21601A702368D3
:1011D800AA79591C21601A7023686A79591C216000
:1011E8001A70FFF784BBDFF8C0A000264FF0080B89
:1011F8000136C6F120020BFA02F2A6F120032AFA00
:1012080006F848EA02082BFA03F348EA0308252EF1
:1012180008F001024FF000030BD01343E8D0F0B2FE
:101228002BF0FEFF0028E3D03146786A03F044FF34
:10123800DEE71B4B1B78DA0701F1EC800026DFF8AC
:101248006C80D7F824A0B14602E00136252E2FD0B5
:101258003146404603F03FFF0028F6D0314650465D
:1012680003F039FF002840F0838009F10109ECE719
:10127800803700203C420020FC1703082835002056
:10128800A4490020EC6300203035002040350020C0
:10129800EC2200205B360020D4690020B9530108F5
:1012A80068740020FC5F002090E33FF4FC6F00208E
:1012B8004D4B4E4EB3F85010204603F018FD4C4BE2
:1012C8001988204689B203F012FD4A4B1A68530167
:1012D80003F02001C2F340030B43C2F3800143EA49
:1012E8004103C2F3C00143EA8103C2F3401143EA58
:1012F800C10102F010021143204603F0F8FC07F187
:101308002C010422204603F0C4FC236831783A4AB1
:10131800581C2060197011886429A8BF64212046D0
:1013280003F0E5FC962D01F07B800021204603F0B8
:10133800DEFC2168B9F1190348BFA9F11203A3F330
:10134800C4034A1C226020461A460B7007F130017C
:1013580003F09FFC2368294A581C1021206019704B
:101368001188204603F0ACFC01231A46FEF71BBF88
:10137800494607F12C0003F09FFE76E7531C3360C3
:1013880013780A2B01F06D80304603F07DFC30465F
:1013980003F07AFC304603F077FC01231A46FEF787
:1013A80002BF531C33601578FF2D01F02B81FE2DF1
:1013B80001F06680304603F05CFC96E80C009B1A4E
:1013C800002B06DD531C3360137813B90B2D41F243
:1013D8000E81242D3FF6E4AE094A012322F81500B8
:1013E8001A46FEF7E0BE00BF981C002040420020CD
:1013F800E4310020C8760020E8310020CC760020B7
:10140800287600207168A5F10B008B1AEF283FF6AB
:10141800C7AE01A555F820F04B210008A911000816
:10142800A9110008A9110008A9110008A9110008AC
:10143800A9110008A9110008A9110008A91100089C
:10144800A9110008A9110008A9110008A91100088C
:10145800A9110008A9110008A9110008A91100087C
:10146800A9110008A9110008A9110008A91100086C
:10147800A9110008A9110008F7200008A9110008FF
:1014880065220008A911000843220008A9110008D4
:10149800A9110008A91100081B220008A9110008B9
:1014A800C1210008A9110008A5220008A9110008F7
:1014B8007F220008A9110008D7220008A9110008F6
:1014C8009F200008A91100084B200008A911000856
:1014D800A9110008A9110008A9110008AB0100080A
:1014E800A91100082F200008A9110008A911000857
:1014F80015200008A9110008BB1F0008A911000841
:10150800A9110008A9110008A9110008AF1F0008B7
:10151800A9110008A9110008A91100086F1F0008E7
:10152800A9110008211F0008A9110008A911000825
:10153800E71E0008A9110008A9110008A911000850
:10154800A9110008A9110008A9110008A91100088B
:10155800111E0008A9110008671D0008A91100083C
:10156800F51C0008A9110008471C0008A91100086B
:101578001F1C0008011C0008A9110008A911000877
:10158800A9110008A9110008A9110008A91100084B
:10159800A9110008A9110008A9110008A91100083B
:1015A800A9110008A9110008A9110008A91100082B
:1015B800A9110008A9110008A9110008A91100081B
:1015C800A9110008A9110008A9110008A91100080B
:1015D800A9110008A9110008A9110008A9110008FB
:1015E800A9110008A9110008A9110008A9110008EB
:1015F800A9110008A9110008A9110008A9110008DB
:10160800A9110008A9110008A9110008A9110008CA
:10161800A9110008A9110008A9110008A9110008BA
:10162800A9110008A9110008A9110008A9110008AA
:10163800A9110008A9110008A9110008A91100089A
:10164800A9110008A9110008A9110008A91100088A
:10165800A9110008A9110008A9110008A91100087A
:10166800A9110008A9110008A9110008A91100086A
:10167800A9110008A9110008A9110008A91100085A
:10168800A9110008A9110008A9110008A91100084A
:10169800A9110008A9110008A9110008A91100083A
:1016A800A9110008A9110008A9110008A91100082A
:1016B800A9110008A9110008A9110008A91100081A
:1016C800A9110008A9110008D51B0008A9110008D4
:1016D800BF1B0008A9110008A9110008A9110008DA
:1016E800A9110008A9110008A9110008A9110008EA
:1016F800A9110008A9110008A9110008A9110008DA
:10170800A9110008A9110008A9110008611B000807
:10171800A9110008291B0008A9110008451A00088A
:101728002B1A00080F1A0008A9110008F51900085B
:10173800A9110008CD190008A91100086D190008A1
:10174800A91100083D190008A9110008A9110008ED
:101758001B190008ED180008D9180008B11800086E
:10176800911800086F180008A9110008A9110008AD
:10177800A9110008A9110008A9110008A911000859
:10178800A9110008A9110008A9110008A911000849
:10179800A9110008A9110008A9110008A911000839
:1017A800A9110008A911000855180008A911000876
:1017B800A9110008FB170008A9110008A9110008C1
:1017C800A9110008A9110008A9110008A911000809
:1017D800A9110008E1170008C14B1B78DB073FF58A
:1017E800DFAC04F06FFE05F08BFC01231A46FEF710
:1017F800DABC531C336013780F2B3FF6D1AC911C25
:101808003160C3EBC303B7495078C854D01C30606B
:101818000B4491785970111D3160D1789970511D20
:1018280031601179D970911D316051791971D11DCB
:1018380031609179597102F108013160D2799A7158
:1018480014F09CFC01231A46FEF7ADBC304603F0A9
:1018580010FAA54DE881304603F00BFA0123A88160
:101868001A46FEF7A0BC304603F003FA9F4D2882C3
:10187800304603F0FEF96882304603F0FAF9012396
:10188800A8821A46FEF78FBC1346511C316013F824
:10189800020B3360D31C51783360927819F04EFEF6
:1018A80000287EF47EAC7BE41346511C31609049DD
:1018B80013F8020B087033608B4953788B70D31C74
:1018C80033608C4B92789A7001231A46FEF76BBCF2
:1018D800894B8A4918684E222DF0C2FB01231A460B
:1018E800FEF761BC1146531C3360854B11F8020B9F
:1018F8001870316051785970D11C316092789A70A3
:10190800304603F0B6F97F4A0123D0801A46FEF725
:101918004ABC304603F0ADF97A4D2880304603F0D2
:10192800A8F96880304603F0A4F90123A8801A4674
:10193800FEF739BCDFF8D88198F80030002B3EF468
:1019480030ACDFF8D0910025304603F092F91CF056
:1019580091F898F80030A9EC010A01359D42F3DBB3
:10196800FEF71FBC0D2B7FF41BAC531C336015789E
:10197800072D3FF615ACDFF8A09130464FF00C0864
:1019880003F077F908FB05F809EB0805A88030464D
:1019980003F06FF9E880304603F06BF9336828816B
:1019A8001A46591C316012F8021BA97232605B7822
:1019B800EB72304603F046F9012349F808001A464D
:1019C800FEF7F1BB531C33601078060600F1AD86B4
:1019D800434B1B78DD073EF5E4AB032828BF002006
:1019E80004F054FD01231A46FEF7DDBB3C4B1B787F
:1019F800D8073EF5D6AB04F035FE05F081FB012390
:101A08001A46FEF7D0BB364B1B78DA073EF5C9AB52
:101A18003D490A78012342F004020A701A46FEF78B
:101A2800C2BB2F4B1B78D9073EF5BBAB374A4FF4E7
:101A3800C871012311801A46FEF7B5BB092B7FF741
:101A4800AFABDFF8D8801346511CD8F8005031608E
:101A580013F8021B297033605378AB70D31C3360C2
:101A68009378642B02F10401A8BF64236B71316081
:101A7800D378642B02F10501A8BF6423AB713160F0
:101A88001379EB71931D33605379642B02F10701CD
:101A9800A8BF64232B7231609379EB7002F10803BD
:101AA8003360D3792B71304603F0E3F872683368FA
:101AB8006881D11A00290CDD591CD8F80000316062
:101AC800521A002A1978417203DD9A1C32605B7839
:101AD80043702BF01DFC01231A46FEF764BB00BFC0
:101AE800687400207438002030350020BC60002065
:101AF800EC630020403500203C4200209437030866
:101B080028350020A4490020907600206C7700201A
:101B1800194E0020FC480020803700204C77002018
:101B2800AC4B1868D31C014621329D1E356013F852
:101B3800035C0D705D1E356013F8025C4D703360F8
:101B480013F8015C8D700333934201F10301ECD16A
:101B58001BF05CFEFEF725BBC3F34705122D3FF6CD
:101B68001FABC5B107F1580307F1320903EB450A6A
:101B7800C846AAF1260A304603F07BF828F8020F77
:101B8800C245F8D1944B39F8022F23F8022FC845E3
:101B9800F9D1112D09D8914A6B00023B1344002159
:101BA800223223F8021F9A42FBD18D4901221346A3
:101BB8000A70FEF7F8BA8B4D002330462B6003F00D
:101BC80041F8012328601A46FEF7EDBA1346511C66
:101BD800316013F8025B3360D31C5078336091781E
:101BE800002D00F0AD85012D7EF4DBAA29F05CF80C
:101BF8002B462A46FEF7D7BA7B4B1B7813F0010118
:101C08007FF4CEAA531C3360107828F08FFF01238D
:101C18001A46FEF7C8BA1346511C3160734913F8C7
:101C2800020BC8703360724953784B71D31C336010
:101C3800704B9278DA7001231A46FEF7B4BA304630
:101C480003F017F8304603F014F8304603F011F8A3
:101C5800304603F019F833685E4D1946581C2A6857
:101C6800306011F8020B82F82C003160597882F844
:101C78003610D91C31609B7882F83730304603F033
:101C880003F8304603F000F8304602F0FDFF304616
:101C9800D5F8008002F0EDFFA8F83A003046D5F8F4
:101CA800008002F0E6FF33687268A8F83800D11A9D
:101CB80001290ADD591C2A6831601B7882F82E3008
:101CC800304602F0E1FF33687268D31A032B0BDD4C
:101CD8003046D5F8008002F0CCFFA8F83200304634
:101CE8002E6802F0C6FFB086286831E7531C3360BF
:101CF800384DDFF81081137888F805303046D5F86C
:101D0800009002F0B6FFA9F820003046D5F8009000
:101D180002F0AFFF72683368A9F81E00D11A0729CC
:101D280000F3E784D11A032900F3D584D21A002AD4
:101D380005DD591C2A6831601B7882F8263004F0CA
:101D4800CBFB23F063FA2C4B28681B68002B00F0B0
:101D5800AD8414F0A7FA01231A46FEF724BA1346F5
:101D6800511C3160DFF89C8013F8021B88F80210C0
:101D78003360224953780B70D31C3360204D93781D
:101D88002B71131D3360D378092BA8BF0923304664
:101D9800AB7002F06EFF336872682880D11A01298F
:101DA80005DD304602F065FF33687268E8819A42C3
:101DB80040F0878404F090FB336872689A423EF4DE
:101DC800F0A95A1C32601B78EB7001231A46FEF703
:101DD800EAB900BF3C420020D6680020D86800203D
:101DE800FC6800205047002068740020303500202F
:101DF800F47500204035002054350020243500209B
:101E0800BC600020EC630020304602F032FF05463B
:101E18001FF0E4FCFF283EF4C4A93F2D00F22E84F5
:101E280007F15802002302F8243D4FEAD50811466D
:101E380007F12C0087F82C307A6208F101081FF0AE
:101E4800ADFC97F82C305FFA88F805F00705434594
:101E580005F1010503D197F83430AB4203D0294688
:101E680040461FF0A7FC33687268D21A012A7EF731
:101E780098A95A1C07F15800326000221D7800F812
:101E88002C2D1FF07FFC97F82C30AB420AD0BA4BB0
:101E98001B683BB19A79AA4204D31B681B690BB132
:101EA800284698473368786A5A1C326000221D78A1
:101EB80087F834201FF05AFC97F83430AB423EF4D0
:101EC80070A9AD4B1B68002B3EF46BA91B685B69BE
:101ED800002B3EF466A928469847FEF762B9A74B3F
:101EE8001B78012B3EF65DA9531C10463360A44DA8
:101EF80010F8023BAB70D31CC91A3060012992F864
:101F080001E0336040F32284304602F0B2FE012340
:101F180028801A46FEF747B9531C336092F80080B0
:101F2800B8F1110F3FF63CA9931C3360954D5378D7
:101F380005F81830304602F09CFE40F6CA03984275
:101F4800A8BF184640F2EE23984205EB4805B8BFF3
:101F580018460123A0F2EE211A46192091FBF0F150
:101F68006970FEF720B91346511C3160864D13F88D
:101F7800021B2971336053786B71304602F079FE89
:101F8800336828805A1C32601B78AB71304602F0E7
:101F980070FE336868805A1C32601B78EB7101232D
:101FA8001A46FEF700B903F03BFA01231A46FEF77A
:101FB800FAB8531C3360754B1278DFF8F8811A7041
:101FC8000023C8F80030304602F03CFE3368D8F8E9
:101FD80000206F496F4D10435A1CC8F8000032604A
:101FE8001B780B72304602F044FE2860304602F03F
:101FF80040FE6860304602F03CFEA860304602F0C1
:1020080038FE304602F035FEFEF7CBB8624B02F1DF
:1020180008010132326012F8010C03F8010F9142F5
:10202800F7D1FEF7BEB81346511C31605B4913F86F
:10203800020B8870336053784B7001231A46FEF701
:10204800B2B80721B3FBF1F1C1EBC1055B1B7FF40B
:10205800A7A8C9B201F1FF395FFA89F900293EF44E
:10206800A0A8DFF83CA109F101091D46531C336003
:1020780092F900104A4B4FF0000893F902208A4267
:1020880003F1080300F07C8208F10108B8F1050F9C
:10209800F3D1FFF785B8531C336013780E2B3FF646
:1020A8007FA8911C31605578032D3FF679A83D48EB
:1020B800062101FB03F1431802F1030E5D71C6F816
:1020C80000E095784554111D3160D1785970511D43
:1020D800316011799970911D31605179D970D11D94
:1020E800316092791A7101231A46FEF75CB8531CC5
:1020F80033601578132D3FF653A8931C336050783E
:102108007A6226F067FE00283FF44AA87A6A264BCE
:10211800017803F82510D11C316003EB8503917811
:102128005970111D3160D0789870501D30601F496A
:102138001279DA7008682BF079F801231A46FEF74D
:1021480032B81B49102B4FF0000228BF10230A6039
:102158004A608A60CA600A74002B3EF422A832687A
:10216800013913440132326012F8010C01F8010FF1
:102178009342F7D1FEF715B8384200209544002065
:10218800A4760020A06A0020C049002070350020F5
:1021980020680020883100201F6800204C3500206E
:1021A800947000205C470020743500203C420020D9
:1021B80024420020A8440020531CBB4D33601378F0
:1021C8002B72304602F055FDA883304602F051FDCF
:1021D8002883304602F04DFD32686883531C336013
:1021E8001278EA747268D31A032B00F3D982336821
:1021F800D11A052900F3C482D21A002A7DF7D1AF7B
:102208005A1C32601B7885F8213001231A46FDF7E5
:10221800CABF531C3360A54815780570C91A002930
:102228007DF7BFAF931C33605278003218BF01228C
:10223800012342701A46FDF7B6BF304602F019FD79
:102248009B4D2860304602F014FD6860304602F06D
:1022580010FD0123A8601A46FDF7A5BF954D002380
:102268002B60304602F0EEFC2A68012302432A6004
:102278001A46FDF798BF511C316015781F2D3EF6A0
:102288008FAF052B7EF48CAF304602F0DBFC8A4B17
:1022980043F825001EF0F4FFFDF783BF864D05F1D6
:1022A8004008304602F0E5FC3368A5F88000591C68
:1022B8001A46316012F8021B85F8821032605B788A
:1022C80085F883300435A845EBD1FDF76ABF531C68
:1022D8003360754B12785A7501231A46FDF763BFB0
:1022E8001346511C3160754D13F8021B6970336039
:1022F80053782B70D31C33609378AB70304602F060
:10230800B8FC336828811A46591C316012F8021B40
:10231800697132605B78AB7101231A46FDF743BFE0
:10232800674B3A6A9B68D4F800905A44934280F00D
:1023380083803A6AA3EB020803F010F84246494644
:10234800386A03F08BF8236803442360002D3DF4BA
:1023580028AF86427DF725AF002100E023680130D1
:102368005A1CB04222601970F8D1FDF71ABF002D2F
:10237800D6D15946204602F0BAFC23685A1C22607E
:102388001D704F4B26689D683B6A0BEB0302AA42FF
:1023980000F2E88102F0E2FF5A463146386A03F05B
:1023A8005DF822680123024422601A46FDF7FBBE4D
:1023B800F4EEC87AF1EE10FA80F207814FF47A71E0
:1023C800FEF765BD236898F802103E4A581C206045
:1023D800197023681278591C21601A70FEF72BBAFD
:1023E8004FF00808FEF7E0BC304602F042FC3268C5
:1023F80071689142834640F0B980064600257B6AA1
:10240800FEF71DB821680123CA1822601A46087011
:10241800FDF7C9BE7B6B43F001037B63FEF70EBF7C
:1024280023680322591C21601A7023687278591C8A
:1024380021601A70FEF77DBF02F090FF5A464946A8
:10244800386A03F00BF823680344236081E73046B9
:1024580002F00FFC1C4DFDF7BFBF4FF00408FEF75C
:10246800A3BC931C3360194B51781970D11C31608F
:1024780091785970111D3160D2789A70FDF791BE2C
:10248800931C33605578022D3EF68AAE304602F032
:10249800F0FB0F4A02EB45024FF0FF33A2F85C0055
:1024A8001A46FDF780BE00BF206800207035002066
:1024B80088310020A8440020E440002094760020C1
:1024C800581C0020243500202035002067430020B8
:1024D8002876002000E08244F4EEC87AF1EE10FA83
:1024E8003EF5F3AC1FED057AF4EEC77AFDEEE77A18
:1024F800F1EE10FA17EE901A00F2A5806FF4F97356
:10250800303903FB01F140F2E73391FBF3F101F2BB
:10251800DB5189B2FEF7BBBC5A1C19463260B04881
:1025280011F8022B027031605B784370042A06D9D7
:10253800FF2A3EF4D3AD21680020FEF758B8A94918
:102548000978994203D8022AF5D1FF2BF3D12268E2
:102558000123D11821601370BAF1000F3DF421AEA8
:10256800A14ACAF800201A46FDF71DBE531C336065
:1025780013780033064618BF01230025FDF75FBF17
:102588000AEBC80B30468BF8021002F072FB336876
:102598002AF838001A46591C316012F8021B8BF8C9
:1025A800031032605A788BF80420DA1C32609A786B
:1025B8008BF806201A1D32600135DB788BF8053060
:1025C800A9457FF453ADFDF7ECBDFDEEE77A40F287
:1025D800E73317EE901A303903FB01F140F2CF735D
:1025E80091FBF3F101F2E93189B2FEF750BC7F4B60
:1025F80000301D4418BF0120012385F84A001A46FF
:10260800FDF7D1BD304602F03FFB3368774D1A46DF
:10261800591C316012F8021B85F85B1032605B7838
:1026280085F85A30304602F024FBA5F856003046AB
:1026380002F01FFB304602F01CFB0123A5F85800EE
:102648001A46FDF7B0BD40F2F313A1F5836103FB11
:1026580001F140F2E73391FBF3F101F2DD5189B268
:10266800FEF715BC4A46FEF77FBD7D62AA46FDF718
:102678007FBFDA46C7F824B0FDF77ABF07F1340305
:1026880018467B621FF066F8BB8EAB423FF4EBAB9B
:10269800574B1B68002B3FF4E6AB1B689B69002B6C
:1026A8003FF4E1AB28469847FFF7DDBB514B524A50
:1026B800524853491A60012302600A601A46FDF71E
:1026C80072BD5A1C32601B78003318BF012388F88A
:1026D8000730FFF76FBB304602F0CBFAA8F80E00C0
:1026E800304602F0C6FA33687268A8F81000FFF79F
:1026F8001DBB304602F0BDFAA8F80A00304602F0C9
:10270800B8FAA8F80C003046D5F8009002F0B1FAF3
:10271800A9F822003046D5F8009002F0AAFA3368EA
:102728007268A9F82400FFF7FDBA00F07F000328BB
:1027380028BF002028F0D4FA01231A46FDF733BD3C
:1027480013F046FF01231A46FDF72DBD2D4B907857
:102758001988012311FB0EF11A4691FBF0F129802B
:10276800FDF721BD3B6AED1A02F0F8FD2A46314615
:10277800386A02F073FE236803442360FDF711BD35
:102788005A1C32601B78EB72304602F05BFA3368F1
:10279800E8605A1C32601B782B74336872682BE52A
:1027A800304602F066FAA884304602F062FA3368CE
:1027B8007268E884D11A03297FF71AAD1A46591CA2
:1027C800316012F8021BA97732605B7885F82030F7
:1027D800304602F04EFA33687268688408E500BF34
:1027E800EC220020194E0020E55D00082876002024
:1027F80038420020EC380020CF2B00084039002058
:10280800A8390020A03300200A4B30B503F1140486
:1028180093F900205D78072AC8BF143A8118043359
:102828000D7313F8025C855413F8012C0A76A34241
:10283800EED130BD401C030803682DE9F041DF6983
:102848001FB13B46BDE8F0411847002A164611DD86
:1028580004460D460E4400E023689B6820469847CE
:102868000028F9D0236815F8011B1B6820469847F3
:10287800AE42F1D1BDE8F0810023232202704370FB
:102888008370C37070472D2343702E2303712F2349
:10289800C3717047F0B484894FF6FF764FF47A74A9
:1028A8000BB300292ED00F78013101E0B44217D0C4
:1028B8000589013CAD07A4B2F8D507734FF47A74C3
:1028C80002E0BCB2B4420BD00589ED0704F1FF3732
:1028D800F7D5057BEDB20AB115700132013BDFE790
:1028E800094B984202D00120F0BC7047074A538B2D
:1028F80001339BB25383508B80B2003018BF012044
:10290800F0BC7047FF27D3E7003800404C70002028
:1029180040F2E93300E09BB10289013B12F0020F5B
:102928009BB2F8D0017340F2E93300E043B1028969
:10293800013B12F0010F9BB2F8D0007BC0B2704788
:10294800064B984201D0FF207047054A538B01334C
:102958009BB25383508BC0B2704700BF0038004011
:102968004C700020002870B51EDB0928044620DDC5
:10297800012303EB83035B00B0FBF3F2092AF8D8C9
:102988007BB10E4EB4FBF3F00928CCBF572230229E
:10299800A6FB03E5024403FB1044EB0801F8012BF6
:1029A800F0D100230B7070BD2D230B704042013114
:1029B800DBE7303001F8010BF3E700BFCDCCCCCC1E
:1029C800884230B44FF001042ED301FB04F4B0FB6D
:1029D800F4F58D42F9D284B1AAB901E0B0FBF4F55F
:1029E800092DCCBF572230222A4404FB150003F8D6
:1029F800012BB4FBF1F4002CF0D100221A7030BC8A
:102A08007047B0FBF4F5092DCCBF372230222A4499
:102A180004FB150003F8012BB4FBF1F4002CF0D1F2
:102A280000221A7030BC70470546002AEBD1D7E760
:102A380003685A1C0260197070472DE9F047089C1A
:102A48002578002B804689460CBF4FF0200A4FF0AE
:102A5800300A661C35B3002A29DD334601E00246F8
:102A680098B113F8011B501E0029F8D1971E60B1C8
:102A78003D46013D51464046C8476B1C002BF8DCDB
:102A8800257827EAE770013055B1041B29464046EE
:102A9800C847301916F8015B002DF7D1BDE8F0875B
:102AA800BDE8F087002A04DC2846BDE8F08700204E
:102AB800EBE7571EDCE783684268D0ED037A00EB4A
:102AC80083010133934281ED040A836004BF00232C
:102AD800836000EB830393ED047A036870EE277A32
:102AE8009A42C0ED037A77EEC77AC0ED037A0CDA22
:102AF800013307EE103AF8EEC76AB7EE007A87EEB0
:102B0800A60A036030EE070A704707EE102AB8EEEF
:102B1800C77A87EE870A704790ED057A90ED004AEC
:102B2800D0ED066AD0ED014AD0ED047A90ED035A53
:102B3800D0ED025AA4EE007AB0EE406AB0EE470A31
:102B4800B0EE667AA6EE247A67EEC07AA0EE457AF1
:102B5800E6EE257A80ED057AC0ED067A7047D0ED6D
:102B6800057A90ED013AD0ED003AD0ED064A90EDA5
:102B7800024A90ED077A90ED035A90ED086AD0ED7D
:102B8800045AC0ED067AF0EE406A27EE830AC0EDDB
:102B9800056AA3EEA60A80ED087AA4EE240AA5EE3B
:102BA800470AA5EEC60A80ED070A7047D0ED007AFD
:102BB80090ED017A30EE670AE7EE007AB0EE670A28
:102BC800C0ED007A704770470A44914214D030B47F
:102BD8000139551E41F2210211F8014F082380EAFC
:102BE800042004044CBF82EA40004000013B80B24C
:102BF800F7D18D42F0D130BC704750F8043C012227
:102C080080F84520103803B11847704790F82030F5
:102C180033B1012B03D14FF40063838270477047AF
:102C28004FF48063838270472DE9F04FDFF81CB2C0
:102C3800DFF81CE2BBF80020DEF80060BBF90430C6
:102C4800BBF90250BBF90A80C2EB261404FB04F45A
:102C580024135200C2EBE60203FB04F305FB02F265
:102C68009B1303EBE223B3F5FA364FEAE37589B019
:102C780045F1FF373246A6FB0645CDE9024502FB82
:102C880007F205EB4202CDE90467029EBBF9084052
:102C9800039208FB02FC4FEAE87906FB09CC3A46A6
:102CA800A8FB0689049ECBF81830E51704FB02F24E
:102CB80006FB0522A4FB0667E14417444FEA1822E5
:102CC80042EA096200924FEA292201923D03DDE9B6
:102CD8000078340345EA16553F19BBF8066006909C
:102CE80048EB05083C1C48F5004503EB8302A4FBB0
:102CF800068906FB0599803213124FEA69064FEAE6
:102D0800E977079356EA07038A4600F09280DDE9DF
:102D18000489BBF90E20DEF80440BBF910004946CF
:102D2800C4F5801ED317DDE9024502FB01F108FB5B
:102D38000311A2FB08230B444FEA43492B46C11752
:102D480000FB03F304FB0133A0FB0401BBF90C40B7
:102D58001944E30001937346DC170023009349EA02
:102D6800D2394FEA4248DDE9002310EB080041EB75
:102D78000901E50712184FEACE744B4145EA5E0592
:102D8800A41A65EB0305221945EB050312196B41DB
:102D980099019001801841EA926159418B008200A3
:102DA80043EA9073101943EB05018B00820043EA54
:102DB800907310460019194632463B4669412BF07C
:102DC80095FDBBF916204C13450B45EAC14502FB9E
:102DD80004F6D31705FB0366A2FB05233344BBF9AE
:102DE800146002FB04F405FB034406FB01FEA2FB8E
:102DF8000523F717234400FB07EE540EA6FB0067D4
:102E0800774444EAC3144FEAD64800194FEA636589
:102E180048EA473869414FEAE74918EB0008BBF927
:102E2800124049EB01094FEA182646EA09662001D3
:102E38003618069B0BB1360A1E60BAF1000F02D095
:102E4800079BCAF8003009B0BDE8F08F9040002019
:102E5800F02200207047704770B5044682B01430E5
:102E6800E56D06236A464321A847B0B19DF80400E2
:102E78009DF800609DF801109DF802509DF8032010
:102E88009DF8053041EA062143EA002342EA05227B
:102E9800A187E287A4F84030012002B070BD70B568
:102EA800044682B00830656A06236A463B21A84773
:102EB800A8B19DF804009DF800609DF801109DF8E8
:102EC80002509DF803209DF8053041EA062143EAA7
:102ED800002342EA0522E18222836383012002B0B3
:102EE80070BD70B40468037B2268022101FA03F301
:102EF8001A4213D042690A49582000FB02124FF6C1
:102F0800FE7650685289C568006829683140296092
:102F1800C168D24392B20A40C260636070BC704715
:102F2800E460002030B4094B1C7864B1084B0025DC
:102F380003EBC4041A6899885562D06808330143C2
:102F4800A342D160F6D130BC704700BFA463002013
:102F5800A863002010B40268047B11680223A34010
:102F6800194209D00649406800240C7001684FF6E0
:102F7800FE742140016053605DF8044B704700BF48
:102F8800E7410020F0B4334C00EB800004EB8004F0
:102F98006468002C5BD0304E49004FF42040CDB21D
:102FA800B060A169090444D460682C4F45F0807171
:102FB800384041F4903101434FF420406160B060E3
:102FC80003E0411E002838D00846A1698F07F8D5CC
:102FD8004FF42040A262B06002E0421E68B310467F
:102FE800A2691106F9D562681C4945F0007545F4D7
:102FF80080350A4015434FF420406560B06002E018
:10300800421ED0B11046A2699207F9D5A362A369FE
:103018004FF420409B06B06005D4431E68B11846A3
:10302800A3699B06F9D52023B060E3610120F0BCB9
:103038007047411E08B10846B3E7094A13880133AF
:103048009BB24FF0FF31B1601380F0BC704720464F
:10305800F0BC7047E8540020F0220020009800FCE3
:10306800E4310020134600200A4668218AE730B57B
:103078000446C06C61710368A26823F00103036011
:1030880087B0A379009213F004023DD04FF4805228
:1030980013F00203019244D102934FF4806300229B
:1030A800039311F00103059237D1049308238D0788
:1030B800694648BF049320F0AFFC6079E36CA179BE
:1030C80000F00202002A15BF4FF440324FF480325C
:1030D8004FF40034002410F0010F586808BF22464E
:1030E800CC074CBF024320EA02025A609A680907DB
:1030F8004CBF42F0080222F008029A601A6842F0B7
:1031080001021A6007B030BD13F0020301920BD020
:103118004FF4005513460295C1E7042304930C238A
:10312800C5E74FF40053B7E70293B8E710B5044674
:10313800C06CA160036823F001030360A37986B023
:1031480013F00402009141D04FF4805213F00203AF
:10315800019244D102934FF4806362790393D107BB
:103168004FF000030493059345BF042304930823F9
:103178000C236946920748BF049320F04DFC607900
:10318800E36CA17900F00202002A15BF4FF4403227
:103198004FF480324FF40034002410F0010F5868C7
:1031A80008BF2246CC074CBF024320EA02025A60FD
:1031B8009A6809074CBF42F0080222F008029A6098
:1031C8001A6842F001021A6006B010BD13F002033B
:1031D800019207D04FF4005113460291BDE74FF416
:1031E8000053B7E70293B8E7002326220360027072
:1031F80027228270012243600271837170472DE992
:10320800F341056906460F467DBBD0F80080C8F338
:103218000A0323B30023D6F80080019322F018FF95
:10322800042819D1214C236943F001032361BBB25F
:10323800A8F8003022F00CFF04282ED108F1020370
:103248000193019B3F0C1F8022F002FF2369042891
:1032580023F00103236125D06FF0010505E022F07A
:10326800F7FE042805D04FF0FF35284602B0BDE828
:10327800F0810E4C236943F002032361C4F81480E3
:10328800236943F04003236122F0E2FE2369042806
:1032980023F002032361BDD0E5E7236923F001038E
:1032A8002361D9E7336804333360DEE70020024046
:1032B800F8B504460D468E180027B54201D120699D
:1032C800F8BDE368591CE160234415F8012B1A7214
:1032D8000429F2D1A1682046FFF791FFE760206139
:1032E800EBE710B490E80600047B40690223A34092
:1032F8004B6013685DF8044B4FF6FE710B4013608A
:1033080004F024BC03685B6A03B11847704703687C
:103318001B6A03B11847704703682DE9F041DF695C
:103328001FB13B46BDE8F0411847002A164611DD9B
:1033380004460D460E4400E023689B6820469847E3
:103348000028F9D0236815F8011B1B682046984708
:10335800AE42F1D1BDE8F08103689B691847036864
:103368005B6918470368DB68184703689B68184758
:1033780003685B68184703681B681847014B18689F
:10338800F9E700BF846F0020054B53F8203033B1B4
:103398001A689B88918A0B4218BF1B049361704777
:1033A8001455002003682DE9F04F03F13845644EA9
:1033B800AD0A0124755D05F01F066D09022D04FA9A
:1033C80006F400F0A280032D00F0A480012D52D055
:1033D8008088B0FA80F4C4F11F04A4B2E50803EBB6
:1033E800850504F007042E6AA4000F27A74026EAE3
:1033F80007062E622E6A01F0030702FA04F47A1E09
:103408003443012AC1F3810CC1F300182C62C1F3C3
:10341800411135D9C60700F19780850700F1A380CF
:10342800440700F1B180020700F1BF80C60600F131
:10343800CD80850600F1DB80440600F1E9800206B4
:1034480000F1F780C60500F10581850500F11381BB
:10345800440500F12181020500F12F81C60400F125
:103468003D81850400F14B81440400F15981020437
:1034780055D4BDE8F08F334D6E6934436C61A7E7CE
:10348800002422464FF0010E4FF0030904E00132F8
:10349800102A04F10204ECD00EFA02F636EA00050E
:1034A800F5D1D3F808A009FA04F5ED430AEA050AAC
:1034B800C3F808A0D3F808B00CFA04FA4AEA0B0AD1
:1034C800C3F808A0B3F804A01FFA8AFA2AEA060685
:1034D8009E80B3F804A008FA02F646EA0A06B6B2D5
:1034E8009E801E682E401E60D3F800A007FA04F6DE
:1034F80046EA0A061E60D3F80CA001FA04F605EAAB
:103508000A0A46EA0A05DD60C1E70E4DAE69344392
:10351800AC615DE70B4DEE693443EC6158E71A681E
:1035280022F040421A601A6842EA87771F60DA6818
:1035380022F0404242EA8171D960BDE8F08F00BFB5
:10354800D43F0308001002401A6822F003021A60F0
:103558001A683A431A60DA6822F003020A438507B8
:10356800DA607FF55DAF1A6822F00C021A601A68FB
:1035780042EA87021A60DA6822F00C0242EA810203
:103588004407DA607FF54FAF1A6822F030021A60FC
:103598001A6842EA07121A60DA6822F0300242EA30
:1035A8000112DA6002077FF541AF1A6822F0C00203
:1035B8001A601A6842EA87121A60DA6822F0C002B2
:1035C80042EA8112C606DA607FF533AF1A6822F440
:1035D80040721A601A6842EA07221A60DA6822F40E
:1035E800407242EA01228506DA607FF525AF1A6843
:1035F80022F440621A601A6842EA87221A60DA687E
:1036080022F4406242EA81224406DA607FF517AF6D
:103618001A6822F440521A601A6842EA07321A609D
:10362800DA6822F4405242EA0132DA6002067FF593
:1036380009AF1A6822F440421A601A6842EA8732CF
:103648001A60DA6822F4404242EA8132C605DA603A
:103658007FF5FBAE1A6822F440321A601A6842EA13
:1036680007421A60DA6822F4403242EA01428505CC
:10367800DA607FF5EDAE1A6822F440221A601A6803
:1036880042EA87421A60DA6822F4402242EA81421A
:103698004405DA607FF5DFAE1A6822F440121A603A
:1036A8001A6842EA07521A60DA6822F4401242EABB
:1036B8000152DA6002057FF5D1AE1A6822F44002A1
:1036C8001A601A6842EA87521A60DA6822F44002DD
:1036D80042EA8152C604DA607FF5C3AE1A6822F066
:1036E80040721A601A6842EA07621A60DA6822F0C1
:1036F800407242EA01628504DA607FF5B5AE1A6865
:1037080022F040621A601A6842EA87621A60DA6830
:1037180022F0406242EA81624404DA607FF5A7AE93
:103728001A6822F040521A601A6842EA07721A6050
:10373800DA6822F0405242EA0172DA6097E60368DA
:1037480003F138422DE9F04F920A584DAA5C02F075
:103758001F0552090124022A04FA05F400F08C809E
:10376800032A00F08E80012A3CD001F003077A1E5C
:10377800012AC1F3810CC1F300188088C1F34111FB
:1037880035D9C60700F19680850700F1A280440765
:1037980000F1B080020700F1BE80C60600F1CC80BF
:1037A800850600F1DA80440600F1E880020600F19F
:1037B800F680C60500F10481850500F112814405F3
:1037C80000F12081020500F12E81C60400F13C8140
:1037D800850400F14A81440400F15881020455D45B
:1037E800BDE8F08F324A55692C435461BDE7002487
:1037F80022464FF0010E4FF0030904E00132102A6F
:1038080004F10204ECD00EFA02F636EA0005F5D10E
:10381800D3F808A009FA04F5ED430AEA050AC3F843
:1038280008A0D3F808B00CFA04FA4AEA0B0AC3F85D
:1038380008A0B3F804A01FFA8AFA2AEA06069E80AE
:10384800B3F804A008FA02F646EA0A06B6B29E8061
:103858001E682E401E60D3F800A007FA04F646EA58
:103868000A061E60D3F80CA001FA04F605EA0A0A53
:1038780046EA0A05DD60C1E70D4A95692C43946163
:1038880073E70B4AD5692C43D4616EE71A6822F0B6
:1038980040421A601A6842EA87771F60DA6822F0A5
:1038A800404242EA8171D960BDE8F08FD43F0308F5
:1038B800001002401A6822F003021A601A683A439C
:1038C8001A60DA6822F003020A438507DA607FF596
:1038D8005EAF1A6822F00C021A601A6842EA870280
:1038E8001A60DA6822F00C0242EA81024407DA60C0
:1038F8007FF550AF1A6822F030021A601A6842EA5F
:1039080007121A60DA6822F0300242EA0112DA601D
:1039180002077FF542AF1A6822F0C0021A601A68DF
:1039280042EA87121A60DA6822F0C00242EA81127B
:10393800C606DA607FF534AF1A6822F440721A605E
:103948001A6842EA07221A60DA6822F4407242EAE8
:1039580001228506DA607FF526AF1A6822F44062F4
:103968001A601A6842EA87221A60DA6822F440620A
:1039780042EA81224406DA607FF518AF1A6822F419
:1039880040521A601A6842EA07321A60DA6822F46A
:10399800405242EA0132DA6002067FF50AAF1A683D
:1039A80022F440421A601A6842EA87321A60DA68DA
:1039B80022F4404242EA8132C605DA607FF5FCAE65
:1039C8001A6822F440321A601A6842EA07421A60FA
:1039D800DA6822F4403242EA01428505DA607FF56E
:1039E800EEAE1A6822F440221A601A6842EA874248
:1039F8001A60DA6822F4402242EA81424405DA6019
:103A08007FF5E0AE1A6822F440121A601A6842EA9A
:103A180007521A60DA6822F4401242EA0152DA6068
:103A280002057FF5D2AE1A6822F440021A601A68BD
:103A380042EA87521A60DA6822F4400242EA815266
:103A4800C604DA607FF5C4AE1A6822F040721A60C4
:103A58001A6842EA07621A60DA6822F0407242EA9B
:103A680001628504DA607FF5B6AE1A6822F040621A
:103A78001A601A6842EA87621A60DA6822F04062BD
:103A880042EA81624404DA607FF5A8AE1A6822F03F
:103A980040521A601A6842EA07721A60DA6822F01D
:103AA800405242EA0172DA6098E610B50409013C16
:103AB800052C17D80C4B33F8142000F00F0042FAED
:103AC80000F313F001030DD0012303FA00F00138CD
:103AD80010402AF05BFF054A054B125D104403EBCA
:103AE800C00010BD002010BDD4460308E0460308FE
:103AF800907100202DE9F04F4A484B4B4B4C4FF04A
:103B080090414FF0010A4FF002094FF004084FF0BE
:103B1800080C4FF0100E20274026802530F8022B85
:103B280012F0010F03D01960A3F804A0083312F0B3
:103B3800020F03D01960A3F80490083312F0040FA1
:103B480003D01960A3F80480083312F0080F03D0DB
:103B58001960A3F804C0083312F0100F03D01960DD
:103B6800A3F804E0083312F0200F02D019609F80F8
:103B7800083312F0400F02D019609E80083312F00B
:103B8800800F02D019609D80083312F4807F05D021
:103B98004FF4807B1960A3F804B0083312F4007F57
:103BA80005D04FF4007B1960A3F804B0083312F471
:103BB800806F05D04FF4806B1960A3F804B0083308
:103BC80012F4006F05D04FF4006B1960A3F804B02D
:103BD800083312F4805F05D04FF4805B1960A3F8B6
:103BE80004B0083312F4005F05D04FF4005B19608D
:103BF800A3F804B0083312F4804F05D04FF4804B7B
:103C08001960A3F804B00833D20B04D04FF4004273
:103C180019609A80083301F58061A1427FF47EAF74
:103C2800BDE8F08FD44603089071002000180048C2
:103C3800002867D003682DE9F04F03F138445C4E43
:103C4800A40A0125345D04F01F066409022C05FA54
:103C580006F558D0032C00F0A580012C58D0808898
:103C6800B0FA80F4C4F11F04A4B2E50803EB85059B
:103C780004F007042E6AA4000F27A74026EA0706C7
:103C88002E622E6A01F00307A2407C1E3243012CEB
:103C9800C1F3810CC1F300182A62C1F341113CD968
:103CA800C60700F18980850700F19580440700F177
:103CB800A380020700F1B180C60600F1BF80850627
:103CC80000F1CD80440600F1DB80020600F1E980B6
:103CD800C60500F1F780850500F10581440500F16E
:103CE8001381020500F12181C60400F12F818504AA
:103CF80000F13D81440400F14B81020400F1598137
:103D0800BDE8F08F70472B4CA6693543A561A6E73F
:103D1800284C666935436561A1E7002422464FF0C7
:103D2800010E4FF0030904E00132102A04F10204E5
:103D3800E6D00EFA02F636EA0005F5D1D3F808A067
:103D480009FA04F5ED430AEA050AC3F808A0D3F80E
:103D580008B00CFA04FA4AEA0B0AC3F808A0B3F848
:103D680004A01FFA8AFA2AEA06069E80B3F804A07D
:103D780008FA02F646EA0A06B6B29E801E682E4087
:103D88001E60D3F800A007FA04F646EA0A061E6089
:103D9800D3F80CA001FA04F605EA0A0A46EA0A056D
:103DA800DD60C1E7034CE6693543E56157E700BFCD
:103DB800D43F0308001002401A6822F003021A6078
:103DC8001A683A431A60DA6822F003020A43850740
:103DD800DA607FF56BAF1A6822F00C021A601A6875
:103DE80042EA87021A60DA6822F00C0242EA81028B
:103DF8004407DA607FF55DAF1A6822F030021A6076
:103E08001A6842EA07121A60DA6822F0300242EAB7
:103E18000112DA6002077FF54FAF1A6822F0C0027C
:103E28001A601A6842EA87121A60DA6822F0C00239
:103E380042EA8112C606DA607FF541AF1A6822F4B9
:103E480040721A601A6842EA07221A60DA6822F495
:103E5800407242EA01228506DA607FF533AF1A68BC
:103E680022F440621A601A6842EA87221A60DA6805
:103E780022F4406242EA81224406DA607FF525AFE7
:103E88001A6822F440521A601A6842EA07321A6025
:103E9800DA6822F4405242EA0132DA6002067FF51B
:103EA80017AF1A6822F440421A601A6842EA873249
:103EB8001A60DA6822F4404242EA8132C605DA60C2
:103EC8007FF509AF1A6822F440321A601A6842EA8C
:103ED80007421A60DA6822F4403242EA0142850554
:103EE800DA607FF5FBAE1A6822F440221A601A687D
:103EF80042EA87421A60DA6822F4402242EA8142A2
:103F08004405DA607FF5EDAE1A6822F440121A60B3
:103F18001A6842EA07521A60DA6822F4401242EA42
:103F28000152DA6002057FF5DFAE1A6822F440021A
:103F38001A601A6842EA87521A60DA6822F4400264
:103F480042EA8152C604DA607FF5D1AE1A6822F0DF
:103F580040721A601A6842EA07621A60DA6822F048
:103F6800407242EA01628504DA607FF5C3AE1A68DE
:103F780022F040621A601A6842EA87621A60DA68B8
:103F880022F0406242EA81624404DA607FF5B5AE0D
:103F98001A6822F040521A601A6842EA07721A60D8
:103FA800DA6822F0405242EA0172DA6002047FF5D0
:103FB800A7AE1A6822F040421A601A6842EA877768
:103FC8001F60DA6822F0404242EA8171D960BDE898
:103FD800F08F002852D0036803F138422DE9F04FE2
:103FE800920A514DAA5C02F01F0552090124022AC7
:103FF80004FA05F443D0032A00F09080012A43D044
:1040080001F003077A1E012AC1F3810CC1F30018DD
:104018008088C1F341113CD9C60700F18980850722
:1040280000F19580440700F1A380020700F1B180F8
:10403800C60600F1BF80850600F1CD80440600F178
:10404800DB80020600F1E980C60500F1F7808505EE
:1040580000F10581440500F11381020500F1218179
:10406800C60400F12F81850400F13D81440400F16C
:104078004B81020400F15981BDE8F08F70472B4A4B
:1040880095692C439461BBE7284A55692C435461D0
:10409800B6E7002422464FF0010E4FF0030904E072
:1040A8000132102A04F10204E6D00EFA02F636EACA
:1040B8000005F5D1D3F808A009FA04F5ED430AEA9A
:1040C800050AC3F808A0D3F808B00CFA04FA4AEABB
:1040D8000B0AC3F808A0B3F804A01FFA8AFA2AEA60
:1040E80006069E80B3F804A008FA02F646EA0A0615
:1040F800B6B29E801E682E401E60D3F800A007FA54
:1041080004F646EA0A061E60D3F80CA001FA04F683
:1041180005EA0A0A46EA0A05DD60C1E7034AD569E5
:104128002C43D4616CE700BFD43F03080010024061
:104138001A6822F003021A601A683A431A60DA68A9
:1041480022F003020A438507DA607FF56BAF1A682D
:1041580022F00C021A601A6842EA87021A60DA68CA
:1041680022F00C0242EA81024407DA607FF55DAF73
:104178001A6822F030021A601A6842EA07121A60B6
:10418800DA6822F0300242EA0112DA6002077FF5AB
:104198004FAF1A6822F0C0021A601A6842EA871202
:1041A8001A60DA6822F0C00242EA8112C606DA60B2
:1041B8007FF541AF1A6822F440721A601A6842EA21
:1041C80007221A60DA6822F4407242EA0122850660
:1041D800DA607FF533AF1A6822F440621A601A6811
:1041E80042EA87221A60DA6822F4406242EA8122AF
:1041F8004406DA607FF525AF1A6822F440521A6047
:104208001A6842EA07321A60DA6822F4405242EA2F
:104218000132DA6002067FF517AF1A6822F44042CD
:104228001A601A6842EA87321A60DA6822F4404251
:1042380042EA8132C605DA607FF509AF1A6822F4CE
:1042480040321A601A6842EA07421A60DA6822F4B1
:10425800403242EA01428505DA607FF5FBAE1A6812
:1042680022F440221A601A6842EA87421A60DA6821
:1042780022F4402242EA81424405DA607FF5EDAE3D
:104288001A6822F440121A601A6842EA07521A6041
:10429800DA6822F4401242EA0152DA6002057FF538
:1042A800DFAE1A6822F440021A601A6842EA87529E
:1042B8001A60DA6822F4400242EA8152C604DA60DF
:1042C8007FF5D1AE1A6822F040721A601A6842EA85
:1042D80007621A60DA6822F0407242EA01628504D5
:1042E800DA607FF5C3AE1A6822F040621A601A6875
:1042F80042EA87621A60DA6822F0406242EA816222
:104308004404DA607FF5B5AE1A6822F040521A60AC
:104318001A6842EA07721A60DA6822F0405242EAE2
:104328000172DA6002047FF5A7AE1A6822F04042F3
:104338001A601A6842EA87771F60DA6822F04042FA
:1043480042EA8171D960BDE8F08F10B103688288B4
:104358001A85704710B1036882889A61704710B552
:10436800014600BF074C23689868FFF7EEFF2368F3
:104378005868FEF7CDFA23689868FFF7EBFF00BF8F
:1043880010BD00BF7C70002038B100298388026806
:1043980014BF002110218B409361704710B40A4B61
:1043A8000A4A1C7801238340234052F8200029B987
:1043B800B3FA83F149095DF8044BE5E7191C18BF06
:1043C80001215DF8044BDFE710550020145500204B
:1043D80030B1036882881B8A1A4214BF012000206A
:1043E800704770B5044690F85900002833D104F19D
:1043F8001405236E80226B2128469847642003F019
:1044080007FA236E284603226B219847236E94F8F7
:1044180054201921284698470F2003F0F9F9236EF4
:1044280094F8522028461A219847236E28461822C5
:104438001B219847236E284618221C219847236E73
:1044480028460222372198472846236E0122382120
:10445800BDE870401847FFF728FB0546FFF7B8FF8F
:1044680001460028C3D1D5B12023E871AB71284695
:10447800FFF7AFFD2146104B41F8103F284624F0C6
:10448800DDFCAB88B3FA83F3C3F11F035A1CAED02B
:1044980001229A4009490B6813430B60A7E7294694
:1044A800FFF797FD2146044B41F8103F284624F0BA
:1044B800C5FC0122EEE700BF032C00080004014000
:1044C8002DE9F0410B4E346873691C400FD0DFF8BA
:1044D80028800127B4FA84F3C3F11F0307FA03F510
:1044E80058F8230003689847AC437561F2D1BDE8DA
:1044F800F08100BF00040140047000202DE9F04164
:104508000B4E346873691C400FD0DFF828800127F0
:10451800B4FA84F3C3F11F0307FA03F558F823002C
:1045280003689847AC437561F2D1BDE8F08100BFDC
:1045380000040140047000202DE9F0410B4E34685E
:1045480073691C400FD0DFF828800127B4FA84F380
:10455800C3F11F0307FA03F558F8230003689847C7
:10456800AC437561F2D1BDE8F08100BF00040140A1
:10457800047000202DE9F0410B4E346873691C402B
:104588000FD0DFF828800127B4FA84F3C3F11F03A2
:1045980007FA03F558F8230003689847AC43756198
:1045A800F2D1BDE8F08100BF000401400470002092
:1045B8002DE9F0410B4E346873691C400FD0DFF8C9
:1045C80028800127B4FA84F3C3F11F0307FA03F51F
:1045D80058F8230003689847AC437561F2D1BDE8E9
:1045E800F08100BF00040140047000202DE9F04173
:1045F8000B4E346873691C400FD0DFF82880012700
:10460800B4FA84F3C3F11F0307FA03F558F823003B
:1046180003689847AC437561F2D1BDE8F08100BFEB
:1046280000040140047000202DE9F0410B4E34686D
:1046380073691C400FD0DFF828800127B4FA84F38F
:10464800C3F11F0307FA03F558F8230003689847D6
:10465800AC437561F2D1BDE8F08100BF00040140B0
:10466800047000200B490C4A0C4808B58B6943F0CC
:1046780001038B61136843F48053136000214022C7
:104688002DF003F8064B4FF0FF321A60C3F80320F1
:1046980008BD00BF00100240000001400470002067
:1046A8004470002003685B6A18472DE9F04104460E
:1046B80018460D461646984629F04EFC2768E672BD
:1046C8002844A07229467D69434632462046AC46B6
:1046D800BDE8F0416047036810B504461B68984779
:1046E800236820469B689847A37B0133A37310BDBA
:1046F80010B5036804469B689847FF23012263733B
:10470800227310BD427A02B9704710B50446036897
:10471800406804F10A0198470023637210BD437A88
:104728005A1C0344D2B242729972037A934200D857
:1047380002B9704710B504460368406804F10A01DD
:1047480098470023637210BD30B40B4D002305F168
:10475800140101E0272B0BD011F8132082424FEAF5
:10476800430403F10103F5D12C44607D30BC70474C
:10477800002030BC704700BF401C030870B5448857
:1047880006460D46C4F30B042246002128462CF0A9
:104798007CFF3369094A934209D3094A934206D2F6
:1047A800224628461946BDE870402AF059BC23B174
:1047B80021462846BDE87040184770BD2C8803087C
:1047C8001E890308064B07498B4202D3002318466B
:1047D80070471A88C2F30B029042F8D01433F3E7FB
:1047E800B88303082C880308024A136823EA0000E8
:1047F80010607047A8440020F8B5174D2B78A32BFC
:1048080028D16B78BE2B25D1022229464FF6FF709E
:10481800FEF7DAF9114FAC1C22884AB1A618BE423D
:1048280018D2052A16D92146FEF7CEF93446F3E701
:1048380021460222FEF7C8F90222A118FEF7C4F9A0
:104848000634074B641B1C8041F60F53C31A5842A9
:104858005841F8BD0020F8BD00F003080000040826
:10486800E63100202DE9F04FDFF848914C4F8BB02E
:104878000326A7EB09071822002104A82CF005FF3E
:10488800484BCDF8109005971A69120604D5464A88
:104898005A6002F188325A6001228DF824203422AD
:1048A800DA60424B424C1B88ADF800300222694660
:1048B80004A8FEF7FDFC022269464FF6FF70FEF7DA
:1048C80083F9DFF8F4A080464FF0000B544536D347
:1048D8000AAC002524F8245D0222214604A8FEF72C
:1048E800E7FC022221464046FEF76EF940BAC04373
:1048F800ADF80800022202A904A8FEF7D9FC07981F
:1049080060B106ABC0F10402294618442CF0BDFE84
:10491800069904A8FEF773FC079508909DF82430C3
:10492800089A23B11F490B6943F080030B61013ECC
:104938002DD0002A9FD1FFF75FFF50B32CE0658888
:104948008DF80DB0C5F30B05AB1DADF80830238805
:10495800C3F30B02ADF80A201B0B062202A904A818
:104968008DF80C30FEF7A4FC062202A94046FEF79B
:104978002BF9616880462A4604A8FEF799FC61680D
:1049880040462A46FEF720F9143480469EE7002A5E
:10499800D1D0052002F080FA0BB0BDE8F08F00BF3F
:1049A800000004080020024023016745A21C0308F8
:1049B800B883030800F003082C8803080378202B29
:1049C800024600F10100F9D0092BF7D02D2B2CD08D
:1049D8002B2B03BF5378B7EE000A0246B7EE000A46
:1049E800A3F13001C8B209289FED467A10D8F2EE3B
:1049F800046A07EE901AF8EEE77A12F8013FE7EE3C
:104A0800267AA3F13001C8B20928B0EE677AF0D946
:104A18002E2B4CD003F0DF03452B0BD0F7EE007A9A
:104A280067EE276A20EE260A70475378BFEE000A21
:104A38000246D5E710B451782D2959D02B290ABF41
:104A48009178501C901C0024A1F13003092B53D8F5
:104A5800002303EB830301EB430310F8011FA1F1CB
:104A68003002092AA3F13003F3D9B3F59A7F28BF9E
:104A78004FF49A73072B42D9DFED236A1A46F7EEF3
:104A8800007A083A072A67EEA67AFAD803F00703ED
:104A98002BB1F2EE046A013B67EEA67AFBD124B390
:104AA800C7EE276A5DF8044B20EE260A7047537854
:104AB800A3F13001C8B2092802F10102AAD8F2EE26
:104AC800046AF0EE665A07EE901AF8EEE77A12F8E2
:104AD800013F87EEA66AA3F13001C8B2092866EE45
:104AE800A56A37EE067AEED994E767EE276AD9E722
:104AF800901C91780124A7E7F7EE007ACFE7F7EE4C
:104B0800007AC5E70000000020BCBE4CB5EEC00A24
:104B1800DFED317AF1EE10FACCBF30EE270A30EE35
:104B2800670ADFED2E7A20EE270A30B5FDEEC07A4F
:104B380087B017EE904A054684EAE470002303A97B
:104B4800A0EBE4700193009302931EF041F9002C4E
:104B5800ACBF20232D2303A88DF8003029F0FCF9E1
:104B6800012803A924D002282DD0032805BF30230B
:104B7800684668468DF801302CF0ADFD684629F08E
:104B8800EBF90338C4B22246694628462CF001FEE8
:104B980000232B55284629F0DFF92E22431C2A54DE
:104BA8000DEB0401E8182CF0B3FD284607B030BD22
:104BB800302368468DF801308DF802308DF80330C7
:104BC8002CF089FDDAE7302368468DF801308DF83E
:104BD80002302CF080FDD1E76F12033A00007A44CE
:104BE8002DE9F041064615460846B6FBF2F43CB9F5
:104BF80005FB1464124B1B5D00F8013BBDE8F08116
:104C0800B4FBF2F767B90E4B05FB174705FB1464B5
:104C1800DA5D00F8012B1B5D00F8013BBDE8F0816F
:104C2800B7FBF2F8B8F1000F02D04046FFF7D8FF03
:104C380005FB1878024B13F8082000F8012BE3E76E
:104C4800B047030830B402681146531C036011F8DA
:104C5800024B0160D31C517803609378151D0560E1
:104C68001B0443EA0123D078234343EA006030BCA5
:104C780070470368591C1A46016012F8021B02604B
:104C8800587841EA0020704703685A1C0260187877
:104C9800704738B50446006815462AF0E1F92268DD
:104CA8002A44226038BD036810B40A0A5C1C0460F8
:104CB8001A7003685A1C026019705DF8044B70473B
:104CC80003685A1C026010B4197003680A0A5C1C55
:104CD80004601A7003680A0C5C1C04601A7003688C
:104CE800090E5A1C026019705DF8044B704703687E
:104CF8005A1C026019700368090A5A1C026019706C
:104D080070472DE9F047002488B080460F461E46BC
:104D1800A14605AD531C0393117839B3252933D126
:104D2800931CCDF810900393507830284ED04FF054
:104D3800000AA0F13003DBB2092B42D96C2819D044
:104D4800642800F0938024D825281CD063D95828DB
:104D580076D063281BD131784046B847039A531C54
:104D680003931178043601340029D7D1204608B0BE
:104D7800BDE8F087039B5A1C03921B78642B7CD0F8
:104D88002AD8252B54D1252140460134B847039A07
:104D9800C0E7732833D044D975284FD106F1040EE3
:104DA80030682B4600220A217646FDF709FE049A50
:104DB8000095534639464046FDF73FFE039A0444A2
:104DC800A8E704AA03A924F055FDB7E7D31C039369
:104DD80090784FF0010AACE7732B10D05BD9752B94
:104DE8003AD0782B96D1A3F15802B2FA82F2306801
:104DF80052092B4610210436FDF7E2FDD7E7336848
:104E0800049A0093394600234046FDF716FE0436FF
:104E18000444039A7EE70028B9D1204608B0BDE8CB
:104E2800F0876E28B3D1039A336804361C6071E7A3
:104E38002AD9582BD7D0632B8DD06BE77828A6D1E9
:104E4800A0F15802B2FA82F2306852092B461021BA
:104E5800FDF7B6FD0436AAE706F1040E30682B46C6
:104E680000220A217646FDF7ABFDA0E7331D306826
:104E780029461E46FDF776FD99E7331D3068294619
:104E88001E46FDF76FFD92E7002B7FF443AF2046E7
:104E980008B0BDE8F0876E2BC6D03BE70EB400B56E
:104EA80084B005AB019053F8042B0649039301A87D
:104EB800FFF727FF019B00221A7004B05DF804EB8E
:104EC80003B07047392A00080FB430B583B006AB79
:104ED8000A490B4853F8042B096800680193FFF747
:104EE80010FF084C05462068FEF739FA0028FAD06A
:104EF800284603B0BDE8304004B070475031002068
:104F080054310020846F0020DFED2B7AB4EEE70ADD
:104F1800F1EE10FA4ADDDFED296A9FED297A01E00A
:104F2800B0EE670AB4EEC70AF1EE10FA70EE667AD0
:104F3800F6DC9FED247AF4EEC77AF1EE10FA38D554
:104F4800DFED1E6A9FED207A01E0F0EE407AF4EE84
:104F5800C77AF1EE10FA37EEA60AF6D4DFED1B7A1F
:104F6800B4EEE70AF1EE10FA14DDDFED137A37EE4E
:104F7800C00A60EE006A9FED166A9FED167ADFEDB3
:104F8800167AA6EE867A20EE266AE6EE877AA6EEEE
:104F9800270A7047DFED117AB4EEE70AF1EE10FA4E
:104FA80044BFDFED087A37EEC00AE2E7F0EE407A58
:104FB800BFE7B0EE670AD1E7DB0F4940DB0FC94016
:104FC800E4CB1641DB0F49C0E4CB16C1DB0FC93F68
:104FD80092E741B99730083C15A82ABEDB0FC9BF34
:104FE80080EAE073A3EBE0738B4205DB002801DD68
:104FF800401A704702D17047002070470844704734
:1050080009B909E0194690FBF1F301FB13030846BF
:10501800002BF7D1084670470146FBE710B507EEAD
:10502800901A2DED028BB8EE678ADFED217A28EE13
:10503800008A044628EE278AB0EE480A2AF064FA65
:10504800F0EE408AB0EE480A2AF0C0F9F7EE007A8E
:105058009FED187AF0EE675AE8EE875A0023A361AD
:10506800B0EE676AC7EEA56A63612362E361A8EEE2
:10507800C76ABDEC028B77EEC07AB6EE007AF8EE1E
:10508800005A27EE877A20EE250A27EE267A26EEA2
:10509800266A67EEA67A20EE260A84ED046AC4ED35
:1050A800017A84ED007A84ED027A84ED030A10BD5A
:1050B80027D4D236F304353F10B44C09012250F8F6
:1050C800243001F01F0102FA01F10B4340F82430AB
:1050D8005DF8044B70474B0901F01F0150F823207D
:1050E800012303FA01F1114214BF1846002070474A
:1050F800074A084B10781B78074A834296BFC31AA1
:10510800C3F180030020126818441044704700BFA0
:10511800D84500205545002058350020064A074B41
:1051280010781B7883428ABFC3F18003C01AC01865
:10513800C0F17F00704700BFD845002055450020CA
:1051480030B5144C237883B01BB90120237003B009
:1051580030BD052200238DF800208DF8013000BFF6
:105168000D4D2B689868FFF7F0F82B6801AA69467F
:10517800586824F0FBF92B689868FFF7EBF800BF34
:105188009DF8053003F0010383F00100237003B09C
:1051980030BD00BF8E7000207C70002070B5064CBA
:1051A8000646256803E023685B1BB34203D8FFF774
:1051B800C7FF0028F7D070BD485500202DE9F04FF3
:1051C80089B0B2F1000A02900491039340F3B080D1
:1051D8000B46002201EB8A0153F8040B8B42024470
:1051E800FAD1039B0592002B00F09A80059B002BB7
:1051F8006AD0544B059A1B68DFF85C9100920099BD
:10520800DAB25118B1F5807F8CBFC2F58072009A6E
:1052180001924D4A92689A426DD9190C1A0A4FF0B8
:10522800020406208DF81F308DF81E208DF81D1001
:105238008DF81C40FFF7B2FF0620FFF790F8434AAD
:105248000123137000BFD9F800309868FFF77DF884
:10525800D9F8003007A95868002224F045F900243D
:10526800049D029E019FA34629684FEA84080022F4
:105278000B46013471B1B9422AD2D9F8000031681D
:105288004068FDF707FB2A68336813443360BF1A88
:10529800C5F800B0A24505F1040506F10406E3D1FE
:1052A800D9F800309868FFF755F800BF254B0199E9
:1052B80000981B68421A0092224A0B441360039A12
:1052C80032B3009A002A9AD1059809B0BDE8F08F48
:1052D800029CD9F8003054F80810586800223B4660
:1052E800FDF7D8FA54F808202B683A44DF1B44F835
:1052F80008202F60D4E70598009C1549154A001B23
:105308000590059800230B70137009B0BDE8F08F65
:10531800059B009A9B1A0593059809B0BDE8F08F84
:10532800FFF70EFF00287FF461AF039B0593CBE7DF
:10533800039C1CB9FFF704FF0594C5E700230593F8
:10534800C2E700BF58350020581C00208E7000208E
:10535800D8450020554500207C70002070B5104DC0
:10536800104E2B7831788B4284B016D00E4A0392B7
:105378001A4402928CBF0C46CA1A04A98CBFC3F106
:1053880080020024012341F8102D02A80222019472
:10539800FFF714FF002333702B7004B070BD00BFFB
:1053A80055450020D84500205845002070B5194CB7
:1053B800194D23782978994284B027D0174A039247
:1053C8001A44029234BF0E46CA1A04A934BFC3F164
:1053D80080020026002341F8102D02A8022201961F
:1053E800FFF7ECFE23781844C0B203062B7848BFB9
:1053F80080F080008342207002D0002004B070BD8D
:10540800002301202B70237004B070BD012004B06C
:1054180070BD00BF55450020D845002058450020E4
:1054280008B545F20820FFF7B9FE0620FEF797FFFA
:10543800064B0122C7201A70FEF791FF0448054960
:10544800054A002303700B70136008BD8E7000209E
:10545800D845002055450020583500202DE9F04159
:1054680082B00346060C050A032406208DF807308F
:10547800884617468DF805608DF806508DF804406B
:10548800FFF78CFEC0B100BF0D4C23689868FEF78B
:105498005CFF236801A95868002224F025F82368D6
:1054A8004246002158683B46FDF7F4F9236898689E
:1054B800FEF750FF00BF384602B0BDE8F08100BFDC
:1054C8007C700020F0B5124B9D6885B00DB905B011
:1054D800F0BDED0A14D0002704AE7C196410E00278
:1054E80010226946FFF7BAFF0F2809DD6B4653F80B
:1054F800042B01320AD1B342F9D12546AF42ECDB85
:10550800FFF72CFF034BED021D60E0E7671CF5E792
:10551800581C002058350020B0F1FF3F0AD002285F
:1055280010B403DC5DF8044BFDF72CBD00205DF8DA
:10553800044B7047002070470378012B00D0704758
:10554800417990F904003123F422E5E7F0B55B4B8B
:105558005B4A97B01968914200AF00F0A38059499F
:10556800594A00234FF47000C1F888003B607B6003
:10557800136843F48033136003E03B68B3F5A04F2E
:1055880009D0136803F400337B603B6801333B6048
:105598007B68002BF1D04C4B1B6813F4003318BF09
:1055A80001237B607B68012B52D0464C464B474A0F
:1055B800E260474A596A11605A6A42F080725A6238
:1055C8005A6942F4FC025A610025032207F10801D6
:1055D800012341F6FF764FF09040FD60BE603A73BC
:1055E800BB7325F0A7FE4FF6FF7307F10801394892
:1055F800BB6025F09FFE07F108013748374E25F0BC
:1056080099FE07F10801364825F094FE07F10801D4
:10561800344825F08FFE07F10801334825F08AFE4B
:1056280007F1080025F098FCBB683049304AA1FB17
:10563800031330499B0CF0204FF0070E5C370B60CA
:10564800566084F823009560C2F800E0BD46F0BDBE
:10565800294A1D4B122111605A685A605A685A60CB
:105668005A6842F480625A605A6822F47C125A607E
:105678005A6842F4E8125A601A6842F080721A6056
:105688001A689201FCD559680F4A21F00301596044
:10569800596841F002015960536803F00C03082B64
:1056A800FAD182E700221A6062B6144B1B6883F3B2
:1056B8000888134B1B689847FEE700BFFC9F002033
:1056C800EFBEADDE00ED00E0001002400005FA0577
:1056D8005855002000040048000800483F19010000
:1056E800000C0048001000480014004883DE1B43EB
:1056F80010E000E04C5500200020024000D8FF1FB9
:1057080004D8FF1F70B50F4C0F4DC0EBC00004EB61
:105718008004686926693043686182B09209667BB3
:10572800A1600025012101A863618DF804608DF84E
:1057380005208DF806508DF807101EF0C9F902B043
:1057480070BD00BF041B002000100240074BC0EBD7
:10575800C00030B403EB8000054C056963692B4336
:1057680063610176427630BC704700BF041B00209D
:10577800001002402DE9F04F5E4C54F8204083B0F1
:10578800002C71D0666D984691465B4B7268E26456
:10579800A160236004F15A014FF4807304F5AD72DF
:1057A8006161A261E36023610746307E1CF098FACC
:1057B800F068A8B1514B00215A68904203F11C03CC
:1057C80000F0928001310C29F6D100207A1CD2B267
:1057D8000C21FFF7BBFFE36CF26822632433A36458
:1057E800B068D8B1454B00215A68904203F11C03B8
:1057F80078D001310C29F7D100257A1CD2B20B21BF
:105808002846FFF7A3FF2346F27E3D492846FFF7C7
:1058180079FFE36CB26862632833636494F85900D3
:10582800FEF743F9054694F85800FEF73EF918F0DC
:10583800080F824696F819B01AD0CDB118F0110F9A
:105848004FF00B0307F1010714BF4E213E21EF7102
:105858005A46AB712846FEF7EBF918F0010F45D010
:10586800236B5BB3636B4BB3204603B0BDE8F08F8B
:1058780018F0010F0CBF4FF02E084FF04E0819F02A
:10588800020F09D045B10B227B1CAA71EB71284687
:105898005A464146FEF7CCF919F0010FE0D0BAF1AB
:1058A800000FDDD001370C238AF807705A464146AD
:1058B8008AF806305046FEF7BBF9D1E7337FB27E4F
:1058C8008DF804209B090021012201A88DF80530DC
:1058D8008DF806108DF807201EF0FAF8204603B060
:1058E800BDE8F08FCDB288E7C8B26FE72846FEF76B
:1058F8002CFDB5E75C310020A41C0308041B002024
:10590800EB3200080348D0F83C3113B100F59A7027
:1059180018477047041B00200348D0F8203113B102
:1059280000F58C7018477047041B00200348D0F816
:1059380004310BB1FC301847704700BF041B00202E
:105948000348D0F8E8300BB1E0301847704700BF83
:10595800041B00200348D0F8CC300BB1C4301847E2
:10596800704700BF041B00200348D0F8B0300BB1CB
:10597800A8301847704700BF041B00200348D0F820
:1059880094300BB18C301847704700BF041B0020BF
:105998000248836F0BB1703018477047041B002012
:1059A8000248C36D0BB1543018477047041B0020E0
:1059B8000248036C0BB1383018477047041B0020AD
:1059C8000248436A0BB11C3018477047041B00207B
:1059D8000248836803B11847704700BF041B0020C2
:1059E800F0B53E4C059D00EB800004EB8004646834
:1059F800002C71D03A4E49004FF42040CFB2B0602D
:105A0800A169090454D46068DFF8E0E047F49031F4
:105A180000EA0E0001434FF420406160B06003E0EB
:105A2800411E002848D00846A1698907F8D54FF4D7
:105A38002040A262B06003E0421E00283CD010461D
:105A4800A2695206F8D5274A6168DFF8A0E0B0607D
:105A580042EA0342174301EA0E0217436760C3B1E3
:105A6800013BDBB201332B44A0694FF4204210F014
:105A7800040002F1FF3207D1511C26D0A06910F0B2
:105A8800040002F1FF32F7D0626A05F8012B9D424B
:105A9800EAD14FF42040B06002E0431E60B11846DE
:105AA800A3699B06F9D52023B060E3610120F0BD0E
:105AB800411E08B10846A3E70B4A138801339BB27D
:105AC8004FF0FF311380B160F0BD0749B2600B8819
:105AD80001339BB20B80F0BD2046F0BDE854002096
:105AE800F022002000240002E4310020009800FC8D
:105AF80070B590F904506C1C82B00AD0022D08DCF5
:105B080016460A46417900962846FFF769FF02B013
:105B180070BD002002B070BD70B50378012B82B053
:105B280004D106236A46F721FFF7E2FF9DF801201A
:105B38009DF804309DF800609DF803509DF80240E0
:105B48009DF80500074912011B0142EA063243EAA3
:105B5800053342EA141243EA10134A600B6002B09C
:105B680070BD00BFF022002000B583B00020009275
:105B78000A466821FFF734FF03B05DF804FB1749B4
:105B8800174B184A184810B4D1F8884044F47004E8
:105B9800C1F888401C6844F001041C605C6822401D
:105BA8005A601A6822F0847222F480321A601A68E5
:105BB80022F480221A605A6822F4FE025A60DA6AD5
:105BC80022F00F02DA621A6B002410404FF00062D4
:105BD80018639C608A605DF8044B704700ED00E034
:105BE800001002400CC07FF8CCFC00FF38B50B4C0D
:105BF80023688BB15A68821A002A054604DA0CE039
:105C08005A68AA1A002A07DB9A68226018461A6896
:105C180090472368002BF3D138BD38BD04400020DD
:105C28000B4B002210B4027203F5A074032102E0AA
:105C3800072A09DC9979890702D519798154013233
:105C48009C4203F11403F3D15DF8044B704700BF85
:105C5800DC3F030810230370704700BF012310B412
:105C680015211424222244704171C27003700371FB
:105C780083705DF8044B70472C2202230270437036
:105C8800704700BF436A8269D154436A0169426B15
:105C980001338B4228BF00234362002A2FD0EFF341
:105CA8001181502383F31288436B1A68D2072CD4CE
:105CB80070B45E686EB9456A826A954217D0846985
:105CC8001444DC600ED9AA1A5A608562002280F852
:105CD80050201A6842F00102C9B21A6081F3118893
:105CE80070BC70470469A21A5A608662EEE7012305
:105CF80080F85030C9B281F3118870BC7047C26C0B
:105D0800136843F0800313607047C9B281F31188A8
:105D1800704700BF026B10B462B1036CC26844697B
:105D2800D11A013B615C5DF8044B08BF134603645C
:105D3800C8B27047016A4369C4685B5C0131A1421B
:105D480028BF114601625DF8044BD8B2704700BF06
:105D5800436B13B190F850007047836A406A181A71
:105D6800B0FA80F040097047416A836A99420AD3C1
:105D7800CB1A416B026961B14968501E0B448342DA
:105D88000AD2C01A704702691144CB1A416B002924
:105D9800F2D1501EC01A704700207047036B43B100
:105DA800026C5B6893422FBF981AC0689B1AC01890
:105DB8007047C269036A9A422FBFD01AC068801818
:105DC800C01A704708B517F0D7FE024B024ADA60CE
:105DD800FEE700BF00ED00E00400FA05024A034BAD
:105DE800127819781BF016BDEC220020ED22002055
:105DF8002DE9F0470569C3681D4028D00F460646BF
:105E08004FF000484FF00009B5FA85F328FA03F27D
:105E1800D2431B3B32611540042B16D8DFE803F050
:105E28003129211903007B6A002B32D003F1FF3A94
:105E38001FFA8AFAC7F824903C6A34B123682046CE
:105E4800514698476468002CF8D1002DDCD1BDE894
:105E5800F0873868716B036889B29847002DD3D1F1
:105E6800F5E77868B16B036889B29847002DCBD104
:105E7800EDE7B868F16B036889B29847002DC3D184
:105E8800E5E7F868316C036889B29847002DBBD103
:105E9800DDE7F36A1FFA83FACEE700BF442800F073
:105EA8007E822DE9F0470C4642D9812800F0808196
:105EB80000F28D80542800F0C38040F273816E2870
:105EC80000F02982802840F07081C14B93F800903F
:105ED80009F1020919F0FF0900F08D80BD4BBE4F92
:105EE800BE4EDFF840A3994403F101080A2516E0E5
:105EF800322D00F05B82A5F13C00C0B2132840F2BD
:105F08005D8200232268511C216015702268C145FA
:105F180002F10101216013706DD018F8015B0A2DA0
:105F2800E6D1BAF80030FF2BA8BFFF23DBB2E9E7C0
:105F3800052800F022821AD8022879D040F2FD8084
:105F4800032800F01082042840F02F810246A4495B
:105F58002046FEF79EFE00212046FEF7C8FE236875
:105F68000022591C21601A700120BDE8F0872428FE
:105F780056D040F2F480282800F09381382840F069
:105F880014810A68974B0120511C21601070226807
:105F9800052115182560117022680A211518256039
:105FA800117022680021151825601170226819786F
:105FB8001518256011702268597815182560117018
:105FC80022689B78111821601370BDE8F087A0281B
:105FD80014D040F28380B82800F0BD81FE2840F03C
:105FE800E480814D05F1080635F8021B2046FEF7CE
:105FF8007EFEAE42F8D10120BDE8F0877B4B084613
:106008001968FEF75DFE7A4B20461968FEF758FEC0
:10601800784B20461968FEF753FE0120BDE8F0874B
:10602800754B08461968FEF74BFE0120BDE8F0875E
:10603800084604227149FEF72CFE0120BDE8F087CE
:106048000B686F4F591C012221601A7023680025C4
:106058009A1822601D70236897F85B20591C2160EC
:106068001A70236897F85A20591C21601A70B7F8DB
:1060780056102046FEF73BFE29462046FEF737FE1F
:10608800B7F858102046FEF732FEBD1E07F1480645
:1060980035F8021F2046FEF72AFEAE42F8D12268E4
:1060A800584B0C21501C20605D181170226813F8A1
:1060B800011F501CAB4220601170F7D123680222E7
:1060C800591C21601A70B7F85C102046FEF70FFEC5
:1060D800B7F85E102046FEF70AFE8CE7822864D1E6
:1060E8000B68494A494D1178494A581C2060197073
:1060F80011892046FEF7FBFD464B22681B88FF2BC3
:1061080002F10101A8BFFF2321601370A96881F380
:106118001001204689B2FEF7EAFD296801F30F0154
:10612800204689B2FEF7E3FD23683B4A591C1278E2
:1061380021601A700120BDE8F087012835D10B686D
:106148000022591C21601A7023685A1C226018709A
:1061580023682422591C21601A70BDE8F087202882
:1061680023D10B682A4D591C6A7821601A7023685C
:106178002A78591C21601A702368AA78591C216052
:106188001A7029892046FEF7B2FD23686A79591CDE
:1061980021601A702368AA79591C21601A7001209D
:1061A800BDE8F08752283FF4DAAE0020BDE8F0875A
:1061B800074B1E78043616F0FF063FF41CAF174B4A
:1061C800174F1E4403F101094FF00A0851E000BFC0
:1061D800194E0020CC1C0308676666661429002047
:1061E80045420020674300203C4E0020ACF7FF1FCB
:1061F800B0F7FF1FB4F7FF1FA8440020D8470308D3
:106208002876002071760020164F0020AC740020FC
:1062180094760020004F0020BC760020DC1C030888
:10622800302A00203C290020B8F1500F00F0C4802B
:10623800B8F15A0F00F0D780B8F1320F00F0D680CD
:10624800A8F13C00C0B2132840F2D38000252946AB
:1062580023685A1C2260204683F80080FEF747FD19
:1062680029462046FEF743FD4E453FF4C4AE19F8D3
:10627800018BB8F10A0FD7D16A4B9D68196805EBF5
:1062880085054FF6FF736D009D42A8BF1D469942D4
:10629800A8BF194625EAE57521EAE171ADB289B2D0
:1062A800D6E70B68DFF8AC815F4E591C02222160EB
:1062B8001A70236806275A1C22601F7023680A2256
:1062C800591C21601A70236801255A1922601D7013
:1062D800B8F800102046FEF70AFDB8F8021020466C
:1062E800FEF705FD23685A1922601F7023685022A3
:1062F800591921601A7023680022591921601A70EF
:1063080031882046FEF7F3FC20467188FEF7EFFC43
:106318002846BDE8F087454B0A681B88444DFF2B8B
:10632800A8BFFF23511C21601370A96881F31001D5
:10633800204689B2FEF7DBFC3E4B20461988FEF763
:10634800D6FC296801F30F01204689B2FEF7CFFC7D
:106358000120BDE8F087384B08461968FEF7B0FC05
:106368000120BDE8F0870B685A1C0A6018700B689A
:106378000222591C21601A70F1E520460B222F4990
:10638800FEF787FC204608222D49FEF782FC2046AE
:1063980007222C49FEF77DFC0120BDE8F0871AB1E1
:1063A800294B136001207047012070473388FF2B69
:1063B800A8BFFF23DBB2A5E5244B5EE71AF056F829
:1063C80000283FF49EAD03780A2B28D8B0F9023094
:1063D80087FB0312DB17C3EBA2039BB2FF2BA8BFFB
:1063E800FF23DBB28EE51A4B5D6847E797E822008A
:1063F80045E71AF03BF800283FF428AF03780A2B4A
:106408003FF624AFB0F90430B0F9061003EB83036C
:1064180083F3500521EAE171ADB289B218E7002390
:10642800DFE700BF6C2900202C2A0020004F002045
:10643800AC740020AA76002050470020E0470308EB
:10644800EC470308F8470308CD5D0008A0290020A1
:10645800AC2900202035002008B501210220FDF7D5
:106468009DFF094B1B7803F00503052B08D000217D
:106478000120FDF793FF00210846FDF78FFFFEE797
:1064880017F00CFCF3E700BF58310020022828BFA2
:10649800022010B4084C094B207000EB8002C0EBBE
:1064A800C20207495DF8044B013003EB4203C0B256
:1064B8000B6021F0C1BD00BF404200207C4300209A
:1064C8003C42002008B513F011FAFEF7CBF9BDE8FD
:1064D800084013F0F3B900BF38B5434B5A8999897E
:1064E800914224BF00225A81198ADA89914224BF35
:1064F8000022DA81DA788AB3072A2FD03B493C4D4B
:1065080091F85700012400210A282C709C70D97139
:106518003DD00C2865D0DFED377A8ABB364C9FED2D
:10652800370AA278002918BFF0EE407A062A04D864
:10653800334901EB820191ED080A217959B3013AF7
:10654800032A4DD8F7EE007A87EE800A28F090FFEC
:106558002388984228BF1846208038BDD97921B1B0
:1065680098780428B8BF04209870204890F85700FD
:106578000A280CD00C28CED1DFED227A002ACDD003
:10658800072ACBD00A282CD1DFED1F7AC6E70A20CC
:10659800DFED1E7AC1E79B78154A07EE103A1178AD
:1065A800B8EEC77A27EE277A07EE901AF8EEE77A60
:1065B80067EE877AB4EEE70AF1EE10FA10DDC0EE66
:1065C800077AFDEEE77A17EE903A102BA8BF102352
:1065D800012BB8BF0123DBB28B4238BF0B461370C7
:1065E80038BDDFED0B7A99E7EC63002000640020EA
:1065F800243500206F120339BC6000206F12033865
:10660800CC1C03080AD7A3390F506E3A5304E93853
:106618006F12833A38B50C4C0C4DAC4206D2616807
:1066280020461434FEF7AAF8AC42F8D3084A094BBE
:10663800094C1460002209491A705A700848086009
:10664800BDE838401AF01CBEB88303082C8803083C
:106658003C420020404200207C4300204C77002030
:106668007053002008B5FFF7D5FF13F03FF9FEF788
:10667800F9F8BDE8084013F021B900BFF0B50C29BE
:106688002BD8DFE801F06F2A2A2A4C2A2A2A2B2A3B
:106698002A2A0700046AB2F80CE097881668674D42
:1066A80024F480540462036A4468C16923F40053E3
:1066B80043EA0E3321F4E641A84243EA073341EAAC
:1066C800062100F0B58005F50065A84200F0B0800D
:1066D80092684460C16102640362F0BD046A9689ED
:1066E8009588D2F800E0554F24F480740462036A58
:1066F8004468C16923F4007343EA062321F0730157
:10670800B84243EA052341EA0E017ED04C4DA84227
:106718007BD092684460C161C2630362F0BD046AC1
:1067280096899588D2F800E0444F24F0100404625A
:10673800036A4468816923F0200321F0807143EAE9
:10674800061321F4E641B84243EA051341EA0E2153
:1067580048D03B4DA84245D092684460816182632D
:106768000362F0BD046A9389B2F804E01768334EF7
:1067780024F001040462056A4468816943EA0E034F
:1067880021F4803125F002059BB221F07301B0425B
:1067980043EA050341EA070114D0294DA84211D064
:1067A80005F54065A8420DD005F58065A84209D0D9
:1067B80005F58065A84205D092684460816142630E
:1067C8000362F0BDD689158A578A23F0080333433C
:1067D8003D43D68824F4407423F00403ADB2334318
:1067E8002C43E9E7D589178AD68823F0800343EA42
:1067F800051324F44064558A23F0400344EA8704CF
:1068080043EA061344EA8504A6E7D589178AD68899
:1068180023F4006343EA052324F44054558A23F4FF
:10682800806344EA071443EA062344EA051470E740
:10683800158A24F4804444EA851449E7002C014071
:10684800003401402DE9F84F4FF48C720021824842
:10685800824C834D834E844FDFF82882DFF82892DC
:106868002AF013FF81488249DFF820E2DFF820C2CE
:1068780000221359834200F0C380B3F1804F00F027
:10688800D580AB4200F0D980B34200F0D880BB423B
:1068980000F0D780734500F0D680634500F0A680ED
:1068A800434500F0D2804B4500F0D280DFF8E4A1E8
:1068B800534508BF4FF4802300F09A801432B2F594
:1068C800AA7FD6D1654D6B4F6B4E05F5AA784FF070
:1068D800030A4FF0020903E01435454500F08E80A5
:1068E800AB79002BF8D02B791C09013C052C03F05F
:1068F8000F03F1D837F8140040FA03F2D207EBD5AA
:106908004FF0010B0BFA03F3013B184028F03EF857
:106918005A4B1B5D184416EBC004DDD056F83030D6
:106928005748297A03F13842920A825C02F01F0024
:106938005209022A0BFA00FB71D0032A68D0012AF7
:1069480005D14B4A4A4852694BEA02024261B4F8FF
:1069580004E0BEFA8EF2C2F11F0292B2D00803EB35
:10696800800002F00702046A92004FF00F0C0CFA44
:1069780002FC24EA0C040462046A01FA02F22243CB
:10698800002402624FF0010C224603E0102A04F1B1
:106998000204A1D00CFA02F030EA0E0102F1010261
:1069A800F4D1D3F808B00AFA04F1C9430BEA010B91
:1069B800C3F808B0D3F808B0C3F808B0B3F804B007
:1069C8001FFA8BFB2BEA00009880988880B2988089
:1069D800186808401860D3F800B009FA04F040EAD3
:1069E8000B001860D8680140D960CFE74FF4005316
:1069F800D1F818A043EA0A038B615FE7BDE8F88F76
:106A0800D1F818A04FF4006343EA0A038B6155E7F5
:106A1800174A1748D2694BEA0202C26197E7144A3B
:106A2800134892694BEA0202826190E70123D1F888
:106A38001CA043EA0A03CB6140E70223F7E70423DB
:106A4800F5E71023F3E72023F1E74FF48033CFE78E
:106A58004FF40033CCE700BF0C730020DC3F030881
:106A6800000400400008004000100040002C0140D5
:106A780000100240D446030890710020E046030845
:106A8800D43F030800400140004401400014004086
:106A9800003401400048014001490248FFF7A8B905
:106AA800FC7300200048014001490248FFF7A0B9E3
:106AB800AC7300200040014001490248FFF798B933
:106AC800847300200008004001490248FFF790B98C
:106AD8005C7300200004004002494FF08040FFF73B
:106AE80087B900BF3473002010B5064C064821460C
:106AF800FFF77EF904F1C8010448BDE81040FFF72C
:106B080077B900BF0C730020002C014000440140FD
:106B180001490248FFF76CB90C730020002C0140B2
:106B28002DE9F0410468514DA30AAB4200F084807E
:106B38000AD94F4DAB4277D00135AB425FD0023D09
:106B4800AB426DD0BDE8F0814A3DAB4270D0013513
:106B5800AB4258D0B3F5801FF4D14FF0480E012650
:106B680047794FEA970C00296AD0B0006346851927
:106B78000227D4F80C809F400CEB4503BFB23D4D73
:106B880003F1040C47EA080745F8231045F82C20C0
:106B9800E760EFF31181502282F31288821905EB26
:106BA800C2021369002B32D013620433821905EB39
:106BB800C202576917B11F6053690433821905EB84
:106BC800C202976917B11F6093690433821905EBF4
:106BD800C202D76917B11F60D36904330027CAB24C
:106BE8001F6082F31188304405EBC000036A8BB93B
:106BF800E3684FF6FE721340E360BDE8F0814FF49E
:106C0800887E0626ACE74FF0980E0326A8E705EB2A
:106C18000E03CBE7E36843F00103E360BDE8F081CE
:106C28004FF0C00E04269BE74FF0E80E052697E7C5
:106C38004FF0700E022693E74FF0200E00268FE7E4
:106C4800BF08022306FA03F0BB40DB43E768094D9F
:106C58009BB23B4087190CEB470CE3600CF1040333
:106C680045F82C1045F8232093E700BF4B0010008F
:106C7800510010000C73002030B503685C4D188873
:106C88005C4CB4FBF2F20139013AAB4294B283B0E6
:106C980089B282B266D05848834263D0B3F1804F3C
:106CA80060D0A0F5983083425CD000F580608342C4
:106CB80058D0524883425BD000F5806083427DD033
:106CC80022F4407200F58C3092B283421A80D96265
:106CD8001C850ED0484A93420BD002F5406293427D
:106CE80007D002F58062934203D002F58062934296
:106CF80001D100221A8601225A611A883C4992B2AF
:106D080042F001028B421A8062D0B3F1804F61D009
:106D18003B4A934260D002F5806293425ED002F50E
:106D2800006293425CD002F5806293425AD002F529
:106D38009032934258D002F54062934256D002F501
:106D4800806293421ED002F58062934208BF0922F6
:106D580019D002A84FF0012340F8043D1CF0B8FEFA
:106D680003B030BD254822F07002834292B2A3D10D
:106D780001201A80D9621C8558611A8892B2024390
:106D88001A80C5E708221F4B03EBC20301A893F83A
:106D980041408DF80440012300228DF805308DF81C
:106DA80007308DF806201CF093FE1B2CD8D1164B0B
:106DB800019301A81CF08CFE03B030BD01201A809D
:106DC800D9621C8558611A8892B202431A809CE7DE
:106DD8000022D8E70122D6E70222D4E70322D2E72D
:106DE8000422D0E70522CEE70622CCE70722CAE72D
:106DF800002C014000A24A04003401400010004069
:106E080000040040CC1C030819010001204B9842E3
:106E18002DD0B0F1804F2CD0A3F5943398422AD0CE
:106E280003F58063984228D003F50063984226D082
:106E380003F58063984224D003F59033984222D01A
:106E480003F54063984220D003F58063984207D049
:106E580003F58063984208BF092202D000207047DA
:106E680008220C4B03EBC20393F840007047002242
:106E7800F7E70122F5E70222F3E70322F1E704220C
:106E8800EFE70522EDE70622EBE70722E9E700BF77
:106E9800002C0140CC1C03082DE9F04F013085B0CF
:106EA800C3B203938E4D8F4F8F4C904E0A2302939B
:106EB800DFF840921BF028FC4FF4FA7A4FF0100CE0
:106EC8004FF47A70D9F80430C3F30803002B40F06C
:106ED800C880EFF31183002B40F0C3802968A268B3
:106EE80000BF2B689942F9D1D7F800E000FB0EF3F8
:106EF8009B1AB3FBFEF300FB01314FF0010E019129
:106F0800D9F80430C3F30803002B40F08E80EFF368
:106F18001183002B40F089802B68A16800BF2A6884
:106F28009342F9D1D7F800B000FB0BF2521AB2FB2A
:106F3800FBF200FB0323019A9B1AB3F57A7FDFD398
:106F4800BAF1010ABED1039B002B40F0C4804FF474
:106F58007A7ADFF8A09150464FF0100CD9F8043037
:106F6800C3F30803002B40F09980EFF31183002B43
:106F780040F094802968A26800BF2B689942F9D133
:106F8800D7F800E000FB0EF39B1AB3FBFEF300FBFF
:106F980001314FF0010E0191D9F80430C3F3080311
:106FA8003BBBEFF3118323BB2B68A16800BF2A68A2
:106FB8009342F9D1D7F800B000FB0BF2521AB2FB9A
:106FC800FBF200FB0323019A9B1AB3F57A7FE3D304
:106FD800BAF1010AC2D1029B013B02937FF468AF68
:106FE8004349444B4448454A0860DA6005B0BDE867
:106FF800F08FEFF311888CF31288A1682368DB0304
:1070080044BFC6F800E0A1682B6832685FFA88F8C8
:1070180088F31188D7F800801A4400FB08F35B1A3C
:10702800B3FBF8F300FB0233CDE7EFF311888CF3E1
:107038001288A1682368DB0344BFC6F800E0A16892
:107048002B6832685FFA88F888F31188D7F80080CF
:107058001A4400FB08F35B1AB3FBF8F300FB023396
:1070680069E7EFF311828CF31288D4F808E02368FB
:10707800D90303D501233360D4F808E02B683168BD
:10708800D2B282F311883A68194400FB02F3A3EBE9
:107098000E03B3FBF2F300FB01312EE7EFF311828D
:1070A8008CF31288D4F808E02368D90303D50123A8
:1070B8003360D4F808E02B683168D2B282F31188C3
:1070C8003A68194400FB02F3A3EB0E03B3FBF2F397
:1070D80000FB01315DE718461BF086F937E700BF72
:1070E800485500204C55002010E000E04455002091
:1070F800FC9F002000ED00E0EFBEADDE0400FA05C5
:107108002DE9F047AD4FAE4E12F0F0FBBE421ED255
:10711800DFF83483DFF834934446258862197DB15B
:107128004A450DD2052D0BD933886188C3F30B036B
:10713800994200F0F280144625886219002DEFD19B
:10714800716830461436FDF719FBBE42E4D39D4AF8
:107158001378A3F1170102290FD99B4911F83300BD
:10716800002840F0FC80D8000144497829B19749AB
:1071780011F83330002B00F01A81954C6378022BFC
:1071880084BF002363702378022B84BF00232370FD
:10719800904B9A78042A00F0018132B91A88B2F526
:1071A800F07F84BF4FF4F0721A808B4D8B4A2B68A6
:1071B8001A40002A00F0FE80D80700F1EA8059043E
:1071C80000F1E2801A0700F1DA809B0400F1D08018
:1071D800834D2B685A8C998C914224BF00225A8483
:1071E800FFF77AF91EF00EFD10B97E4820F0EEF98F
:1071F8008020FDF7F9FA4FF40070FDF7F5FA4FF427
:107208000010FDF7F1FA4FF00070FDF7EDFA4FF0BE
:107218008060FDF7E9FA6378022B06D8724A734951
:1072280003EB430302EB83030B602378022B07D89D
:1072380003EB83016E4AC3EBC10302EB43032B60EC
:1072480026F066F8002130226A482AF01EFA2868DB
:1072580016F064F9684B2E6803F1500102E004331C
:1072680099427AD01A78002AF9D19C78D878844241
:10727800F5D26249624B91F804E06248624D5C6B5A
:10728800624B2860C827642111FB0E71DFF8C0E14A
:1072980059605F4F30F8061C5E4DAEF800100021B3
:1072A8009960D960196159619961D96183F8201091
:1072B80083F821103A702E600CB112F0DDF9564BAC
:1072C8009FED565A1B88564A9FED566A5579564C7B
:1072D80056495748086006EE903AF8EEE66A138871
:1072E800C5EE265A07EE103A53881279C4ED005AB3
:1072F80007EE903AB8EEC77A4E4BF8EEE77A1D7271
:107308005A7227EE067A67EE867ABDE8F04783ED73
:10731800017AC3ED007A12F0D1BA63799B077FF442
:107328000AAF716894F804A03046FDF727FA33884D
:10733800BAEB133F04D01436BE42FFF4EDAE06E7B5
:1073480073887068AA1FC3F30B039A4204F10601FD
:10735800A8BF1A4627F084FEEDE7012289E7D80086
:107368000C186468002C7FF4FFAE17241470FBE639
:107378003148FDF739FA4020FDF736FA28E72F485B
:10738800FDF732FA2B6820E72D48FDF72DFA2B6818
:1073980018E72C48FDF728FA2B6810E79A8AB2F507
:1073A8007A7FBFF402AF4FF47A729A82FDE618230F
:1073B8001370E2E643F001032B60FDE62C88030816
:1073C800B883030870350020304103088833030868
:1073D80040420020BC600020A84400200960000250
:1073E8003C42002094700020705300204C7700200D
:1073F8007C430020D428002074350020C049002098
:107408009453002036350020D46F0020E05300202C
:10741800112100200829002054240020C0C9FB485D
:107428000423002017B7D13858240020284700200B
:107438003661023D04470020094000020160000255
:10744800092000020860000202F003080000040896
:10745800643C002008B512F049FAFDF703FA12F06F
:107468002DFAFFF74DFE0120BDE8084020F0E4BDED
:107478002DE9F04F013085B0C3B203930B4602915A
:107488008B4C8C4E002B00F099808B4D8B4FDFF886
:1074980030921BF039F94FF4FA7A4FF0100C4FF490
:1074A8007A70D9F80430C3F30803002B40F0DE806B
:1074B800EFF31183002B40F0D9802968A26800BF40
:1074C8002B689942F9D1D7F800E000FB0EF39B1A1C
:1074D800B3FBFEF300FB01314FF0010E0191D9F827
:1074E8000430C3F30803002B40F08780EFF31183C7
:1074F800002B40F082802B68A16800BF2A68934265
:10750800F9D1D7F800B000FB0BF2521AB2FBFBF22C
:1075180000FB0323019A9B1AB3F57A7FDFD3BAF1F4
:10752800010ABED1039B002B40F0BD804FF47A7A4C
:10753800DFF88C9150464FF0100CD9F80430C3F3A3
:107548000803002B75D1EFF31183002B71D1296843
:10755800A26800BF2B689942F9D1D7F800E000FB78
:107568000EF39B1AB3FBFEF300FB01314FF0010E43
:107578000191D9F80430C3F3080313BBEFF3118367
:10758800FBB92B68A16800BF2A689342F9D1D7F8E4
:1075980000B000FB0BF2521AB2FBFBF200FB032314
:1075A800019A9B1AB3F57A7FE3D3BAF1010AC4D1E1
:1075B800029B013B0293002B7FF467AF05B0BDE847
:1075C800F08FEFF311888CF31288A1682368DB032E
:1075D80044BFC6F800E0A1682B6832685FFA88F8F3
:1075E80088F31188D7F800801A4400FB08F35B1A67
:1075F800B3FBF8F300FB0233D2E7EFF311888CF307
:107608001288A1682368DB0344BFC6F800E0A168BC
:107618002B6832685FFA88F888F31188D7F80080F9
:107628001A4400FB08F35B1AB3FBF8F300FB0233C0
:1076380070E7EFF311828CF31288D4F808E023681E
:10764800D90303D501233360D4F808E02B683168E7
:10765800D2B282F311883A68194400FB02F3A3EB13
:107668000E03B3FBF2F300FB01317FE7EFF3118266
:107678008CF31288D4F808E02368D90303D50123D2
:107688003360D4F808E02B683168D2B282F31188ED
:107698003A68194400FB02F3A3EB0E03B3FBF2F3C1
:1076A80000FB013118E718461AF09EFE3EE700BFBE
:1076B80010E000E044550020485500204C550020BB
:1076C80000ED00E0204B5B68C3F3080330B4BBB99E
:1076D800EFF31183A3B91D4B1D4C1868A16800BFB7
:1076E8001A689042F9D11B4B1C684FF47A7202FB5E
:1076F80004F3591AB1FBF4F130BC02FB00107047D7
:10770800EFF31182102383F3128811498C680B68F8
:1077180013F4803F104B02D0012018608C680B498D
:10772800D2B20D68186882F311880A4B19684FF4B1
:107738007A72284402FB01F31B1B30BCB3FBF1F344
:1077480002FB0030704700BF00ED00E04855002004
:1077580010E000E04C550020445500202DE9F84F7A
:107768008046FFF7AFFF254E2549DFF8A0E0254A00
:10777800254D844610274FF47A740120DEF8043032
:10778800C3F30803D3B9EFF31183BBB90B68D2F87D
:1077980008A000BFD1F800904B45F7D1D6F800B04B
:1077A80004FB0BF9A9EB0A09B9FBFBF904FB0393EA
:1077B800A3EB0C034345E1D3BDE8F88FEFF3118A3F
:1077C80087F31288D2F808B01368DB0344BF286037
:1077D800D2F808B00B68D5F800905FFA8AFA8AF3F5
:1077E8001188D6F800A0994404FB0AF3A3EB0B0315
:1077F800B3FBFAF304FB0933DAE700BF4C5500206A
:107808004855002010E000E04455002000ED00E05D
:107818002DE9F04FDFF830C1474A4849484E494DF5
:107828008046102718F1FF38C0F08480DCF8043057
:10783800C3F30803002B5CD1EFF31183002B58D15D
:107848000B68946800BF08688342F9D1D6F80090A5
:107858004FF47A7000FB09FEAEEB040EBEFBF9FE96
:1078680000FB03EEDCF80430C3F308034FF47A742A
:107878000120FBB9EFF31183E3B90B68D2F808A034
:1078880000BFD1F800904B45F7D1D6F800B004FB03
:107898000BF9A9EB0A09B9FBFBF904FB0393A3EB6A
:1078A8000E03B3F57A7FBDD2DCF80430C3F30803C6
:1078B800002BDFD0EFF3118A87F31288D2F808B0D3
:1078C8001368DB0344BF2860D2F808B00B68D5F80A
:1078D80000905FFA8AFA8AF31188D6F800A09944D2
:1078E80004FB0AF3A3EB0B03B3FBFAF304FB093322
:1078F800D5E7EFF3118487F31288D2F8089013685C
:10790800D80303D501232B60D2F808900B682868A8
:10791800E4B284F31188D6F800A04FF47A7400EB2F
:10792800030E04FB0AF3A3EB0903B3FBFAF304FB0E
:107938000E3E97E7BDE8F08F10E000E048550020C4
:107948004C5500204455002000ED00E030B4EFF322
:107958001183102282F312880649074C0A680748E7
:10796800013200250A602560DBB2026883F31188C2
:1079780030BC7047485500204455002010E000E016
:107988000F4B1B88014643B90E4B0F4A1B781068F2
:107998000BB981F00101FCF7F7BC0C4B5A691AB11D
:1079A80018B91A68106058747047094A186811881D
:1079B800084A92FBF1F2012102605974704700BF36
:1079C800205500202255002024550020285500204D
:1079D8004055002020A107001D4B70B59C68E36C42
:1079E800226BDD69C2B1636B2BB12B0702D5E36C47
:1079F80008221A6270BD2A06F7D5A26A616A8A420D
:107A08001FD0511CA069A162825C2069E66C81428A
:107A18003285EAD3A362E8E7A906E4D5E26A1AB197
:107A2800988C80B29047DEE7E1699B8C6069DBB295
:107A38004E1CE6614354E169E368994228BFE2615C
:107A4800D1E7E26C136823F080031360CDE700BF31
:107A58005C3100201D4B70B55C68E36C226BDD69FE
:107A6800C2B1636B2BB12B0702D5E36C08221A62F3
:107A780070BD2A06F7D5A26A616A8A421FD0511CD6
:107A8800A069A162825C2069E66C81423285EAD3F2
:107A9800A362E8E7A906E4D5E26A1AB1988C80B235
:107AA8009047DEE7E1699B8C6069DBB24E1CE661BA
:107AB8004354E169E368994228BFE261D1E7E26C87
:107AC800136823F080031360CDE700BF5C3100200A
:107AD8001D4B70B51C68E36C226BDD69C2B1636B2A
:107AE8002BB12B0702D5E36C08221A6270BD2A0657
:107AF800F7D5A26A616A8A421FD0511CA069A162A7
:107B0800825C2069E66C81423285EAD3A362E8E7A9
:107B1800A906E4D5E26A1AB1988C80B29047DEE7EC
:107B2800E1699B8C6069DBB24E1CE6614354E169F4
:107B3800E368994228BFE261D1E7E26C136823F059
:107B480080031360CDE700BF5C31002070B4EFF311
:107B58001186502383F31288436B1A68D20720D406
:107B68005D686DB9446A826A944217D0816911448C
:107B7800D9600ED9A21A5A608462002280F8502077
:107B88001A6842F00102F1B21A6081F3118870BCE0
:107B9800704701698A1A5A608562EEE7012380F806
:107BA8005030F1B281F3118870BC70472DE9F04F65
:107BB8002DED0C8B3C4B1B7895B0012B099001F0F7
:107BC8007F873A4C94F80021002A41F0C180072BA6
:107BD800374D01F07087002305936B683448984748
:107BE800002800F06981B5F8B470002285F85520A6
:107BF800002F40F04387B5F93E00AA6AB5F93C600A
:107C0800696AB5F94030DFF8B4B0821AE86A6A6385
:107C1800711A1B1A2963274895F85610AB6311F09F
:107C2800ADFCDBF80030990040F1F080D5ED0D5A3D
:107C3800D5ED0C7A204A94ED716AD4ED726A94ED10
:107C4800737AD4F8D0311268B8EEE58AD5ED0E5AB9
:107C5800F8EEE77AF8EEE58A013377EE867A38EEC1
:107C6800268A78EE878A9342C4ED717A84ED728A07
:107C7800C4ED738AC4F8D03101F0A5840A4B1F788B
:107C8800142F03F025810023D4F8D8610693062E1B
:107C980000F2AF80DFE816F0EC1746177B16B11834
:107CA80014005A17DF1600BF384E00201423002096
:107CB8000064002030640020D83C00209466002036
:107CC800D84B1A78D4F8DCE1DFF8D0C39FEDD67A28
:107CD8004FEACE000CEB000383ED007A002A7DD03A
:107CE800D249B0EE476AF0EE476A0023F1EC017A18
:107CF800013367EEA77A05EE903AB4EEE77AF1EE33
:107D080010FAF8EEE55AB8BFB0EE677A934276EE0D
:107D1800A76AA7EEA56AE9D1F5EEC06A0CEB0003E5
:107D2800F1EE10FA83ED007A58DDC6EE265AC04B04
:107D3800C04A1288F7EE007A75EEE75AD3ED007A5A
:107D480065EEA77AFDEEE77A17EE903A812B43F3BA
:107D580086879342A8BF134607EE903AF8EEE77A73
:107D6800B54B00EB0E0103EB810393ED057AD3EDE0
:107D7800003A93ED066A93ED014AD3ED046AD3ED18
:107D8800034A93ED025AA3EEA77AA4EE276A66EE99
:107D9800C76AA7EE646ABDEEC77AE5EE276A17EEF2
:107DA800101A812983ED056AC3ED066A43F35487E7
:107DB8008A42A8BF0A4607EE902AF8EEE77AFCEE58
:107DC800E77ACDED077ABDF81C300CEB0002938002
:107DD800BEF1000F02D1132F04F02184152F42F0B9
:107DE8002B866044DFF8B882838828F81E30D4F8E0
:107DF800D861924B013683FB06239A19F317C3EB1C
:107E0800A203C3EBC303F61AC4F8D8618C4B1B78E2
:107E1800002B01F0B4818B4EDFF88892DFF880A246
:107E280006F5BC780027884BD5ED087A1B78172B08
:107E380001F05D8496ED007AB8EEC78A082B28EE2B
:107E4800278A07D1B0EE480A069327F011FB069B54
:107E58002AF81700DBF8002092000BD5002F04F059
:107E68003787B0EE480AD5F8143208F17000984701
:107E7800B0EE408AB0EE480AD5F83431A8F1700067
:107E88009847D5F8A431404698476F4B1B78032B89
:107E9800B0EE408A01F03884D6F8F800D5F8B8304A
:107EA800B0EE480A98470137032F08F12408A9ECD7
:107EB800010A06F10406B6D1634B93F80090B9F1B4
:107EC800070F00F0988694F8E831002B40F0A08660
:107ED8005E4B5B79002B40F0CB8501235A4A84F82E
:107EE800E8311278072A02F0028200230B93584BDC
:107EF80094ED7B9A93ED007A564BD4ED41CAD3F8B2
:107F080000A0554B0693F7EE007A37EEC9CA534BDB
:107F180008932CEE07CA524B0A93B4EEE7CA514BAA
:107F280007930025F1EE10FA4F4BDFF87C91DFF84C
:107F38007CB1DFED4E8A9FED4EAADFED3BBADFED57
:107F48004D9A9FED4DBADFED4DAADFF864814C4F95
:107F5800059388BFB0EE67CA2E464A4B99ED008A52
:107F68002B44D3ED007AF5EE407AF1EE10FA17D0F3
:107F7800454B2B44D3ED006A38EE667AB0EEC76AFB
:107F8800F4EEC67AF1EE10FA08D5B5EEC07AF1EE45
:107F980010FACCBF37EEA68A36EEE78A83ED008A60
:107FA800069B1A88930700F08580022E00F08280D5
:107FB8009AF82E10354B07EE901A2B4493ED007A61
:107FC8004B42F8EEE76A07EE903A26EE877AF8EE2B
:107FD800E77AB4EEE77AF1EE10FA0AD407EE901ACF
:107FE800F8EE677AF4EEC77AF1EE10FA88BFF0EE91
:107FF800477A274B274903EB460331F91600B3F9B3
:108008000C30C01A07EE100AB8EEC77AD007E7EEB0
:10801800687A40F10586204B93ED008A27EE888A1E
:1080280048E000BFDE3C00200000000014230020D0
:10803800E03C0020DC3C0020143F002093244992BF
:10804800D43C002030640020384E0020EC6300202F
:10805800C84800203C4200200C42002000000020BC
:10806800687400208466002010330020CDCCCC3DFD
:10807800AE47813F0000C84200003443610BB63B65
:108088001C330020BC48002004250020B024002018
:10809800303500201C420020A4480020FC3E00206F
:1080A8003C4E00208866002048240020E838002044
:1080B80028330020079B94F8FC212B44D3ED01DAE8
:1080C80038EE6DDA002A3DD0D24BD4F80022099957
:1080D8001B688A1A9A4235DD9AF84830022B02F05A
:1080E800A381022E04F00C85CB4B1B68990741F144
:1080F8002D80CA4BCA49DFF890E331F916C09EEDCE
:10810800008ADFF888E3C7ED00BA03EB460028EEE3
:10811800288AB0F90C00A0EB0C0007EE900AF8EEE4
:10812800E77ADEF8000027EE888A904238EE6DDAAA
:10813800C1F21E82F7EE007AB4EEE79AF1EE10FA79
:1081480001F1ED81B74B2B4493ED000A059B2CEE12
:10815800800A022E20EE0D0AA3EC010A059304F012
:10816800F884089BDBED007A93ED007AAE4BD7EDEF
:10817800006A93ED006AAD4B67EE277A2B4427EE31
:108188008C7AD3ED007A67EE277AF0EE665AEDEE38
:10819800275AB1EE467AB4EEE57AF1EE10FA08DC29
:1081A800F4EEC65AF1EE10FA8CBFB0EE467AB0EE95
:1081B800657A94ED7B6AF7EE007AB4EEE76AF1EE41
:1081C80010FAACBF0123002343B1F0EEE66AF0EEEB
:1081D800C77AF4EEE67AF1EE10FA01D587ED007A67
:1081E800022E04F08684924A924B52F826001B68AD
:1081F800B0EE6D0A9847904A904B52F826001B68DB
:1082080098479AF8373023B1069B1B88002B00F05B
:108218006B85B0EE6B8A8A4B9BED007A38EE400A8C
:108228002B4493ED008A83ED000A9AF8483030EE2B
:10823800480AC0EE077A2BB30A9B1B78D80721D5CA
:10824800B7EE007AB4EEC79AF1EE10FA04DB94F8B0
:10825800FC31002B01F02F80D4F80032099AD31A90
:108268006C4A12689A420DDD764B93ED007AB0EEB7
:10827800CDDAB4EEC7DAF1EE10FA41F195810023B8
:1082880084F8FC31704B94F80C222B4493ED007A5F
:108298002CEE877A67EE277AC8ED007A32B9059B0B
:1082A800C7ED00BA43ED01BAC8ED00BA0136032E96
:1082B80009F1040908F1040807F1040705F10405A8
:1082C8007FF44BAE614B1B78072B01F01E84012B0A
:1082D80001F0FA87002794F81432002B40F0008749
:1082E8005B4A5C4B10681B6810F4805A93F82C307A
:1082F80040F06F87584A594992ED006A498B584AAD
:1083080084ED896A92ED007A564A84ED8A7A07EEFE
:10831800901AF8EEE76AD2ED037A534A84ED876A39
:1083280037EE467A77EEE67AD2ED006A84ED867A01
:10833800012284F82C22C7EEA65A4C494C4A91EDEA
:10834800005A4C499FED4C6A91ED004A4B49DFEDCC
:108358004C6AD1ED004A92ED007A35EE045AF7EEF8
:10836800007AF4EEE75A35EE245AF1EE10FA88BF97
:10837800F0EE675A25EE065AF4EEE65AB1EE476A71
:10838800F1EE10FAB4EEC65AB8BFF0EE665AF1EE46
:1083980010FAC4ED8C5A01F1A381B4EEC75AF1EE7C
:1083A80010FA88BFB0EE475A304ADFED336AD2ED93
:1083B800017A304A92ED014A304A77EE847AD2ED5A
:1083C800014A77EEA47A67EEA67AB4EEE76AF1EE90
:1083D80010FA08DCB4EEE77AF1EE10FA8CBFB0EED2
:1083E800676AB0EE476A214ADFED236AD2ED027A66
:1083F800204AD2ED024A234A77EEA47A92ED007A17
:1084080067EEA67AB1EE473AF4EEC37AF1EE10FAC7
:1084180047D43DE0D0480020C87600203035002001
:108428001C42002078480020EC48002084480020A6
:10843800F0380020EC380020443900204039002072
:1084480018250020DC48002090480020384E0020E5
:10845800946600203C420020B033002020680020B1
:1084680014350020184F0020AC490020103300209C
:10847800F04800201C3300206F12833A2833002074
:1084880000000000F4480020A4480020CC48002048
:10849800F4EEC77AF1EE10FA8CBFB0EE473AB0EEC0
:1084A800673AF04A52780AB9B1EE433A002B41F0E4
:1084B800FC84F7EE003AEC4D2A78002A03F0AD80F0
:1084C800EA4BDFEDEB7AD3ED024AD3ED016A93ED87
:1084D800037A66EE244AE5EE264AE3EE074A63EE9F
:1084E800A44AF4EEE74AF1EE10FAB4BFB0EE674AD8
:1084F800B0EE644A98BFF0EE647A012ACDED0C4ADA
:1085080003F0B08093ED067AD3ED052AD3ED076A20
:1085180026EE077AA5EE227AA3EE267A23EE877A4C
:10852800B4EEE77AF1EE10FAB4EEC47A8CBFF0EE4E
:10853800676AF0EE476AF1EE10FA88BFF0EE676AF4
:10854800B4BFF0EE447AF0EE477A022A8DED0D7A48
:1085580000F0DE8093ED0A7AD3ED092A93ED0B4AF9
:1085680026EE077AA5EE227AA3EE047A23EE877A1E
:10857800B4EEE67AF1EE10FAB4EEE77A8CBFB0EE1C
:10858800664AB0EE474AF1EE10FA98BFF0EE446A38
:10859800A8BFF0EE477A032A8DED0E7A00F0B88076
:1085A80093ED0E7AD3ED0D2A93ED0F4A26EE077A56
:1085B800A5EE227AA3EE047A23EE877AB4EEE67A61
:1085C800F1EE10FAB4EEE77A8CBFB0EE664AB0EE80
:1085D800474AF1EE10FA98BFF0EE446AA8BFF0EEF1
:1085E800477A042A8DED0F7A00F0928093ED124AB3
:1085F800D3ED112A93ED137A26EE044AA5EE224A0A
:10860800A3EE074A23EE844AB4EEE64AF1EE10FAE6
:10861800B4EEE74A8CBFB0EE667AB0EE447AF1EE7B
:1086280010FA98BFF0EE476AA8BFF0EE447A052A20
:108638008DED104A6CD093ED164AD3ED152A93EDC3
:10864800177A26EE044AA5EE224AA3EE074A23EE3D
:10865800844AB4EEE64AF1EE10FAB4EEE74A8CBF6B
:10866800B0EE667AB0EE447AF1EE10FA98BFF0EE0A
:10867800476AA8BFF0EE447A062A8DED114A47D022
:1086880093ED1A4AD3ED192A93ED1B7A26EE044A84
:10869800A5EE224AA3EE074A23EE844AB4EEE64A40
:1086A800F1EE10FAB4EEE74A8CBFB0EE667AB0EE9F
:1086B800447AF1EE10FA98BFF0EE476AA8BFF0EEE0
:1086C800447A072A8DED124A22D093ED1E7AD3ED13
:1086D8001D2A93ED1F4A26EE077AA5EE227AA4EE0C
:1086E800037A27EE237AB4EEE67AF1EE10FAB4EEC6
:1086F800E77A8CBFB0EE666AB0EE476AF1EE10FA20
:108708008DED137A98BFF0EE466AA8BFF0EE477A6F
:1087180077EEE67AF7EE006AF4EEE67AF1EE10FA12
:10872800C4ED7B7A43F35B8786EEA77A022ADDEDF8
:108738000D7A67EE244A67EE877ACDED0C4ACDEDC7
:108748000D7A2DD0DDED0E7A67EE877A032ACDED0E
:108758000E7A25D0DDED0F7A67EE877A042ACDED03
:108768000F7A1DD0DDED107A67EE877A052ACDEDF8
:10877800107A15D0DDED117A67EE877A062ACDEDED
:10878800117A0DD0DDED127A67EE877A072ACDEDE2
:10879800127A05D0DDED137A27EE877A8DED137AFC
:1087A800344B1E6816F0805601F0A381F6EE005A8D
:1087B800C4ED8C5A002A02F025872F4BD4ED8A4A43
:1087C80093F8038094F92C320A99D4ED896A91F8C8
:1087D80000E0DFF8B0C02949DFF8AC90B1F9061025
:1087E8009CED007A059106EE103AFDEEE44A244B22
:1087F80099F80090B3F81AB094ED865AD4ED877AB8
:1088080014EE903AFDEEE64A00F0100C00F48000F9
:108818000EF0010EB8EEC66A14EE901A0690B8F182
:10882800000F41F09D83DFF84480BCF1000F41F058
:10883800A38198ED007ADDED0C6ADFF850C025EED3
:10884800877AA6EE267AF0EE676AE5EE076ABDEE4D
:10885800E67A17EE106A17EE100A9E42A8BF18466D
:1088680016E000BF70350020194E00201C4900207A
:1088780000000000C0760020E0530020485F002080
:1088880020680020F8480020E060002070330020B5
:10889800B142C8BF084607EE100AB8EEC77A012AE7
:1088A8008CED007A00F0DC8098ED047ADDED0D6A3D
:1088B80025EE877AA6EE267AF0EE676AE5EE076A75
:1088C800BDEEE67A17EE106A17EE100A9E42A8BFB0
:1088D8001846B142C8BF084607EE100AB8EEC77A74
:1088E800022A8CED017A00F0BB8098ED087ADDED64
:1088F8000E6A25EE877AA6EE267AF0EE676AE5EE2E
:10890800076ABDEEE67A17EE106A17EE100A9E4265
:10891800A8BF1846B142C8BF084607EE100AB8EE0D
:10892800C77A032A8CED027A00F09A8098ED0C7AC7
:10893800DDED0F6A25EE877AA6EE267AF0EE676AF5
:10894800E5EE076ABDEEE67A17EE106A17EE100A32
:108958009E42A8BF1846B142C8BF084607EE100A93
:10896800B8EEC77A042A8CED037A79D098ED107A9C
:10897800DDED106A25EE877AA6EE267AF0EE676AB4
:10898800E5EE076ABDEEE67A17EE106A17EE100AF2
:108998009E42A8BF1846B142C8BF084607EE100A53
:1089A800B8EEC77A052A8CED047A59D098ED147A76
:1089B800DDED116A25EE877AA6EE267AF0EE676A73
:1089C800E5EE076ABDEEE67A17EE106A17EE100AB2
:1089D8009E42A8BF1846B142C8BF084607EE100A13
:1089E800B8EEC77A062A8CED057A39D098ED187A50
:1089F800DDED126A25EE877AA6EE267AF0EE676A32
:108A0800E7EE056ABDEEE67A17EE106A17EE100A71
:108A18009E42A8BF1846B142C8BF084607EE100AD2
:108A2800B8EEC77A072A8CED067A19D098ED1C7A29
:108A3800DDED136A65EE875AE6EE265AE5EE257AED
:108A4800FDEEE77A17EE900A8342A8BF03468142FB
:108A5800C8BF0B4607EE903AF8EEE77ACCED077AF6
:108A6800BEF1000F40F04983002A40F0418344E3FF
:108A7800AB4B1B78013BDBB2FFF730BAA94B07932E
:108A88004FF47A761B68B6FBF3F3C3EB4316A6499B
:108A9800DFF8B88291F801A0A449B8F9060091F866
:108AA800009003EB8603DE00B6B2B74202F0F8820C
:108AB800D5F88810B5F93CE0EB6E4A1C07EE90EA51
:108AC8007344012AC5F88820EB66F8EEE77A02F0CD
:108AD800F282D5ED1E5AD5ED206A07EE102A37EE40
:108AE800E56AB8EEC75A012F86EE057A37EE257A81
:108AF80077EEC77A85ED1F7AE7EE866A85ED1E7AEE
:108B0800F0EE667AC5ED216AC5ED206A02F0EF86BF
:108B1800D5F89C10B5F93EE02B6F4A1C07EE90EA99
:108B28007344012AC5F89C202B67F8EEE77A02F017
:108B3800DB82D5ED235AD5ED256A07EE102A37EEEC
:108B4800E56AB8EEC75A012F86EE057A37EE257A20
:108B580077EEC77A85ED247AE7EE866A85ED237A83
:108B6800F0EE667AC5ED266AC5ED256A02F0E8865C
:108B7800D5F8B010B5F940E06B6F4A1C07EE90EAE3
:108B88007344012AC5F8B0206B67F8EEE77A02F063
:108B9800C482D5ED285AD5ED2A6A07EE102A37EE99
:108BA800E56AB8EEC75A012F86EE057A37EE257AC0
:108BB80077EEC77A85ED297AE6EE276A85ED287A79
:108BC800F0EE667AC5ED2B6AC5ED2A6A02F0E186F9
:108BD800A8F80600B5F8B430544A013B92F8009062
:108BE800A5F8B43007990023B9F1070F4B608B60E3
:108BF800CB607FF468A9FEF765FD059BDFF84C8123
:108C0800C01A94F8E831A8F80000002B3FF460A9D6
:108C1800013B84F8E83115B0BDEC0C8BBDE8F08F52
:108C280094ED6A7AB1F90000D4ED6B6AB1F902E00B
:108C38003F4AF4EEC76A80EAE0738EEAEE71A3EB6E
:108C4800E073F1EE10FAA1EBEE71B8BFF0EE476AEF
:108C58008B42B8BF0B4607EE103A1378B8EEC77AC6
:108C680027EE287A002B40F0F782324B93ED006A0A
:108C7800B4EECA6AF1EE10FA41F18E82F7EE005AAC
:108C880075EEC65A3BEE477A65EEAA5A2A4BA7EE0E
:108C9800256A93ED007A26EE076AB5EEC06AF1EE12
:108CA80010FA40F22287C9EE865AB7EE007AB0EE83
:108CB800476AA6EEE56AF0EE466AF4EEC76AF1EE98
:108CC80010FA88BFF0EE476AF5EEC06AF1EE10FAC6
:108CD800B8BFF0EE6B6A194B93ED007A67EE877AAE
:108CE800A7EEA68AFFF7E6B9154B164A2B4493ED73
:108CF800007AD2ED007A144B67EE277AF7EE006A15
:108D0800F4EEE67AF1EE10FA93ED007A88BFF0EE11
:108D1800667A67EE877A27EE888AFFF77CBA00BF03
:108D28002435002084660020EC630020384E0020A3
:108D3800B0480020B8480020AC480020A8480020CF
:108D4800BC240020A04800209C4800203C4E002065
:108D5800072B02F0828400230793D04ED04D33684E
:108D68000693580501F17782CE4BCF491F68B1F9B8
:108D780006A07A899245C0F2C982BAF5FA6F81F2E3
:108D8800BE82387AAAEB020303FB00F3C2F5FA624B
:108D980093FBF2F3C3F1640307EE903AF8EEE77A37
:108DA8009FEDC27A67EE877AC4ED417ADFF82093A7
:108DB800DFF820B3B9F81880B1F900309BF9042026
:108DC8009BF800009BF801C0A3EB080686EAE67E44
:108DD800002AAEEBE67E14BF01224FF0FF32BEF54B
:108DE800FA7FA8BF4FF4FA7E704580F2DD84AEEBBF
:108DF800000607EE906AF8EEE77AAD4E4345C6EDF9
:108E0800007A03DAF1EE677AC6ED007AB1F902E08A
:108E1800AEEB0803002BB8BF5B42B3F5FA7FA8BFDF
:108E28004FF4FA739842059380F2BA841B1A07EE3E
:108E3800903AF8EEE77AC645C6ED017A03DAF1EE24
:108E4800677AC6ED017AB1F90410A1EB080383EA49
:108E5800E370A0EBE370B0F5FA7FA8BF4FF4FA70A7
:108E68006045CCBFA0EB0C0C4FF0000C02FB0CFCD7
:108E780007EE90CAF8EEE77A4145069BC6ED027AFE
:108E8800BCBFF1EE677AC6ED027A13F480530593FE
:108E980000F04084BAF5FA6F5246A8BF4FF4FA6260
:108EA800B2F57A7F94F80831B8BF4FF47A72A2F518
:108EB8007A72002B40F047847E49DFF81CE281FB80
:108EC8000230D317C3EB6013581C6FF0630C3EF9E4
:108ED80010003EF913E00CFB0323A0EB0E0003FB8C
:108EE80000F381FB0321DB17C3EB61139E440FFAE8
:108EF8008EFE07EE90EA059BB8EEE78A86ED038AB8
:108F0800002B41F0B4816C4B198811F0400240F0FD
:108F18003F876A4B1B6813F0140F03D011F4027FCC
:108F280041F0F481664B1B789BB1B9F81A30534570
:108F38000FDB644B1B78012B02F03681192B02F0F2
:108F480033810E2B05D0082B03D00023B360C4F85F
:108F58003C3194F8423113B1890742F0138394F8F5
:108F68004831002B41F01D8199F81E10002900F0AE
:108F78001F84022902F03B81032901F0D183524961
:108F8800488899F81F100231C9B2002B02F02181DC
:108F9800002802F01E81DFF844E1DEF800A0B0FBF3
:108FA800FAF00FFA80FAA4F878A1A9B307EE90AA0C
:108FB800F8EEE77AF7EE006A86EEA77A0129D6ED91
:108FC800007AD4ED636A77EEE67A67EE877AC4EDC5
:108FD8005F7A21D0D6ED017AD4ED646A77EEE67A2D
:108FE800022967EE877AC4ED607A15D0D6ED027A49
:108FF800D4ED656A77EEE67A032967EE877AC4EDE1
:10900800617A09D0D6ED037AD4ED666A77EEE67A0E
:1090180067EE877AC4ED627A2C480078092803F055
:109028003283BAF1000F40F3C98391B394ED637AA8
:10903800D4ED5F7A77EE877A0129C4ED637AC6EDBD
:10904800007A21D094ED647AD4ED607A77EE877A4D
:109058000229C4ED647AC6ED017A15D094ED657ADB
:10906800D4ED617A77EE877A0329C4ED657AC6ED87
:10907800027A09D0D4ED667A94ED627A77EE877A2F
:10908800C4ED667AC6ED037A01390229B8BF022118
:10909800C9B2002B18BF022191E300BF94660020DB
:1090A800006400204C770020485F00200AD7233C4A
:1090B800184F00201F85EB510C420020C876002075
:1090C800112100207035002030540020384E002037
:1090D80020680020283500205077002054350020D3
:1090E8000A9B8D4D1B78D90700F14A812A7822B155
:1090F80092008A498A4825F0B3FF8A4B1B68002BE7
:1091080040F0F282884B1B789BB1287870B1DFF869
:109118001082DFF864920026F0B2D9F80030B8EC7B
:10912800010A9847287801368642F5DB7F4B1B6891
:1091380098477F4B1B78072B00F0E084012384F8C5
:10914800003115B0BDEC0C8BBDE8F08F794BC7ED45
:1091580000BA1B689342BEF6EDAF774B1A8800231E
:1091680084F8FC31002A41F09187744A744B1178D5
:10917800186881F00101FBF707F9FEF7E3BF714EAC
:10918800DFF8F89106F5F47806F51577F6EC017A2C
:1091980095ED080AD5F81432F8EEE77A404627EE3E
:1091A800800A9847A8F1E000D5F834319847A8F12B
:1091B8007000D5F8A4319847D6F8F400D5F8B8303F
:1091C800984708F124084745A9EC010ADED1FEF7C3
:1091D80073BE0A9A1278D20703D45B4A128BA4F89A
:1091E80020225A4A5A49128891ED037A07EE902AAA
:1091F800F8EEE77AB4EEE77AF1EE10FA41F2A881D8
:109208005449098807EE901AF8EEE77AB4EEE77A3F
:10921800F1EE10FAC1F2DD804F49504AD1ED006AF3
:1092280092ED006A4E49C4ED896ABCEEC75A76EEE3
:10923800665A15EE102AC4ED876AC4ED865A84ED85
:109248008A6AA4F820220122D1ED006A84F82C222F
:1092580077EE677AFFF76FB8424B93ED005AB5EE99
:10926800C05AF1EE10FA40F340843F4BD3ED004A68
:10927800F5EEC04AF1EE10FA40F3378434EEC77ABF
:1092880066EEE95A87EE246AC5EE856AB7EE007A7B
:10929800B4EEC76AF1EE10FA88BFB0EE476AB5EED1
:1092A800C06AF1EE10FA76EE876AB8BFB0EE6B6A64
:1092B80066EE266A01E52D4A92ED007AF0EEE76A3D
:1092C800F4EEC76AF1EE10FA7EF7C6AF284A92EDBF
:1092D800007AF0EECD6AF4EEC76AF1EE10FA7EF786
:1092E800BBAF244A99ED007AD2ED006AB0EEC77A96
:1092F800B4EEE67AF1EE10FA7EF5AEAF01220999E6
:10930800C4F8001284F8FC21FEF7AABF4FF07E5380
:10931800C4F804314AE500BF194E0020FC4800207B
:1093280070330020E4380020E8630020DC6000206F
:10933800384E0020CC48002020550020225500201F
:10934800245500203064002020680020B049002007
:10935800184F0020B24900209C49002014350020F5
:10936800B8490020AC480020B4480020E04800205C
:10937800DC480020E4480020D460002088660020F3
:109388002B78002B3FF4B9AED4ED6B3A94ED6A6AB2
:10939800D4ED877AF24A94ED867AD2ED005A94EDAC
:1093A800684AD4ED674ADFF8E483DFF8E4C3F4EEF3
:1093B800C63AF3EE046AF1EE10FA37EEA65A01F156
:1093C800008198ED026A26EE446AF0EE674AE6EEFE
:1093D800074AF4EEC54A34EEE66AF1EE10FA48BFE1
:1093E800B0EE656A012B8CED006A3FF486AE98ED0D
:1093F800066A26EE446AF0EE674AE6EE074AB4EEDD
:10940800E45A34EEE66AF1EE10FA88BFB0EE656A07
:10941800022B8CED016A3FF470AE98ED0A6A26EED5
:10942800446AF0EE674AE6EE074AF4EEC54A34EEBF
:10943800E66AF1EE10FA48BFB0EE656A032B8CEDD0
:10944800026A3FF45AAE98ED0E6A26EE446AF0EED0
:10945800674AE6EE074AB4EEE45A34EEE66AF1EEFD
:1094680010FAC8BFB0EE656A042B8CED036A3FF4AE
:1094780044AE98ED126A26EE446AF0EE674AE6EECC
:10948800074AF4EEC54A34EEE66AF1EE10FA48BF30
:10949800B0EE656A052B8CED046A3FF42EAE98EDAC
:1094A800166A26EE446AF0EE674AE6EE074AB4EE1C
:1094B800E45A74EEE66AF1EE10FAC8BFF0EE656A97
:1094C800062BCCED056A3FF418AED8ED1A6A66EEA5
:1094D800C46AF0EE674AE6EE874AB3EE046AB4EE71
:1094E800E45A74EEC66AF1EE10FAC8BFF0EE656A87
:1094F800072BCCED066A3FF400AED8ED1E6A26EEC7
:10950800C44AE4EE077AB4EEE75A77EEC67AF1EE8B
:1095180010FAC8BFF0EE657ACCED077AEDE5079949
:10952800904BD1ED017A93ED007AF0EEE77AF4EE04
:10953800C77AF1EE10FA7EF505AED1ED027AF0EEBB
:10954800E77AB4EEE77AF1EE10FA7EF7FBADD1EDEB
:10955800037AF0EEE77AB4EEE77AF1EE10FA7EF7E6
:10956800F1AD814B1B689B077FF5F7AD7F49804BB9
:10957800B3F90C20B1F900E07E48AEEB020E0068AA
:109588008EEAEE72A2EBEE728242BEF6DBADB3F962
:109598000E30B1F90220D21A82EAE273A3EBE27329
:1095A80098427EF7CFADD8E5734B99ED007AD3EDAD
:1095B800006AB0EEC77AB4EEE67AF1EE10FA7EF7FA
:1095C80061AEFEF75CBE07EE103A6C4BDFF8C48163
:1095D8001B78C4F8D071B8EEC77AF7EE006A132B7F
:1095E80086EE879AB8F90400B4F8D46195ED080AB4
:1095F80001F0B484624B634A93ED001AD3ED053A47
:1096080093ED122A93ED173AD3ED091AD3ED0E4ACA
:1096180093ED016A93ED064A93ED0A7AD3ED0F5A5A
:10962800D3ED132AD3ED186A93ED045AD3ED030A48
:1096380067EE897A69EE288A29EE088AE1EE273AE8
:1096480002EB86070021A2EE283AC4F8C411C4F838
:10965800C811E1EE884AA6EE274AE7EE085A93EDCC
:10966800167A93ED0D6A93ED021AD3ED0C1AC7ED35
:10967800003AE2EEA86A25EE635A27EE437A93EDA4
:109688000B2AD3ED152AC7ED204AA0EEE34A26EEB1
:10969800646AD3ED143A83ED054AA1EE275AF0EE39
:1096A800477AE1EEE45AA2EE086AE2EEC36AE3EE14
:1096B800A87A83ED065AC3ED0E5A83ED0F6A87ED3B
:1096C800403AC3ED176AC3ED187AC4F8CC11731C7D
:1096D80003F01F03A4F8D431A8F80400FEF7CEBAAB
:1096E800B0EE465AFEF760BE0CF098F90AE596ED22
:1096F800007A05EB4702B8EEC78A928F2AF817203E
:1097080028EE278AFEF7A6BB25F0B2FE2AF8170036
:10971800FEF7C2BBB9F81A209245C0F2ED85BAF53A
:10972800FA6FD4BFC2EB0A03C2F5FA634FF47A7139
:1097380001FB03F194F80801C2F5FA63B1FBF3F2F7
:1097480000283FF4B9AB94F809310F4902FB03F242
:1097580081FB0213D217C2EB6312FFF7ADBB00BF48
:10976800F8480020D8480020C87600201C42002075
:1097780030350020D4480020E4480020384E00202E
:10978800803F0020FC3C00201F85EB511C49002035
:10979800703300203C4E0020000000000AD7233C14
:1097A8005FED037AFFF747BB5FED057AFFF725BB4F
:1097B800A4F878118A46002B00F06A8102213B78D0
:1097C8005FED0A6AB87807EE903AF8EEE77AB0EEFD
:1097D800007A67EEA67AD74BF4EEC77AF1EE10FA64
:1097E80093F800E040F3928337EEC77ADFEDD26A50
:1097F800B0EE676AA7EE266AB0EE467A9FEDCF6AAA
:10980800D6ED006A66EE866AB0EEE66AC4ED676A6F
:1098180084ED6A6A98B105EE900AB8EEE55ADFED74
:10982800C85A66EEA64A25EE255AF7EE005A75EE96
:10983800C55A64EE864AE4EE855A66EEA56ADFEDFF
:10984800C15A7B7927EE257A27EE267ACBB1DFED50
:10985800BC6ADFEDBD5A26EE266A06EE903AF8EEAF
:10986800E66A26EE266AB4EEE56AF1EE10FA00F32F
:109878009686F7EE005A35EEC66AC5EE866A27EE7A
:10988800267ABEF10C0F9FEDB18ADFEDB16A00F0C8
:10989800DC85B4EEC87AF1EE10FA98BFB0EE478ACC
:1098A800B4EEE68AF1EE10FAB8BFB0EE668A84ED3F
:1098B8004D8A002900F0E080B0EE007AF4EEC77A15
:1098C800F1EE10FA05DD37EEC77ADFED9B6AE7EEB9
:1098D800267A96ED017ADFED996A27EE267AB0EEC0
:1098E800C76A84ED687A84ED6B6A98B106EE900ACF
:1098F800DFED935AF8EEE66A27EE075A66EEA56A98
:10990800F7EE005A75EEE65A25EE065AE5EE265AA7
:1099180027EE257ADFED8B6ABB7967EEA67A67EECC
:10992800877AABB107EE103AB8EEC77ADFED845A02
:10993800DFED856A27EE067A27EE257AB4EEE67A19
:10994800F1EE10FA40F32F86DFED826A67EEA67A11
:10995800BEF10C0F00F0A085DFED7C6A9FED7C7AEC
:10996800F4EEE67AF1EE10FA88BFF0EE667AF4EEDD
:10997800C77AF1EE10FAB8BFF0EE477A0129C4EDC4
:109988004E7A79DD7B78DFED6E6A07EE903AF8EE75
:10999800E77AB0EE007A67EEA67A7B7AF4EEC77AB9
:1099A800F1EE10FA05DD37EEC77ADFED636AE7EE10
:1099B800267A96ED027ADFED616A27EE267AB0EE16
:1099C800C76A84ED697A84ED6C6A9BB106EE903AB9
:1099D800DFED5B5AF8EEE66A27EE075A66EEA56AEF
:1099E800F7EE005A75EEE65A25EE065AE6EE855A67
:1099F80027EE257ADFED536AFB7967EEA67A67EEE4
:109A0800877A0BB307EE103AB8EEC77ADFED4C5AF7
:109A1800DFED4D6A27EE067A27EE257AB4EEE67A70
:109A2800F1EE10FA0CDCB5EEC07AF1EE10FA01F1A5
:109A3800C683B7EE006A36EE477AC6EE076A01E0DB
:109A4800DFED446A67EEA67ABEF10C0F00F01A85C6
:109A5800DFED3E6A9FED3E7AF4EEE67AF1EE10FA1B
:109A680088BFF0EE667AF4EEC77AF1EE10FAB8BF66
:109A7800F0EE477AC4ED4F7ABEF1090F00F0C884C2
:109A880099F82160002E40F05E84002384F8483164
:109A9800314B1B7823B9314EB278002A41F0FA8352
:109AA800244B1B78072B00F018850022072B84F81D
:109AB80000217EF490A8FDF705FE0590FEF78DB80D
:109AC800274B284C1A68284BDFF8A88094F8000127
:109AD800D2691B88A8F80020A8F8023000287FF473
:109AE8003AA90590214DFEF778B8DFED216AFFF716
:109AF800F2B843023EF55AAEFEF75CBEFDF7E2FD52
:109B08001C4BC01BD880FFF719BBFDF7DBFD094BC9
:109B18000B9A1B78DFF85C80801A012BA8F80200EA
:109B280000F0D483072B7EF4D5ABFDF7CBFD0746B9
:109B3800FEF7D1BB384E0020D7A368416F12033B14
:109B48000AD7233C00004843A4707D3F00C0F94475
:109B580000C0F9C40000C8426A530020A47600205F
:109B68000876002014230020E8310020006400203B
:109B7800000000003C4E0020BEF1000F41F0A88517
:109B880098ED007ADDED0C6ADFF8CCC325EE877A14
:109B9800A6EE867AF0EE676AE7EE056ABDEEE67A2B
:109BA80017EE106A17EE100A9E42A8BF1846B14277
:109BB800C8BF084607EE100AB8EEC77A012A8CED2E
:109BC800007A3FF495AA98ED047ADDED0D6A25EE4A
:109BD800877AA6EE867AF0EE676AE7EE056ABDEE4A
:109BE800E67A17EE106A17EE100A9E42A8BF1846CA
:109BF800B142C8BF084607EE100AB8EEC77A022A73
:109C08008CED017A3FF474AA98ED087ADDED0E6ABE
:109C180025EE877AA6EE867AF0EE676AE7EE056AA1
:109C2800BDEEE67A17EE106A17EE100A9E42A8BF3C
:109C38001846B142C8BF084607EE100AB8EEC77A00
:109C4800032A8CED027A3FF453AA98ED0C7ADDEDE5
:109C58000F6A25EE877AA6EE867AF0EE676AE7EE57
:109C6800056ABDEEE67A17EE106A17EE100A9E42F4
:109C7800A8BF1846B142C8BF084607EE100AB8EE9A
:109C8800C77A042A8CED037A3FF432AA98ED107A49
:109C9800DDED106A25EE877AA6EE867AF0EE676A21
:109CA800E7EE056ABDEEE67A17EE106A17EE100ABF
:109CB8009E42A8BF1846B142C8BF084607EE100A20
:109CC800B8EEC77A052A8CED047A3FF411AA98ED0C
:109CD800147ADDED116A25EE877AA6EE867AF0EE23
:109CE800676AE7EE056ABDEEE67A17EE106A17EEC8
:109CF800100A9E42A8BF1846B142C8BF084607EEE0
:109D0800100AB8EEC77A062A8CED057A3FF4F0A956
:109D180098ED187ADDED126A25EE877AA6EE867A36
:109D2800F0EE676AE7EE056ABDEEE67A17EE106AAE
:109D380017EE100A9E42A8BF1846B142C8BF08468F
:109D480007EE100AB8EEC77A072A8CED067A3FF4B8
:109D5800CFA998ED1C7ADDED136A65EE875AE6EE19
:109D6800265AE5EE257AFDEEE77A17EE900A834249
:109D7800A8BF03468142C8BF0B4607EE903AF8EEEB
:109D8800E77ACCED077A002A7FF4B2A9FFF7B5B9D4
:109D9800604BDFF8C8E1B3F90430B4F81001DFED27
:109DA8005E6A9FED5E7A8EFB03CEDB17C3EBAE03D4
:109DB8001B1A1BB207EE903AF8EEE77A67EEA67A1E
:109DC80077EE876ABDEEE66A16EE103A2033402B2E
:109DD80041F21882DFED526ABDEEE77A17EE103ACB
:109DE8002033402B01F20A829FED4E7AF4EEC77AB7
:109DF800F1EE10FA42F30784DFED4B5A9FED4B6A00
:109E080001E0F0EE477AF4EEC67AF1EE10FA37EE9A
:109E1800E57AF6DCDFED467AB4EEE77AF1EE10FA91
:109E280042F1ED83DFED405A9FED426A01E0B0EE6A
:109E3800677AB4EEC67AF1EE10FA77EE257AF6D4A0
:109E48009FED367AF4EEC77AF1EE10FA00F39985B1
:109E58009FED397AF4EEC77AF1EE10FA44BF9FED20
:109E6800347A77EE677A67EEA75A9FED345A9FEDFA
:109E7800346A9FED347AA5EE856A27EEA55AA5EED9
:109E8800867AE5EE077A96ED016AD6ED005A27EE56
:109E9800C67A65EEA77AA5EEA67AE6EE267A86ED6C
:109EA800007AC6ED017AFFF734B8274B5A79002AB1
:109EB8003EF4FFAA254A1278002A3EF4FAAA1B7833
:109EC800DFED234A07EE903A224BB8EE677A1B88FB
:109ED80007EE902A06EE903AF8EEE77AF8EE666A10
:109EE80067EE277AB7EE007AC7EEA63AF4EEE43AC0
:109EF800F1EE10FA88BFF0EE643AF4EEC73AF1EEEC
:109F080010FAB8BFF0EE473AFEF7D5BAB0EE677A66
:109F180074E400BF1C42002035FA8E3CDB0FC93FB9
:109F280000000000DB0F4940DB0FC940E4CB1641BD
:109F3800DB0F49C0E4CB16C1DB0FC9BF92E741B9BB
:109F48009730083C15A82ABE94760020164F0020AA
:109F5800713DAA3F004F0020703300206766666697
:109F6800BCF1000F00F0F083BEF1000F42F07E80DC
:109F7800DFF8D085B9F1000F41F0BF86D8ED006A4F
:109F8800DDED0C4ADFF8C0C565EEA66ABDEEC77AFE
:109F980017EE101AB0EE667AA4EE867AF0EE676ACB
:109FA800E7EE056ABDEEE67A17EE106A17EE100ABC
:109FB8009E42A8BF1846B142C8BF084607EE100A1D
:109FC800B8EEC77A012A8CED007A3FF491A898ED93
:109FD800047ADDED0D6A25EE877AA6EE867AF0EE34
:109FE800676AE7EE056ABDEEE67A17EE106A17EEC5
:109FF800100A9E42A8BF18468E42B8BF084607EE10
:10A00800100AB8EEC77A022A8CED017A3FF470A8DC
:10A0180098ED087ADDED0E6A25EE877AA6EE867A47
:10A02800F0EE676AE7EE056ABDEEE67A17EE106AAB
:10A0380017EE100A9E42A8BF18468E42B8BF0846BF
:10A0480007EE100AB8EEC77A032A8CED027A3FF4BD
:10A058004FA898ED0C7ADDED0F6A25EE877AA6EE0B
:10A06800867AF0EE676AE7EE056ABDEEE67A17EEE5
:10A07800106A17EE100A9E42A8BF18468E42B8BF53
:10A08800084607EE100AB8EEC77A042A8CED037A60
:10A098003FF42EA898ED107ADDED106A25EE877A48
:10A0A800A6EE867AF0EE676AE7EE056ABDEEE67A16
:10A0B80017EE106A17EE100A9E42A8BF18468E4285
:10A0C800B8BF084607EE100AB8EEC77A052A8CED25
:10A0D800047A3FF40DA898ED147ADDED116A25EEA7
:10A0E800877AA6EE867AF0EE676AE7EE056ABDEE35
:10A0F800E67A17EE106A17EE100A9E42A8BF1846B5
:10A108008E42B8BF084607EE100AB8EEC77A062A8C
:10A118008CED057A3EF4ECAF98ED187ADDED126A15
:10A1280025EE877AA6EE867AF0EE676AE7EE056A8C
:10A13800BDEEE67A17EE106A17EE100A9E42A8BF27
:10A1480018468E42B8BF084607EE100AB8EEC77A1E
:10A15800072A8CED067A3EF4CBAF98ED1C7ADDED3C
:10A16800136A65EE875AE6EE265AE5EE257AFDEE85
:10A17800E77A17EE900A8342A8BF03468142D8BF08
:10A18800194607EE901AF8EEE77ACCED077A002A1E
:10A198007EF4AEAFFEF7B1BFD64B93ED006AFEF783
:10A1A8007CBDD549D548D1F8EC10006844F6206E3E
:10A1B8007145A8BF7146B1F57A7FB8BF4FF47A717F
:10A1C80089B2C006A4F84A1141F18B83059800288A
:10A1D80040F0CF83CA48D0F80080B8F932C0DFF821
:10A1E80030E3D4F84C01AEFB01E14FEA911E642143
:10A1F80091FBFEF11429FDEEC87A04EB400AA8BFD2
:10A20800142101308142C4F84C0117EE90EADCBFFA
:10A218000020C4F84C0104EB4000AAF850E1B0F962
:10A22800501107EE901AF8EEE77A38EE678AFDEEDD
:10A23800C87ACDED057ABDF9140080EAE071A1EB8A
:10A24800E071614502F3BC81AE4908464FF07E518A
:10A258000160FEF789BEAB68002B3EF485AD05F1C1
:10A2680050012846984733680693FEF77DBD1D21A7
:10A27800A248FAF730FF00283EF445AEA24BDB783F
:10A28800002B7EF440AEDFEDA17AA14938EE678A53
:10A29800C8F5FA62FDEEC87A12B2CDED087ABDF9BA
:10A2A80020301B0381FB0301DB17C3EBA11302FB67
:10A2B80003F343F30F33434407EE903AB8EEE78ACB
:10A2C80086ED038AFEF71FBEDFF88082FDF7FAF9F4
:10A2D800904AD4F810321268C4F81002C31A9A1AB5
:10A2E8000746A8F80430A8F80620FDF7F4BFFDF7E4
:10A2F800E9F90B90FDF7FBBD1946FFF71BBA3B7A4E
:10A30800C3F1640307EE903AFEF748BD824B1B7811
:10A3180013F0100301F0A78494F81401D4F818314D
:10A3280096ED017A00280CBF01204FF0FF3003FBA7
:10A3380000F307EE903AF8EEE77A77EE877AC6ED03
:10A34800017AFEF7EFBD1E216C480592FAF7C3FEAD
:10A3580000283FF49AAB059A002A7FF496AB94F84C
:10A36800B431B34242F0B881664BD4ED6E7A93EDC6
:10A37800010AD4ED4F5A9FED696ADFED696A27EE4D
:10A38800E57A68EE277AA8EE007AE5EE807AB4EEF0
:10A39800C67AF1EE10FA88BFB0EE467AB4EEE67AE5
:10A3A800F1EE10FAF4EEC67AB8BFB0EE667AF1EEC6
:10A3B80010FA88BFF0EE467AF4EEE67AF1EE10FA7B
:10A3C800B8BFF0EE667A84ED4D7AC4ED4F7AFFF7A8
:10A3D8005CBBB4F82012914240F28F855149524A31
:10A3E800D1ED007A92ED007A5049C4ED897A77EE82
:10A3F800676AC4ED877A0122C4ED866A84ED8A7A99
:10A40800D1ED006ADFED4A7A84F82C22FDF793BF7C
:10A41800FDEEC87ADFF8348117EE903AA8F804A068
:10A42800A8F80630FFF72CBB424B1B88002B40F0E6
:10A438008385414A414B11781868F9F7A5FFD4F88C
:10A448000022099B9A1AFDF74CBEB4EEC87AF1EEC9
:10A4580010FA98BFB0EE478ABDEEC77AB4EEE68A26
:10A46800DFF8E880F1EE10FA17EE103AB8BFB0EE58
:10A47800668A84ED4D8AA8F8003000297FF41CAA6A
:10A48800FFF7FEBABDEEE77ADFF8C08017EE103AA4
:10A49800A8F80430FFF7DCBA9FED207ADFED206AD8
:10A4A800DFF8A880F4EEC77AF1EE10FA98BFB0EEA4
:10A4B800677AFDEEE77AB4EEE67AF1EE10FA17EE77
:10A4C800903AB8BFB0EE667A012984ED4E7AA8F8C2
:10A4D80002303FF757AAFFF7D3BAFDF7F3F8079A08
:10A4E800DFF86880164B801A1B78A8F80400FFF77D
:10A4F800DCBA00BFAC480020981C0020C0760020C1
:10A508003C42002000000020E053002000007A4474
:10A51800D34D6210543500209076002000C0F944D5
:10A5280000C0F9C49C49002014350020B849002017
:10A53800000000002055002022550020245500204E
:10A54800384E00201C490020703300203C4E00206B
:10A55800784A7949D2ED006A784A91ED006A127812
:10A56800C4ED896A84ED8A6A002A40F0C28476EED6
:10A57800C65AF0EE466ABCEEC76A7149C4ED865AFF
:10A5880016EE102AC4ED876AA4F82022FF22D1ED26
:10A59800006A84F82C2277EEC77AFDF7CCBEDFED8F
:10A5A800696AFFF76CB9B5EEC07AF1EE10FA00F1FE
:10A5B8000286B7EE006A36EE477AC6EE076AFFF7FC
:10A5C800C5B998ED016A26EE646AB0EE674AA6EE50
:10A5D800074AB4EEC45A34EE666AF1EE10FAC8BF00
:10A5E800B0EE656A012B8CED006A3EF486AD98EDFD
:10A5F800056A26EE646AB0EE674AA6EE074AB4EE2C
:10A60800C45A34EE666AF1EE10FAC8BFB0EE656A55
:10A61800022B8CED016A3EF470AD98ED096A26EEC6
:10A62800646AB0EE674AA6EE074AB4EEC45A34EE3E
:10A63800666AF1EE10FAC8BFB0EE656A032B8CEDBE
:10A64800026A3EF45AAD98ED0D6A26EE646AB0EEE1
:10A65800674AA6EE074AB4EEC45A34EE666AF1EECB
:10A6680010FAC8BFB0EE656A042B8CED036A3EF49D
:10A6780044AD98ED116A26EE646AB0EE674AA6EE1C
:10A68800074AB4EEC45A34EE666AF1EE10FAC8BF4F
:10A69800B0EE656A052B8CED046A3EF42EAD98ED9C
:10A6A800156A26EE646AB0EE674AA6EE074AB4EE6B
:10A6B800C45A74EE666AF1EE10FAC8BFF0EE656A25
:10A6C800062BCCED056A3EF418ADD8ED196A66EE96
:10A6D800E46AB0EE674AA6EE874AB3EE046AB4EEBF
:10A6E800C45A74EE466AF1EE10FAC8BFF0EE656A15
:10A6F800072BCCED066A3EF400ADD8ED1D6A66EE78
:10A70800E44AE4EE877AF4EEC57A77EEC67AF1EE9B
:10A7180010FAB8BFF0EE657ACCED077AFEF7EDBC1B
:10A7280099F82010C1EB411001EB8000C00080B205
:10A73800FEF727BCB0330020A0490020E0600020CD
:10A74800B44900200000C842DFF81485B9F1000FB1
:10A7580041F03681D8ED006ADDED0C4ADFF804C51A
:10A7680065EEA66ABDEEC77A17EE101AB0EE667AE5
:10A77800A4EE867AF0EE676AE7EE056ABDEEE67A41
:10A7880017EE106A17EE100A9E42A8BF1846B1428B
:10A79800C8BF084607EE100AB8EEC77A012A8CED42
:10A7A800007A3EF45DA998ED047ADDED0D6A25EE98
:10A7B800877AA6EE867AF0EE676AE7EE056ABDEE5E
:10A7C800E67A17EE106A17EE100A9E42A8BF1846DE
:10A7D8008E42B8BF084607EE100AB8EEC77A022ABA
:10A7E8008CED017A3EF43CA998ED087ADDED0E6A0D
:10A7F80025EE877AA6EE867AF0EE676AE7EE056AB6
:10A80800BDEEE67A17EE106A17EE100A9E42A8BF50
:10A8180018468E42B8BF084607EE100AB8EEC77A47
:10A82800032A8CED027A3EF41BA998ED0C7ADDED33
:10A838000F6A25EE877AA6EE867AF0EE676AE7EE6B
:10A84800056ABDEEE67A17EE106A17EE100A9E4208
:10A85800A8BF18468E42B8BF084607EE100AB8EEE1
:10A86800C77A042A8CED037A3EF4FAA898ED107A98
:10A87800DDED106A25EE877AA6EE867AF0EE676A35
:10A88800E7EE056ABDEEE67A17EE106A17EE100AD3
:10A898009E42A8BF18468E42B8BF084607EE100A67
:10A8A800B8EEC77A052A8CED047A3EF4D9A898ED5B
:10A8B800147ADDED116A25EE877AA6EE867AF0EE37
:10A8C800676AE7EE056ABDEEE67A17EE106A17EEDC
:10A8D800100A9E42A8BF18468E42B8BF084607EE27
:10A8E800100AB8EEC77A062A8CED057A3EF4B8A8A5
:10A8F80098ED187ADDED126A25EE877AA6EE867A4B
:10A90800F0EE676AE7EE056ABDEEE67A17EE106AC2
:10A9180017EE100A9E42A8BF18468E42B8BF0846D6
:10A9280007EE100AB8EEC77A072A8CED067A3EF4CD
:10A9380097A898ED1C7ADDED136A65EE875AE6EE66
:10A94800265AE5EE257AFDEEE77A17EE900A83425D
:10A95800A8BF03468142D8BF194607EE901AF8EE01
:10A96800E77ACCED077ABEF1000F7EF4C6ABFEF7AE
:10A978007BB8AE48D0F80080B8F832C04FEA5C0C1B
:10A988002DE49FEDAB7A77EE677AFFF76CBADFF8C4
:10A99800D892D4ED017A94ED006AB9F80000D9F89C
:10A9A800143077EEA77AF0EE006AB0EE677AA6EE7A
:10A9B800267A013804EBC002D6EE267A083A10331C
:10A9C800F6EE003A27EE237A67EEA37A84ED207A32
:10A9D800C4ED217A974CA64604F1800192ED027AE3
:10A9E80092ED036ADEED036ADEED027A53ED014A69
:10A9F80013ED025A37EE674A76EEC65A77EE277A93
:10AA0800E4EE845A0138A2F10802E5EE047A0EF168
:10AA1800080E03F1080336EE267A01F10801E4EE88
:10AA2800877AE5EE475A67EEA37A25EEA37AC1ED59
:10AA3800007A81ED017AD1D1142F7DF4DAA9FCF7DF
:10AA480041FE069BDFF82482C01AA8F80200D4F859
:10AA5800D861FDF7CEB9D4F8DC81B4F8D4A1764B2F
:10AA6800CAF120095FFA89F90AEB481E03EB8E0E3A
:10AA78005FEA990301F0FC85013318016F49704AB8
:10AA88000EEB000C0EF1100313ED024A13ED035AFE
:10AA980013ED016A13ED047A51ED024A51ED035AA0
:10AAA80051ED016A51ED047A64EE244A65EE255AA7
:10AAB80066EE266A67EE277A10339C4542ED024A15
:10AAC80042ED035A42ED016A42ED047A01F11001A8
:10AAD80002F11002D8D15B49A0F11002964401EBB3
:10AAE800020C224419F0030309D0BEEC017AFCECF5
:10AAF800017A67EE277A013BE2EC017AF5D1BAF1E7
:10AB0800000F41F05982142F7DF473A9FCF7DAFD88
:10AB1800069BDFF85881D4F8D861C01AA8F802005B
:10AB2800FDF767B9DFF840914248D9F80820B9F82D
:10AB38000C1023F0B1F9444B1F78142F01F0A586AF
:10AB4800D4F8D8610136C4F8D86122E7D4F8DC918A
:10AB58003E4A3F4BDFED3F7AD3ED008A3E4B4FEA4A
:10AB6800C9010A44F8EE688A928809EE102A643A04
:10AB7800C82AA8BFC82268EEA78AF8EE497A782AB8
:10AB8800B8BF782268EEA78A07EE902A4944B0EE4B
:10AB9800680A03EB8108B8EEE78A24F0B5FCB8EE42
:10ABA800C99AF0EE409AB0EE680A24F00FFC38EE2D
:10ABB800097A79EE487A28EE098A67EE877AB7EE3D
:10ABC800006A88EE277A142FF8EE007A77EE076A83
:10ABD80060EE277A89EEA67A77EE065A36EE477A3D
:10ABE800C6EE256A67EEA67A27EE267AC8ED006AD1
:10ABF80088ED047AC8ED026AC8ED017AC8ED037AD7
:10AC080001F06986154B104A09F1010983FB0938DF
:10AC1800A8EBE97808EB48080136A9EB080817788B
:10AC2800C4F8D861C4F8DC8117E700BF3C420020B3
:10AC3800DB0F494014230020FC3C00208C3E002000
:10AC4800242300207C3E0020384E0020FC3E0020BB
:10AC58008466002027D4D2361866002056555555EC
:10AC68001C49002070330020E43C00203C4E0020AA
:10AC7800DFF80494B9F800E0D9F804C04FEA5E0898
:10AC88004FEA880204EB8E065FEADE0E04EB02034D
:10AC980000F0A08010320EF1010EEB4803EB0E1EFF
:10ACA800324410330CF1100706F1100151ED032A5C
:10ACB80051ED043A10ED043A10ED032A51ED026A01
:10ACC80011ED016A10ED020A10ED018A12ED044A35
:10ACD80012ED035A53ED044A53ED035A13ED027A69
:10ACE80053ED017A52ED020A12ED011A73EE238A2E
:10ACF80072EE221A40ED048A40ED031A70EE268A9D
:10AD080078EE061A40ED028A40ED011A74EE848A44
:10AD180075EE851A43ED048A43ED031A77EE208A0F
:10AD280077EE811A43ED028A43ED011A73EE633A16
:10AD380075EE655A17ED035A32EE623A74EE644ABC
:10AD480065EE631A17ED044A23EE052A64EE652AB8
:10AD5800E3EE041A10339E4524EE843AA3EE842AC7
:10AD680000F1100007F11007A5EE853A01F1100176
:10AD780002F11002E4EE852A41ED071A01ED082AD6
:10AD880002ED073A42ED082A57ED055A17ED065A23
:10AD980070EE666A38EE466A30EEC77A71EE677A08
:10ADA80026EE253A65EEE63A25EE674A67EE054A4D
:10ADB800E6EE053AA6EE853AA7EE254AE7EEA54A5D
:10ADC80001ED063A41ED053A02ED064A42ED054A23
:10ADD8007FF46CAF1FFA88F8624641469B481EF024
:10ADE800A3F84146D9F8042030461EF09DF8984B48
:10ADF8001B78142B7FF42BAE21E6DFF8809299F8AC
:10AE08000020900801F0F485DFF874C200F1010811
:10AE18004FEA48180CEB080E0CF12003ACF1700156
:10AE280013ED076A53ED056A13ED037A53ED017AC2
:10AE380053ED025A13ED084A53ED064A13ED045A2E
:10AE480026EE066A66EEA66A27EE077A67EEA77A06
:10AE5800A4EE046A20339E45E4EEA46A01F11001D1
:10AE6800A5EE057AE5EEA57AF1EEC65AB1EEE66AE8
:10AE7800F1EEC76AB1EEE77A41ED085A01ED076ACB
:10AE880041ED066A01ED057ACAD1A8F12008C4444B
:10AE980004EB001012F0030318BF0CF1080C0FD0DC
:10AEA8005CED017A1CED027A67EEA77A013BE7EECA
:10AEB800077A0CF1080CB1EEE77AA0EC017AEFD131
:10AEC800142F01F08C840136C4F8D861FCF7FABE5F
:10AED800FCF7F8FB5E4B06901F78142F05BFDFF8D0
:10AEE800A481D4F8D861D4F8D861A8F80060FCF738
:10AEF800CEBE76EE665AFFF73EBB564A5649D2EDAD
:10AF0800007A564A91ED007A1278C4ED897A84ED78
:10AF18008A7A002A01F04E8377EE676A5049C4EDB9
:10AF2800877AC4ED866AFF22D1ED006ADFED4D7A9B
:10AF380084F82C22FDF7FFB94B494B69002B3DF4EF
:10AF4800D0A84A484A4B008893FBF0F00B684FF0B2
:10AF5800010E186081F811E0FDF7C3B8454FDFF81E
:10AF6800289197ED004A97ED057AD7ED014A97EDBC
:10AF7800066AD7ED046A97ED035AD7ED025A67EED1
:10AF8800897A09EB8603A4EE277AA4EEA76A66EE0F
:10AF9800C76AA5EE476AE5EEA76A20EE070A87EDBD
:10AFA800056AC7ED066A83ED007A29EE088A24F05F
:10AFB8005FFA69EE288AD7ED0E5AD7ED176A97ED32
:10AFC800091AD7ED121A97ED0F5A97ED187A97EDDF
:10AFD8000A2AD7ED132A97ED0D6AD7ED167A97ED61
:10AFE8000C3AD7ED0B3A97ED154AD7ED144AE1EE36
:10AFF800085A002209EB8603E8EEA16A00B2C4F8F9
:10B00800C421A2EE085AC4F8C821C4F8CC21A8EE7D
:10B01800A27A26EE656A67EEE67AA3EE655AA3EE93
:10B02800886AA6EEC47AE8EEA47A87ED0E5AC3EDD4
:10B03800205A87ED0F6AC3ED406A87ED177AC7ED8E
:10B04800187AFEF744BB00BF2423002014230020F5
:10B05800384E0020B0330020A0490020E0600020D6
:10B06800B449002000000000285500204055002069
:10B0780020A10700803F0020E43C0020DE3C0020A7
:10B08800942300203C4E0020FC3C0020BD494A6926
:10B09800002A3DF457A80A6813604B74FDF752B8AC
:10B0A800B5F93C306A6207EE903A0122F8EEE77A89
:10B0B800EB66C5F888200023012FC5ED1F7AC5ED82
:10B0C8001E7AC5F8803001F0A682B7427DF420AD23
:10B0D800B5F93E302B6707EE903A00220123F8EECF
:10B0E800E77AAA62C5F89C300023012FC5ED247ABF
:10B0F800C5ED237AC5F8943001F08982B7427DF412
:10B1080037ADB5F940306B6707EE903A002201235E
:10B11800F8EEE77AEA62C5F8B0300023012FC5EDF2
:10B12800297AC5ED287AC5F8A8307DF451AD9FED90
:10B13800968AB9F1030F46D0BAF1000F09D007EE8D
:10B1480090AAF8EEE77AF4EEC87AF1EE10FA01F177
:10B158009C848E4A6B6F126894F8E011A8F8060078
:10B1680003EB560393FBF6F60023EE629362136338
:10B17800D36231B1864B1B8823F40063002B7DF426
:10B1880029AD844B1B6813F4003341F030828249A7
:10B198001A46C85C012803F10C0300F08A850132C5
:10B1A800152AF6D1FDF716BD7C4B9B7B002B3DF491
:10B1B800CCAEFDF7CEBEF7EE006AFEF7C7BBF7EEE2
:10B1C800006AFEF73FBCB0EE480A24F051F900B21D
:10B1D800B2E7B4F878A10AF1FF3A0FFA8AFABAF19D
:10B1E800000FA4F878A13DF720AFFEF7E4BAB4F851
:10B1F8004A0100F57A7080B2FDF7C3BEDFED627ACE
:10B20800FEF741BEF4EEC77AF1EE10FA41F3DF82A1
:10B21800DFED635A9FED636A01E0F0EE476AF4EEF2
:10B22800C66AF1EE10FA36EEE57AF6DCDFED5E6A14
:10B23800B4EEE67AF1EE10FA41F1CD82DFED585A1C
:10B248009FED5A6A01E0B0EE667AB4EEC67AF1EE86
:10B2580010FA77EE256AF6D49FED557AF4EEC76AB0
:10B26800F1EE10FA40F3EB849FED527A77EE666ABE
:10B2780066EEA65A9FED505A9FED506A9FED507AA0
:10B28800A5EE856A26EEA55AA5EE867AE5EE076A4A
:10B29800FEF7A2BD4B4F3B78013B0D2B17D8DFE8DB
:10B2A80013F0B3006601C0009900160016005001A3
:10B2B8003C010F01F9005D00520033010E001F2010
:10B2C800059221F0ADFF059A08B901233B70012AC8
:10B2D80000F05286F378002B3EF4E2AB3A4B1B7831
:10B2E800D80706D4059213F06BF8059A002841F0A8
:10B2F800D882364ED4F8C0113368994201F2D88208
:10B308003B78012B3EF4CCAB94F8BC21002A3EF4E8
:10B31800C7AB0B2B0DD801229A4040F6030112EA65
:10B3280001080BD112F4C06F03D0093B012B41F285
:10B338008B84274B32685A600B233B70002384F8B8
:10B34800BC31FEF7ADBB012A01D1FAF769F80D232C
:10B3580013203B701CF090FDB278B8E71C4B1B49DA
:10B368005B680968C8338B4204D323F01BFEB278AC
:10B378000028ACD0032A01F0318401233B70B27855
:10B38800A5E700BF2855002000000000087600202F
:10B39800CC76002050470020FC390308C0700020FC
:10B3A800DB0FC940E4CB1641DB0F49C0E4CB16C123
:10B3B800DB0FC93FDB0F494092E741B99730083CA2
:10B3C80015A82ABE9544002068740020485500201E
:10B3D8001835002011F098F9AB4A0292A2F10C033B
:10B3E800262101930091A2F10A035021163A49201F
:10B3F80009F0D6FD98B9A54BB27818604FF0FF3127
:10B40800596007233B7062E7A14B1B78DB0701F10A
:10B4180066831F2021F004FF08B10C233B70B2782B
:10B4280055E7DFF8688211F06FF99A4AD8F80430C6
:10B43800126864339342F2D2402011F03BF900289D
:10B44800EDD1D8F80030DFF884B2DFF864A24FF00D
:10B4580040090FE011F00CFADAF80020D8F80030B3
:10B46800013A0133B9F10109CAF80020C8F80030DF
:10B4780001F0E3831BF803301846002BEAD10023C0
:10B488004FF0FF32C8F800300423C8F804203B709E
:10B49800B2781CE7804B1B78002B01F0A4821A209D
:10B4A80021F0BEFE002841F09E8294F8BC31002BAA
:10B4B80041F0998209233B7009F046F8B27806E713
:10B4C8001A2021F0ADFE0028F6D0744B1B88002B03
:10B4D800F2D1734B4520D3F8008011F0C9F90E2042
:10B4E80011F0C6F9404608F0DFFCDDF8248040463C
:10B4F80008F0DAFC6B4A6C4B12681A6040460A2363
:10B508003B7008F055FDD7E7012A01F0DA820E23D7
:10B5180013203B701CF0B0FC81E711F0F5F809F03E
:10B5280049F800283FF47BAF23F03CFD00283FF4A6
:10B5380076AF5C4A5C4B12681A600A233B70B2789B
:10B54800C5E611F0E1F8594B002105208DE803000C
:10B55800A3F108020291532009F022FD00287FF48C
:10B568005EAF4A4BB278186008233B70AFE6494B90
:10B5780046491B684B604E4800230B60032103605B
:10B588003970A4E64B49DFED4C7A91ED080A08932F
:10B59800B4EEE70AF1EE10FA40F264850A9223F05D
:10B5A800FDFFD4ED517A20EE270A23F061FFB0F5B4
:10B5B800617F0A9A089B00F3908607EE900AF8EEDE
:10B5C800E76ADFED3E7A66EEA76A07EE903AB8EED4
:10B5D800E77AFDEEE67A17EE903A2033402B41F2F7
:10B5E80088819FED370A089223F042FF00B207EEE8
:10B5F800900A089AF8EEE77A38EE278A86ED038AE9
:10B60800FDF7ADBC0A9B93F800E00EF0010EBEF109
:10B61800000F7DF472ADFDF727BA2A4BDFED2A7AC9
:10B628001E68C4ED7B7A16F0805640F05A8310F4F9
:10B63800800600F0BB810026B6EE007A67EE877AB6
:10B64800F4EEE57AF1EE10FAC8BFF0EE675A40F36F
:10B658004883C4ED8C5AFDF7ADB8FCF733F8079072
:10B66800FDF77BBB74EE677AB7EE007AF4EEC77A23
:10B67800F1EE10FAC4ED7B7A40F3B18784EEA77A35
:10B688008DED0C7AFDF78CB8BE1D03081835002027
:10B698006874002048550020C435002094330020E9
:10B6A80090330020A43300209C330020781F030827
:10B6B8004C450020DC4600208FC2753CD06D393ADD
:10B6C80000000000C076002000000080581D03081C
:10B6D800BAF1000F00F0588698ED007ADDED0C6A9B
:10B6E800DFF8D0C825EE877AA6EE867AF0EE676A8C
:10B6F800E7EE056ABDEEE67A17EE106A17EE100A55
:10B708009E42A8BF1846B142C8BF084607EE100AB5
:10B71800B8EEC77A012A8CED007A3DF4EEAC98EDCC
:10B72800047ADDED0D6A25EE877AA6EE867AF0EECC
:10B73800676AE7EE056ABDEEE67A17EE106A17EE5D
:10B74800100A9E42A8BF1846B142C8BF084607EE75
:10B75800100AB8EEC77A022A8CED017A3DF4CDAC16
:10B7680098ED087ADDED0E6A25EE877AA6EE867AE0
:10B77800F0EE676AE7EE056ABDEEE67A17EE106A44
:10B7880017EE100A9E42A8BF1846B142C8BF084625
:10B7980007EE100AB8EEC77A032A8CED027A3DF458
:10B7A800ACAC98ED0C7ADDED0F6A25EE877AA6EE43
:10B7B800867AF0EE676AE7EE056ABDEEE67A17EE7E
:10B7C800106A17EE100A9E42A8BF1846B142C8BFB9
:10B7D800084607EE100AB8EEC77A042A8CED037AF9
:10B7E8003DF48BAC98ED107ADDED106A25EE877A82
:10B7F800A6EE867AF0EE676AE7EE056ABDEEE67AAF
:10B8080017EE106A17EE100A9E42A8BF1846B142FA
:10B81800C8BF084607EE100AB8EEC77A052A8CEDAD
:10B82800047A3DF46AAC98ED147ADDED116A25EEE0
:10B83800877AA6EE867AF0EE676AE7EE056ABDEECD
:10B84800E67A17EE106A17EE100A9E42A8BF18464D
:10B85800B142C8BF084607EE100AB8EEC77A062AF2
:10B868008CED057A3DF449AC98ED187ADDED126A55
:10B8780025EE877AA6EE867AF0EE676AE7EE056A25
:10B88800BDEEE67A17EE106A17EE100A9E42A8BFC0
:10B898001846B142C8BF084607EE100AB8EEC77A84
:10B8A800072A8CED067A3DF428AC98ED1C7ADDED7C
:10B8B800136A65EE875AE6EE265AE5EE257AFDEE1E
:10B8C800E77A17EE902A9342A8BF13468A42A8BF88
:10B8D800194607EE901AF8EEE77ACCED077AFDF7ED
:10B8E8000CBC0698C0003EF571ACFDF73DBB012AC3
:10B8F80040F3918607EE101AB8EEC77AC7EE876A4A
:10B90800B1EEE68AB9F1030F14D0BAF1000F09D0ED
:10B9180007EE90AAF8EEE77AF4EEC87AF1EE10FA9C
:10B9280001F1B380EB6E03EB560393FBF6F36B6206
:10B93800FFF7CBBBB0EE480A23F09AFD00B2E4E76C
:10B94800012A40F3648607EE101AB8EEC77AC7EEEC
:10B95800876AB1EEE68AB9F1030F14D0BAF1000F85
:10B9680009D007EE90AAF8EEE77AF4EEC87AF1EE7D
:10B9780010FA01F18A802B6F03EB560393FBF6F361
:10B98800AB62FFF7BBBBB0EE480A23F071FD00B213
:10B99800E4E7012A7FF7CBAB07EE101AB8EEC77AB7
:10B9A800C7EE876AB1EEE68AFFF7C3BBB6EE007A48
:10B9B800F4EEC75AF1EE10FA3FF73EAEFCF7FABEC6
:10B9C800D8ED004A9DED0C4ADFF8E8C565EEA44ABB
:10B9D800FDEEC73AE4EE064AB0EE674AA4EE854AA1
:10B9E80013EE901AF4EEC46AF1EE10FAF0EE444A3F
:10B9F80088BFF0EE474AFDEEE44A14EE900A14EED2
:10BA0800906A9842A8BF1E468142C8BF0E4604EEFF
:10BA1800906AF8EEE44A012ACCED004A3DF420A8E9
:10BA2800D8ED044A9DED0D4A65EEA44AE4EE064AB7
:10BA3800B0EE674AA4EE854AF4EEC46AF1EE10FA55
:10BA4800F0EE444A88BFF0EE474AFDEEE44A14EEB1
:10BA5800900A14EE906A9842A8BF1E468842B8BF62
:10BA68000E4604EE906AF8EEE44A022ACCED014A4A
:10BA78003CF4F6AFD8ED084A9DED0E4A65EEA44AAF
:10BA8800E4EE064AB0EE674AA4EE854AF4EEC46ACC
:10BA9800F1EE10FAF0EE444A88BFF0EE474AFDEEA8
:10BAA800E44A14EE900A14EE906A9842A8BF1E4623
:10BAB8008842B8BF0E4604EE906AF8EEE44A032ABC
:10BAC800CCED024A3CF4CCAFD8ED0C4A9DED0F4AC0
:10BAD80065EEA44AE4EE064AB0EE674AA4EE854A4B
:10BAE800F4EEC46AF1EE10FAF0EE444A88BFF0EEC4
:10BAF800474AFDEEE44A14EE900A14EE906A984222
:10BB0800A8BF1E468842B8BF0E4604EE906AF8EEFB
:10BB1800E44A042ACCED034A3CF4A2AFD8ED104A1B
:10BB28009DED104A65EEA44AE4EE064AB0EE674A77
:10BB3800A4EE854AF4EEC46AF1EE10FAF0EE444A37
:10BB480088BFF0EE474AFDEEE44A14EE900A14EE80
:10BB5800906A9842A8BF1E468842B8BF0E4604EEB7
:10BB6800906AF8EEE44A052ACCED044A3CF478AF32
:10BB7800D8ED144A9DED114A65EEA44AE4EE064A52
:10BB8800B0EE674AA4EE854AF4EEC46AF1EE10FA04
:10BB9800F0EE444A88BFF0EE474AFDEEE44A14EE60
:10BBA800900A14EE906A9842A8BF1E468842B8BF11
:10BBB8000E4604EE906AF8EEE44A062ACCED054AF1
:10BBC8003CF44EAFD8ED184A9DED124A65EEA44AF2
:10BBD800E4EE064AB0EE674AA4EE854AF4EEC46A7B
:10BBE800F1EE10FAF0EE444A88BFF0EE474AFDEE57
:10BBF800E44A14EE900A14EE906A9842A8BF1E46D2
:10BC08008842B8BF0E4604EE906AF8EEE44A072A66
:10BC1800CCED064A3CF424AFD8ED1C4A9DED134AFE
:10BC280065EEA45AE6EE045AE5EE257AF4EEE76AE4
:10BC3800F1EE10FAC8BFF0EE477AFEF784BE9FED2A
:10BC4800D87AF4EEC76AF1EE10FA44BF9FEDD57AC0
:10BC580077EE666AFFF70CBB8223FCF7B6B8DFED18
:10BC6800D27AFCF77DB89BF803C0BCF1000F00F056
:10BC78004E83B4F91CC19BF802E0AAEB0C0888EAD1
:10BC8800E870A0EBE870704540F3D784E245C8BF80
:10BC9800CEF1000E07EE90EAF8EEE77A012038EED2
:10BCA800278AC4F8203184F8240186ED038AFDF739
:10BCB80039B9D4F8E46153003EB1981801EB80001B
:10BCC80076784078B042BCF485AF134401EB830129
:10BCD8000023C4F8E411A4F83432C4F83832FCF76D
:10BCE80079BFB7EE007A77EE677AF4EEE75AF1EEAD
:10BCF80010FA88BFF0EE675AABE4D8ED004A9DED24
:10BD08000C4ADFF8B0C265EEA44AFDEEC73AE4EE8D
:10BD1800064AB0EE674AA4EE854A13EE901AF4EE8E
:10BD2800C46AF1EE10FAF0EE444A88BFF0EE474AD2
:10BD3800FDEEE44A14EE900A14EE906A9842A8BF09
:10BD48001E468142C8BF0E4604EE906AF8EEE44AE9
:10BD5800012ACCED004A3DF4CBA9D8ED044A9DED6B
:10BD68000D4A65EEA44AE4EE064AB0EE674AA4EE30
:10BD7800854AF4EEC46AF1EE10FAF0EE444A88BF40
:10BD8800F0EE474AFDEEE44A14EE900A14EE906A8B
:10BD98009842A8BF1E468842B8BF0E4604EE906A75
:10BDA800F8EEE44A022ACCED014A3DF4A1A9D8ED07
:10BDB800084A9DED0E4A65EEA44AE4EE064AB0EE46
:10BDC800674AA4EE854AF4EEC46AF1EE10FAF0EE82
:10BDD800444A88BFF0EE474AFDEEE44A14EE900A62
:10BDE80014EE906A9842A8BF1E468842B8BF0E4615
:10BDF80004EE906AF8EEE44A032ACCED024A3DF4D8
:10BE080077A9D8ED0C4A9DED0F4A65EEA44AE4EEF9
:10BE1800064AB0EE674AA4EE854AF4EEC46AF1EE2B
:10BE280010FAF0EE444A88BFF0EE474AFDEEE44AC5
:10BE380014EE900A14EE906A9842A8BF1E468842F3
:10BE4800B8BF0E4604EE906AF8EEE44A042ACCED38
:10BE5800034A3DF44DA9D8ED104A9DED104A65EE10
:10BE6800A44AE4EE064AB0EE674AA4EE854AF4EE28
:10BE7800C46AF1EE10FAF0EE444A88BFF0EE474A81
:10BE8800FDEEE44A14EE900A14EE906A9842A8BFB8
:10BE98001E468842B8BF0E4604EE906AF8EEE44AA1
:10BEA800052ACCED044A3DF423A9D8ED144A9DEDAA
:10BEB800114A65EEA44AE4EE064AB0EE674AA4EEDB
:10BEC800854AF4EEC46AF1EE10FAF0EE444A88BFEF
:10BED800F0EE474AFDEEE44A14EE900A14EE906A3A
:10BEE8009842A8BF1E468842B8BF0E4604EE906A24
:10BEF800F8EEE44A062ACCED054A3DF4F9A8D8ED57
:10BF0800184A9DED124A65EEA44AE4EE064AB0EEE0
:10BF1800674AA4EE854AF4EEC46AF1EE10FAF0EE30
:10BF2800444A88BFF0EE474AFDEEE44A14EE900A10
:10BF380014EE906A9842A8BF1E468842B8BF0E46C3
:10BF480004EE906AF8EEE44A072ACCED064A3DF47E
:10BF5800CFA8D8ED1C4A9DED134A65EEA45AE6EE2B
:10BF6800045AE5EE257AF4EEE76AF1EE10FAC8BF56
:10BF7800F0EE477AFEF7FBB80C490D4B89681B6851
:10BF880099423FF6A7A93B780C3B022B7DF688AD7A
:10BF980094F8BC313A70002B3DF482ADFFF7CEB96E
:10BFA800DB0FC9BFDB0F49C000000243581C00204B
:10BFB8005835002070330020EB4B4FEA890E5FEABA
:10BFC8009A0901EB0E0C03EBC818A64400F0808513
:10BFD80009F101094FEA091908EB090008F11003F2
:10BFE8000CF110010EF1100213ED024A13ED035A81
:10BFF80013ED016A13ED047A51ED024A51ED035A2B
:10C0080051ED016A51ED047A64EE244A65EE255A31
:10C0180066EE266A67EE277A1033984242ED024AA6
:10C0280042ED035A42ED016A42ED047A01F1100132
:10C0380002F11002D8D1A9F11009C8440CEB09018A
:10C04800CE441AF0030A3EF45EADB8EC017AF1EC86
:10C05800017A67EE277ABAF1010AEEEC017AF4D197
:10C06800FEF751BDDFEDC17AFFF7C6BABAF1000F8E
:10C0780000F0C583DFF808839DED0C4AD8ED004A2F
:10C0880065EEA44AE4EE064AB0EE674AA4EE854A95
:10C09800F0EE444AB9F1000F06D0F4EE446AF1EE2E
:10C0A80010FAC8BFF0EE474ABDEEC77A17EE101A6D
:10C0B800BDEEE47A04EE901A17EE100A814200F3FE
:10C0C800F0849842A8BF184607EE100AB8EEC77A5F
:10C0D800DFF8B0C2012A8CED007A3DF40EA898ED85
:10C0E800047A9DED0D4A25EE877AA4EE067AB0EE25
:10C0F800674AA7EE054AB0EE447AB9F1000F00F09E
:10C10800B984F4EEC46AF1EE10FA40F3B384084639
:10C118009842A8BF184607EE100AB8EEC77A022A56
:10C128008CED017A3CF4E9AF98ED087A9DED0E4A62
:10C1380025EE877AA4EE067AB0EE674AA7EE054A9E
:10C14800B0EE447AB9F1000F00F08984F4EEC46AC5
:10C15800F1EE10FA40F3838408469842A8BF1846C7
:10C1680007EE100AB8EEC77A032A8CED027A3CF47F
:10C17800C4AF98ED0C7A9DED0F4A25EE877AA4EEB0
:10C18800067AB0EE674AA7EE054AB0EE447AB9F1EE
:10C19800000F00F05984F4EEC46AF1EE10FA40F38F
:10C1A800538408469842A8BF184607EE100AB8EE0E
:10C1B800C77A042A8CED037A3CF49FAF98ED107A85
:10C1C8009DED104A25EE877AA4EE067AB0EE674A0E
:10C1D800A7EE054AB0EE447AB9F1000F00F02984C1
:10C1E800F4EEC46AF1EE10FA40F32384084698424C
:10C1F800A8BF184607EE100AB8EEC77A052A8CEDD4
:10C20800047A3CF47AAF98ED147A9DED114A25EE44
:10C21800877AA4EE067AB0EE674AA7EE054AB0EE32
:10C22800447AB9F1000F00F0FA83F4EEC46AF1EE33
:10C2380010FA40F3F48308469842A8BF184607EE60
:10C24800100AB8EEC77A062A8CED057A3CF455AF89
:10C2580098ED187A9DED124A25EE877AA4EE067AB3
:10C26800B0EE674AA7EE054AB0EE447AB9F1000F7E
:10C2780000F0CB83F4EEC46AF1EE10FA40F3C58304
:10C2880008469842A8BF184607EE100AB8EEC77AC3
:10C29800072A8CED067A3CF430AF98ED1C7A9DEDB8
:10C2A800134A65EE875AE4EE065AE5EE857AB9F147
:10C2B800000F00F0A283F4EEE67AF1EE10FA40F1F6
:10C2C8009C830A469A42A8BF1A4604EE902AF8EEC2
:10C2D800E44ACCED074AFCF710BF07EE903ADFEDD1
:10C2E800246AB8EEE77A66EEA65A9FED225A9FEDC9
:10C2F800226ADFED227AA5EE856A26EEA55AE5EEDA
:10C30800867AE5EE276A26EE870AFFF76CB9B4F954
:10C318001C819BF80200AAEB080383EAE37EAEEBDC
:10C32800E37E864540F3968103EBD37301205B10CF
:10C33800C4F82C3184F8300184F82401D4F8183179
:10C348004344B3F5FA6FA8BF4FF4FA63B3F57A7FA5
:10C35800B8BF4FF47A7307EE903AB8EEE78A86EDE5
:10C36800038AFCF7DFBD00BFFC3C00200000000092
:10C3780084F9223F92E741B99730083C15A82ABEB4
:10C388001C49002070330020D8ED006ADDED0C4A0E
:10C3980065EEA66AE4EE866AF0EE674AE6EE854A3E
:10C3A800FDEEE46A16EE90EA714500F369819E4558
:10C3B800A8BF9E4606EE90EAF8EEE66A002E00F068
:10C3C8006284DFF8BCC5012ACCED006A3CF495AE66
:10C3D800D8ED046ADDED0D4A65EEA66AE4EE866ADC
:10C3E800F0EE674AE6EE854AFDEEE46A16EE90EA5C
:10C3F800714500F342819E45A8BF9E4606EE90EA2D
:10C40800F8EEE66A002E00F07E84022ACCED016A7E
:10C418003CF473AED8ED086ADDED0E4A65EEA66A07
:10C42800E4EE866AF0EE674AE6EE854AFDEEE46AD7
:10C4380016EE90EA714500F3C4819E45A8BF9E465A
:10C4480006EE90EAF8EEE66A002E00F0E983032A89
:10C45800CCED026A3CF451AED8ED0C6ADDED0F4A22
:10C4680065EEA66AE4EE866AF0EE674AE6EE854A6D
:10C47800FDEEE46A16EE90EA714500F39F819E4551
:10C48800A8BF9E4606EE90EAF8EEE66A002E00F097
:10C49800BD83042ACCED036A3CF42FAED8ED106AB4
:10C4A800DDED104A65EEA66AE4EE866AF0EE674AAC
:10C4B800E6EE854AFDEEE46A16EE90EA714500F371
:10C4C80083819E45A8BF9E4606EE90EAF8EEE66A8E
:10C4D800002E00F0E983052ACCED046A3CF40DAE89
:10C4E800D8ED146ADDED114A65EEA66AE4EE866AB7
:10C4F800F0EE674AE6EE854AFDEEE46A16EE90EA4B
:10C50800714500F358819E45A8BF9E4606EE90EA05
:10C51800F8EEE66A002E00F0A583062ACCED056A3F
:10C528003CF4EBADD8ED186ADDED124A65EEA66A6B
:10C53800E4EE866AF0EE674AE6EE854AFDEEE46AC6
:10C5480016EE90EA714500F3C4809E45A8BF9E464A
:10C5580006EE90EAF8EEE66A002E00F0AF83072AAE
:10C56800CCED066A3CF4C9ADD8ED1C6ADDED134A82
:10C5780065EEA65AE6EE245AE5EE257AFDEEE77A50
:10C5880017EE902A914203DC9A42A8BF1A46114638
:10C5980007EE901AF8EEE77A002E7FF49EA9069B24
:10C5A800002B7FF49AA9059B5B45B8BFF0EE477A4C
:10C5B800FFF793B977EEC76AF0EE477AFEF7AEBC9D
:10C5C800B8F834109FEDDC7A07EE901AF8EEE77AA7
:10C5D800DA4967EE877AC1ED007AFCF7C5BCD84B1B
:10C5E8001E6816F080567FF427A8FFF720B8D54BB1
:10C5F8001B78032B00F06F820023FEF7C8BDF0EE16
:10C60800477AFDF71DBCB0EE677AFDF703BC9FEDD6
:10C61800CE8AFFF7A0B99FEDCC8AFFF773B99FEDDB
:10C62800CB0ADFF8608325EE800A22F021FFD4F8D8
:10C63800D861A8F80600FBF7DCBB94F8240128B100
:10C64800C34884F824310368C4F82831D4F8183171
:10C65800634476E694F82431002B3FF46FAEBC4B6C
:10C6680084F830C11B6884F824C1C4F8283165E611
:10C67800B849B94A8C46FEF735BA06EE901ABFE6B5
:10C6880006EE901A98E696ED000A06930891059230
:10C6980022F0EEFEDFF8F0E2DFF8F0C2DEF8ECE0C0
:10C6A800DFF8E082059AA8F800008CFB0E3C4FEA00
:10C6B800EE7ECEEBAC1E07EE90EAF8EEE77A069B2C
:10C6C8000899FDEEE77A17EE900AA8F80200FCF741
:10C6D800A8BC06EE901A3DE707EE906AF8EEE78AE6
:10C6E800DFED9E7A9FEDAB0A84F8B46168EEA78A05
:10C6F80038EE800AFDEEC07A17EE903A2033402BD0
:10C7080040F2CC819FED900A8C4BFDEEE87A83EDE8
:10C71800010A17EE903A2033402B00F2BC81DFED7E
:10C728009E7AF4EEE78AF1EE10FA40F36C82DFEDC0
:10C738008C6ADFED8C7A01E0F0EE478AF4EEE78A46
:10C74800F1EE10FA38EEE67AF6DCDFED957AB4EE23
:10C75800E77AF1EE10FA40F153829FED816ADFED3E
:10C76800826A01E0B0EE677AB4EEE67AF1EE10FA8A
:10C7780077EE067AF6D49FED877AF4EEC77AF1EE73
:10C7880010FA40F392819FED847A77EE677A27EE6C
:10C79800A76ADFED765ADFED766A9FED767AE6EEE8
:10C7A800256A67EE865AA6EE267AE5EE877AC4ED04
:10C7B8006E7AFDF7DEBD06EE901AA9E606EE901A2F
:10C7C80062E606EE901A3DE606EE901A7EE6B0EEB8
:10C7D800667AFEF72BBDF0EE476AFEF73DBDFAF725
:10C7E80071FF654BDFF89C811F78069B99F8002044
:10C7F800D4F8D861C01AA8F80400FEF764BBFDEEAF
:10C80800C74A0DF1300E9A46DFF884C1DFF870810F
:10C8180014EE901A0EEB82024B4606E09645E8ECC1
:10C82800014A0CF1100C3CF468ACDCED004ABEEC9B
:10C83800014A65EEA44AE6EE044AB0EE674AA5EE60
:10C84800244AF0EE444A33B1F4EE446AF1EE10FAA9
:10C85800C8BFF0EE474AFDEEE44A14EE909A494507
:10C8680004EE901A04DCD145A8BFD14604EE909A94
:10C87800F8EEE44A002ED1D106980028CED10598CA
:10C888005845B8BFF0EE474AC8E7FAF71BFF3A4BDE
:10C89800DFF8F0801F78069BC01AA8F80200FEF7A0
:10C8A8004FB9364B1B6803F59C530833C4F8C031A5
:10C8B8003B78012B7DF4F4A894F8BC31002B7DF46F
:10C8C800EFA8032A00F0D88122F020FA012384F887
:10C8D800BC31FDF7E5B8FAF7F5FE069BDFF8A48052
:10C8E800D4F8DC91D4F8D861C01AA8F80200FEF791
:10C8F80089B9DFED297AF4EEE76AF1EE10FA40F330
:10C90800D081DFED175A9FED176A01E0F0EE676AF4
:10C91800F4EEC66AF1EE10FA76EEE57AF6DCDFEDB3
:10C92800206AF4EEE67AF1EE10FA40F1B781DFED15
:10C938000C5A9FED0D6A37E06F12833A0000002011
:10C94800C0760020BC760020000000000000C8422D
:10C95800B07600207C3E00201423002035FA8E3C5F
:10C96800DB0FC940E4CB1641E4CB16C192E741B9CD
:10C978009730083C15A82ABE384E0020485500209C
:10C98800703300203C4E0020981C0020D34D6210CC
:10C998001C490020DB0FC93FDB0F4940DB0FC9BF33
:10C9A800DB0F49C0F0EE667AF4EEC67AF1EE10FAC3
:10C9B80077EEA56AF6D45FED097AF4EEE76AF1EE50
:10C9C80010FA04DD5FED0C7A77EEE66A8BE45FED32
:10C9D8000D7AF4EEE76AF1EE10FA44BF5FED107AD3
:10C9E80077EEE66A7FE4099807F0E2FAFEF764BD9D
:10C9F800CA4800F1800CFEF74DBAFDEEE77A17EE53
:10CA0800902A8A42FFF663AC5CE4BDEEC77A17EE63
:10CA1800100A8842BFF635AC07EE101A36E4BDEEB0
:10CA2800C77A17EE100A8842BFF606AC07EE101A4E
:10CA380007E4BDEEC77A17EE100A8842BFF6D7ABF7
:10CA480007EE101AFFF7D8BBBDEEC77A17EE100A2B
:10CA58008842BFF6A7AB07EE101AFFF7A8BBBDEEDA
:10CA6800C77A17EE100A8842BFF677AB07EE101A9E
:10CA7800FFF778BBBDEEC77A17EE100A8842BFF6FB
:10CA880047AB07EE101AFFF748BBA8F80600A5F851
:10CA9800B460FCF7A7B8DFEDA27A88E6F8F734FAB5
:10CAA80032E607EE101AFFF711BB9FED9E7AF4EEFF
:10CAB800C77AF1EE10FA44BF9FED9B7A77EE677A5A
:10CAC80065E6F8F73DFB00283EF4A9ACFEF71FBD6C
:10CAD8006146FFF7B6BA1BF0B3F9FCF77BB88020C4
:10CAE80016F064FB08B105F0BBFD22F00FF9FEF764
:10CAF80090BC94F80C32002B7BF4E4ABFBF7CFBB73
:10CB0800DFED8A7AF4EEE7DAF1EE10FA63DCDFEDB6
:10CB1800887AF4EEE7DAF1EE10FA5CD4854BD3EDBF
:10CB2800007AB1EE677AB4EEC7DAF1EE10FA00F1E6
:10CB38008180B4EEE7DAF1EE10FA88BFB0EE67DA7A
:10CB48007D4BC7ED00BA1B689342BBF6F3AAFCF70E
:10CB580008BD7A4A7A4B10681B689847089BDBED3A
:10CB6800007A93ED007A774BD7ED006A83ED020ADD
:10CB7800754B67EE277A2B4427EE8C7AD3ED007A33
:10CB8800724B67EE277AF0EE665AE7EE8D5A93ED10
:10CB9800006AB1EE467AF4EEC75AF1EE10FA08D4FC
:10CBA800B4EEE56AF1EE10FA8CBFB0EE657AB0EE3D
:10CBB800467A674B1B78012B02D0192B7BF4F9AA14
:10CBC800DFED647AB4EEE7DAF1EE10FACCBF0123B8
:10CBD8000023FBF7F9BA9FED52DAB1E7DFF8888155
:10CBE800D8F8000005F014FD5B4B1B780022022BDF
:10CBF800C8F800207EF4C1AB04F060FFFEF7BDBBAF
:10CC0800F0EE477AB7E5B0EE687A9EE50698002818
:10CC18007FF43FAC05985845B8BFF0EE476A38E452
:10CC2800069800287FF413AC05985845B8BFF0EE75
:10CC3800476A0CE4B0EE47DA82E71BF80330002BB2
:10CC48007EF4EDABFEF71BBC45200FF011FEFF2074
:10CC58000FF00EFE41480FF07DFD40460FF008FE34
:10CC6800FEF767BB069800287FF457AC059858452F
:10CC7800B8BFF0EE476A50E4802016F097FA002813
:10CC88007CF40EAF20E6069800287FF49AAB05984E
:10CC98005845B8BFF0EE476AFFF793BBF0EE676AF6
:10CCA80089E6F0EE667A3AE6069800287FF413AC37
:10CCB80005985845B8BFF0EE476A0CE40698002876
:10CCC8007FF44DAC05985845B8BFF0EE476A46E486
:10CCD800132B05D1B0EE480A22F0CAFBAAF80000CF
:10CCE800B0EE480AD5F814321D4898471D4B1B78FA
:10CCF800132BB0EE408A7BF4BDA822F0B9FBAAF84A
:10CD08000200FBF7B7B8069800287FF47EAB0598B9
:10CD18005845B8BFF0EE476AFFF777BB14230020E9
:10CD280000000000DB0FC9BFDB0F49C000C0F8449A
:10CD380000C0F8C4E8480020CC48002094390020FE
:10CD4800A83900201033002084480020EC48002037
:10CD58007C37002000009642503500200448030824
:10CD680018660020384E0020504500202DE9F04F6D
:10CD78002DED028B93B083461EF068FFB94B1D78EA
:10CD880025B113B0BDEC028BBDE8F08FB64B1B6824
:10CD98005B05F6D5B54FB64E3B68002B5CD0B54C5D
:10CDA8003168D4F810218A1A7C2A55D994F81421AC
:10CDB800DFF810839FEDB08AC4F81011013284F8AF
:10CDC80014214FF0240A5E20984750463B68984744
:10CDD800AA4BF8EC016A9B8A07EE103AF8EEE66A6D
:10CDE800B8EEC77A0AF1010AC6EE877A5FFA8AFABC
:10CDF80067EE887AFDEEE77ACDED027ABDF9089004
:10CE08005FFA89F01EF094FEC9F307201EF090FE29
:10CE1800BAF1270F3B68D6D15E2098473B6830208F
:10CE28009847974BD3F800805FFA88F01EF080FE91
:10CE3800C8F307201EF07CFE3B685E20984794F8F4
:10CE4800143113F0030800F0898113F0070801F08A
:10CE58007782282B01F04A838A4B1B78002B72D0EB
:10CE6800844C894AD4F81831ABEB0303934200F29F
:10CE7800898794F82091B9F1000F35D1DFF84882FD
:10CE8800D8F80000F6F774FAC0B201280FD90228C2
:10CE98007E4F41F0C4833B78002B41F01086D4F8D4
:10CEA8002431ABEB0303B3F57A6F81F0B787D4F87D
:10CEB8002831002B47D094F82031C3B9744B1B6834
:10CEC8009B7801211E3B00228B4284F8201184F8B4
:10CED800342141F26687D8F80000022104301EF0A0
:10CEE800A5FD94F82C3111E0D4F828315BB3D4F8BF
:10CEF800303140F6B732ABEB0303934223D994F8B1
:10CF08002C31002B01F0DB82DFF8BC81013BDBB266
:10CF180084F82C31002B00F0A987D4F8287194F8F4
:10CF2800342117F8011B94F83531D8F80000C4F8FB
:10CF380028710A44013384F8342184F83531F6F72E
:10CF48001AFAC4F830B1534BD6F800801B7843B1B5
:10CF5800514F386828B1514B1B78013B012B40F2E7
:10CF680095874F4B1B7863B14E4F3B684BB1414C93
:10CF7800D6F80090D4F84C31A9EB0303632B00F2E8
:10CF88002081DFF8488198F80030022B01F0768282
:10CF98003E4F97F87430032B00F05287424B1B78B2
:10CFA80073B1424D2B685BB1324CFAF78BFBD4F866
:10CFB8005831029044F61F62C31A934200F25C8112
:10CFC8003B4B1B78002B40F083803A4B1B7843B1D6
:10CFD800284CD4F8A83203F5C333A0339B4580F01E
:10CFE8007F86354B1B78002B3FF4CBAE214E334C5C
:10CFF800334D06F2C9272068F6F7BAF900283FF43E
:10D00800C0AE2068F6F7AEF92B7880465A1E33B1C9
:10D0180020682A70F6F7ACF90028F2D1B1E60322AD
:10D028003946781E24F017FB96F8C83296F8C922BC
:10D0380086F8CB8283F47F4383F0FF039B1A1FFAA1
:10D0480088F89BB2B8EB132FD5D196F8CA22DBB279
:10D058009A42D0D1781E13F083FA2B78184428709E
:10D06800C9E700BF6A53002094660020C8740020F6
:10D07800485500205825002000007A449453002089
:10D088004C4200205A7500203F0D03000800002084
:10D09800C47400205C750020BC74002064750020F6
:10D0A8006C750020F85D00207475002078750020EC
:10D0B800B8750020C97500207E7500208475002091
:10D0C80088750020CC530020C0740020CA69002055
:10D0D8005B4C2278A2B15B4B9B7A53B1FAF7F2FA18
:10D0E800594B1B68C31AA3F57A73B3F5FA6F07D8BF
:10D0F8002278564B56491868F6F70EF90023237024
:10D10800544CD4F8A03203F5C333A0339B45FFF445
:10D118005CAF514DC4F8A0B22B78002B41F0498385
:10D128004E4D2B78002B41F031824D4994F8A422C2
:10D138008D5CE90701F10685AA0701F1C6846B0732
:10D1480001F1B283474A94F8A4321178013393FB72
:10D15800F1F201FB123384F8A43236E7D4F8102137
:10D1680041F288339A4201F226823B685E20984752
:10D178003B68142098473C4B3C4AB3F9043082FB87
:10D1880003124FEAE378C8EBA2080FFA88F85FFAAF
:10D1980088F01EF0CDFCC8F307201EF0C9FC3B68E0
:10D1A8005E2098473B681C20984700201EF0C0FC72
:10D1B80000201EF0BDFC3B685E20984794F81431AF
:10D1C80043E6DFF8A4A0DFF8A480412013F010FCA8
:10D1D800BAF9023088FB0320DB17C3EBA00080B24A
:10D1E80013F0ECFBBAF9003088FB0320DB17C3EB24
:10D1F800A00080B213F0E2FBBAF9043088FB0320E8
:10D20800DB17C3EBA00080B213F0D8FB184B3868CB
:10D218001978F6F7B0F894F8503113F0010801F0D6
:10D228001F82144AC4F84C910133DBB2A2FB0312EB
:10D23800D20802EB8202A3EB420384F85031A0E645
:10D248004C750020206800203C400020BC75002060
:10D258000C75002058250020C0750020C1750020DD
:10D26800C4750020C87500201C42002067666666E9
:10D27800F05F0020CDCCCCCC94F85E31002B41F08F
:10D288008081DB4B1A6802F00803002B48F6034143
:10D298004AF60B404BF60F4349F6074704BF0346CF
:10D2A8000F4612F0040F4FF0190118BF1F469206DF
:10D2B80084F85E1103D547F4804747F02007CD4B2B
:10D2C8005A79C7F30909002A41F0D5859B79002BC3
:10D2D80041F0D786984664204FF0FF3A4FF0000C93
:10D2E8000A970B97ADF834C0CDF83AC0CDF83EC0D8
:10D2F800CDF842C0CDF83090ADF83680ADF838A002
:10D308008DF846000AAF0FCFDFF800E384F805C0B8
:10D31800AEE80F0097E80F00AEE807002EF8023BD2
:10D3280071464FF0010C1B0CFE271F20C82201F884
:10D338001E39A770A27184F807C0E07094F86E01D6
:10D34800207180F0F10383EA0313DAB2130983F042
:10D35800E70343EA022383EAC2031BB283EA031208
:10D36800D2B2C3F3072383EA121343EA022383EA00
:10D37800C2031BB283F0C80282EA0212D2B2C3F31C
:10D38800072383EA121343EA022383EAC2031BB288
:10D3980083EA0C0787EA0717FFB2C3F3072282EA7A
:10D3A800171242EA072200EB0C0382EAC7070EEBCA
:10D3B8000C0084F86E31278011F8013B7B4083EA2A
:10D3C8000313DBB21A0982EA172242EA032282EA2D
:10D3D800C3031BB29FB281422780EDD183F07C0347
:10D3E80083EA0313DBB24FEA131E8EEA172E8EEA86
:10D3F800032E8EEAC30E0FFA8EFE1FFA8EFADFF89E
:10D4080010C2A4F800A05FFA8EFE4FEA1A2A84F828
:10D4180028A084F827E00CF5CB7804F12209DCF881
:10D428000000DCF80410DCF80820DCF80C30474673
:10D438000FC70CF1100CCC45B846F0D1DCF8000051
:10D4480038606D4F9CF8043088F8043007F12708DD
:10D4580084F8BDE184F8BEA117F8011F2868F5F724
:10D468008AFFB845F8D194F85F31002B41F08480E9
:10D478006249326809780A2084F85F01002901F0BE
:10D4880009825F4F01293888069041F20F860229E8
:10D49800B7F802E001F00A85B8880590032901F081
:10D4A800FE85F8880490042901F015860529388935
:10D4B80001F00C860629B7F80A9001F003860729BF
:10D4C800B7F80C8001F0FB85FB89039394F86E1183
:10D4D8000A920B4683F0300282EA0212D2B217098E
:10D4E8004849079387F07A0747EA02270988237192
:10D4F80087EAC202444FC1EB012187FB013A069B30
:10D508004FF0000C63F30F0C059B6EF31F4C4FF0AC
:10D51800000E63F30F0E049BCDF82CC012B28A44A0
:10D528000027C91763F31F4EC1EB6A2A039BCDF886
:10D5380030E082EA021160F30F070020C9B268F3F5
:10D548000F00C2F3072269F31F4782EA111263F33F
:10D558001F404FF000090D978DF83DA00E908DF8F3
:10D568003C9042EA01220DF1280C82EAC107BCE88E
:10D578000F003FB287F0C80888EA0818DFF88CE087
:10D5880084F805905FFA88F8C7F30727AEE80F001C
:10D5980087EA181747EA08239CE8030083EAC803C8
:10D5A8001BB283F023024EF8040B82EA0212D2B2B5
:10D5B800C3F30723079F83EA1213704643EA022343
:10D5C80083EAC20207F1010C20F814194FF023086E
:10D5D8001621FE27C82384F86EC1228084F80780AC
:10D5E8000EF1020EA770E170A371114612E000BFA0
:10D5F800C876002094760020EF26002030540020C2
:10D60800485F0020AA7600200308208060250020BB
:10D618005A25002010F8013B4B4083EA0313DBB284
:10D628001A0982EA112242EA032282EAC3031BB2E0
:10D6380099B270452180EDD183F0F40383EA031396
:10D64800DBB24FEA131E8EEA112E8EEA032E8EEA03
:10D65800C30E0FFA8EFE1FFA8EF8E44FA4F800806E
:10D668004FEA182C5FFA8EFE84F81EE084F81FC07B
:10D678007968BA683868FB6807F5CB78A8E80F00BE
:10D6880038697969BA6904F29717A8E8070004F2BB
:10D69800B51884F8B5C184F8B4E117F8011F2868F3
:10D6A800F5F769FEB845F8D194F866C1BCF1000FEA
:10D6B80040F05C87CE4B94F86E71B3F90010B3F963
:10D6C8000220B3F904309FEDCB6ADFF844E384F815
:10D6D80005C007EE103A33680A9387F06A0383EAB5
:10D6E800031306EE901AD9B20B0983F0D50343EA67
:10D6F800012383EAC1031BB283EA03115242C9B270
:10D7080007EE902AC3F3072383EA111343EA0123A0
:10D71800F8EEE77AF8EEE66AB8EEC77A83EAC1036C
:10D728001BB267EE867A66EE866A27EE067A0020D6
:10D7380083F0C808CDED0C7ACDED0B6A8DED0D7A2E
:10D748000E900F90109088EA08160DF12809F6B28D
:10D75800C3F30728B9E80F0088EA161848EA06282C
:10D7680088EAC6080FFA88F8AEE80F0088F01E06A7
:10D7780099E8070086EA0616F6B2C8F3072383EA93
:10D78800161343EA06238EE8070083EAC6061C2020
:10D79800C8214FF005084FF01E0CFE237A1CE070DC
:10D7A800A17184F8668184F807C0A370AEF11001F6
:10D7B80027710EF10C00268084F86E2111F8013BC8
:10D7C800734083EA0313DBB21A0982EA162242EA9B
:10D7D800032282EAC3031BB29EB281422680EDD1A6
:10D7E80083F0270383EA0313DBB24FEA131E8EEAA2
:10D7F800162E8EEA032E8EEAC30E0FFA8EFE1FFA3D
:10D808008EFC7A4FA4F800C05FFA8EFE4FEA1C2CFB
:10D8180084F825C084F824E007F5CB7804F12209C0
:10D8280038687968BA68FB6846460FC610374F45AE
:10D83800B046F5D1704E3B88A8F8003006F12407B1
:10D8480084F8BAE184F8BBC116F8011F2868F5F717
:10D8580092FDB742F8D194F867A1BAF1000F40F0F1
:10D868007F86664B1B68052213F0140F84F8672126
:10D8780040F08987DFED627A94F86EC15C4B614AAB
:10D88800B3F90410B2F906205F4E6048CDED0C7A6A
:10D898008CF0220383EA0313DFB23B0983F05903B8
:10D8A80043EA072383EAC703B2F5FA6F1BB2A8BF9E
:10D8B8004FF4FA6283EA0317FFB2B2F57A7FC3F333
:10D8C800072383EA1713B8BF4FF47A724FF0640E38
:10D8D80043EA0723A2F57A720EFB02F283EAC70332
:10D8E80086FB02E680FB01E01FB2D217C9174FF092
:10D8F8000008C2EBA612C1EBA00187F0C806ADF87C
:10D908003A20ADF83810CDF82880CDF82C80CDF825
:10D9180034800DF1280E86EA0616BEE80F00F6B22E
:10D92800C7F3072787EA161747EA062787EAC606CE
:10D93800374FDEF800E084F804C00FC736B286F02F
:10D948004A0383EA0313DBB2C6F3072181EA131102
:10D958003A4641EA03210CF1010C81EAC303142081
:10D9680042F810E9FE264FF04A0E002184F86EC1F5
:10D978004FF0C80CE0702380043784F807E0A670E5
:10D98800617184F806C0184612F8011B414081EA0B
:10D998000111C9B20B0983EA102343EA012383EA80
:10D9A800C10109B288B2BA422080EDD181F01401D8
:10D9B80081EA0111C9B24FEA111E8EEA102E8EEAD1
:10D9C800012E8EEAC10E0FFA8EFE1FFA8EF6074F51
:10D9D80026804FEA16295FFA8EFE84F81D9084F897
:10D9E8001CE079683868BA68FB6813E05A2500209B
:10D9F8001C42002088C3E43AEF260020C8760020A5
:10DA080000000000485F0020D34D6210676666661C
:10DA180060250020B7F8188007F5CB7CACE80F002C
:10DA280038697969ACE8030004F29716ACF800800D
:10DA380084F8B391B04684F8B2E104F2B31918F847
:10DA4800011F2868F5F797FCC145F8D1C44BC54AB2
:10DA58001B781278013B12F00100DBB214BFC02121
:10DA68004021172B03D8C04A134493F830A0BF4B6A
:10DA78001A8893071ABF002341F01001012312F4FA
:10DA8800027F18BF022312F0100F18BF062312F0EE
:10DA9800200F18BF1023002841F0B2814FF0030C6B
:10DAA80094F86E910A9389F0460383EA0313DAB275
:10DAB800130983F0920343EA022383EAC2031BB2E9
:10DAC80083EA0310C0B2C3F3072282EA101242EAC3
:10DAD800002282EAC00212B282F0C80E8EEA0E1E3E
:10DAE8005FFA8EFEC2F30722002382EA1E12032089
:10DAF8008DF82CA08DF82FC08DF82D3042EA0E2C11
:10DB08008DF82E108DF830000AAA07CA8CEACE0EBE
:10DB18000FFA8EFEDFF868A2E3718EEA0E1CAAE8FF
:10DB280003005FFA8CFCCEF3072E8EEA1C1E4EEA29
:10DB38000C2181EACC0C94F808E08AF800200FFA4E
:10DB48008CFC8EEA0C0E8EEA0E1E5FFA8EFECCF36B
:10DB5800072282EA1E1242EA0E22607AA17A94F81B
:10DB68000BC0637182EACE0212B2504080EA001EF6
:10DB78005FFA8EFEC2F3072080EA1E1040EA0E20EC
:10DB880080EACE0000B2414081EA0111C9B2C0F377
:10DB9800072282EA111242EA012282EAC10212B283
:10DBA8008CEA020C8CEA0C1C5FFA8CFCC2F307228C
:10DBB80082EA1C1242EA0C2294F80CE0607BA17BFA
:10DBC80094F8108084F8049082EACC0212B28EEAAB
:10DBD800020E8EEA0E1E5FFA8EFEC2F3072282EA5A
:10DBE8001E1242EA0E2282EACE0212B2504080EAA7
:10DBF8000010C0B2C2F3072282EA101242EA0022E1
:10DC080082EAC00212B2514081EA0111C9B2C2F3DC
:10DC1800072282EA111242EA012282EAC102E17B6A
:10DC280013B281EA030282EA0212D2B2C3F30723D3
:10DC380083EA121343EA022383EAC2031BB288EA87
:10DC4800030282EA0212D2B2C3F3072383EA121351
:10DC580043EA022383EAC2031BB283F0320282EA58
:10DC68000212D2B2C3F3072383EA121343EA022350
:10DC780083EAC2031BB29AB24FF0FE0C4FF0090EB2
:10DC8800C82009F10101DBB284F802C084F803E07E
:10DC98004FEA122CA07184F86E11228084F812C009
:10DCA800637438687968BA68B7F80C900AF5C47E66
:10DCB800AEE807000AF5CC7A8EF80280AEF800903C
:10DCC80084F8A8C184F8A73116F8011F2868F5F769
:10DCD80052FBB245F8D1029BC4F85831FFF770B92E
:10DCE80094F8AC32204AC4F8A8B202EB8302926CD2
:10DCF80042B312AD04F2B3231D4E45F8203D002176
:10DD080004F2C52331800B9380211523A52784F8BD
:10DD1800B232284684F8B11284F8B0729047284687
:10DD28003188F6F7E4FF0A9D124804F52C716D1A44
:10DD3800152DA8BF15252A4621F092F90E4A94F808
:10DD4800AC3215700D4A013382FB0312A2EBE37269
:10DD580002EB42029B1A84F8AC32FFF742B900BFCB
:10DD68007035002068740020981F03080C420020BA
:10DD7800A8740020483B00205D3B002056555555AF
:10DD880060250020D24AD34B92F80BE03068D4F8D3
:10DD98001C211B88D049801A4FF47A72DFB202FB2B
:10DDA8000EF21B0A8F770F7590424FF00007CB7762
:10DDB8004B758F700F7180F0F083C84BDFF840E32C
:10DDC8001B68C74AC748176800689268C4F818B142
:10DDD8008EFB038CDB17C3EB6C13DFF828C38EFBB9
:10DDE800008E8CFB07988CFB029CD217C2EBAC020E
:10DDF80003F5FA734FEAE07C9BB2CCEB6E1CFF177D
:10DE080000F5EA4EC7EBA8070EF1300E8B761B0A19
:10DE18000CF1780C4FEA2E2E3030CB764FEA2728BB
:10DE280013120F7781F81D8081F8202081F82130A6
:10DE380081F824C081F823E081F82200FFF719B89F
:10DE4800DFF8C492D9F80000F5F789FA00283FF402
:10DE5800A5A8D9F800000121F5F77EFA02220023CF
:10DE680087F8742088F80030FFF798B894F83411D0
:10DE780094F83531D8F800004A1C013384F834216D
:10DE880084F83531F5F777FAFFF75BB8964CDFF889
:10DE98007C924FF0000A0AE01B2B00F005830D2B43
:10DEA80000F018824FF0010389F801303868F5F75F
:10DEB8005FFA002838D03868F5F754FA83B27E2B19
:10DEC80032682AD099F801100029EFD194F8362148
:10DED800002AE1D07D2B00F0128294F844E1BEF1D3
:10DEE800000F04D080F02003DBB284F84411511CE9
:10DEF800C9B22244092984F8361182F8383100F071
:10DF0800F2810829D2D8B4F84221134403EB132331
:10DF180003F0FF03A4F84231C8E784F836A184F877
:10DF280037A189F801A0C1E794F8453133B194F8D5
:10DF3800393184F84501302B00F05A8794F837219D
:10DF48006A4BDFF8CCC1DFF8CCE1DFF8CCA10127C0
:10DF5800104600283FF405A83268A2EB0802012AFF
:10DF680000F2B38194F84691B9F1000F40F0B38202
:10DF780094F8471133F8112012B984F84771E8E78B
:10DF88000131B2F5826F84F8471100F021811FD961
:10DF9800B2F5E26F00F0C28035D9B2F5046F00F037
:10DFA800CC80B2F5116F00F0D580B2F5E46FD0D116
:10DFB80010464F4A176C918A642303FB07F393FBBF
:10DFC800F1F112F04BFD002384F83731FEF7C9BF99
:10DFD800B2F5007F00F0D8802DD8B2F5807F00F030
:10DFE8004A81B2F5887FB4D1DCF800205207B0D559
:10DFF8003C4B4FF48870196812F030FD002384F808
:10E008003731FEF7AEBFB2F5C06F00F0D180B2F580
:10E01800E06F9ED1364A906B918A642303FB00F32C
:10E028004FF4E06093FBF1F112F018FD002384F83F
:10E038003731FEF796BFB2F5047F00F02C81B2F5B8
:10E04800806F86D194F848310133DBB2032B00F29C
:10E058005D8142F2107184F8483101FB03F1254BD0
:10E068001B88002B40F050810131234B1B78DF07C0
:10E07800224B1B8848BF0431D80748BF0A319A078A
:10E0880048BF14311F0648BF2831D80548BF28317A
:10E098005A0748BF64311F0748BFC831980548BFB1
:10E0A80001F5C8719A0648BF01F57A71DF0648BFC5
:10E0B80001F5FA61580648BF01F57A614FF48060AE
:10E0C80012F0CCFC002384F83731FEF74ABF00BFBA
:10E0D800084F0020004F00208C750020B0760020EB
:10E0E800AC7400204C42002058250020981F0308DB
:10E0F80094530020CC760020687400200C42002045
:10E108001F85EB5167666666506A0020080000208C
:10E11800C876002094760020164F002010467E4ACC
:10E12800D76B918A642303FB07F393FBF1F112F099
:10E1380095FC84F83791FEF714BF784BB3F90410B7
:10E1480001EB81011046490012F088FC84F83791F0
:10E15800FEF707BF9EF80520002A3FF4FAAE9AF8AA
:10E16800001000293FF4F5AE6D4B1B8803EB8303C9
:10E178005B004FF4116093FBF1F112F06FFC002388
:10E1880084F83731FEF7EDBE9EF8061000293FF4FB
:10E19800E0AE644B64491B68104681FB0321DB1722
:10E1A800C3EBA10112F05AFC84F83791FEF7D9BEEF
:10E1B8009EF80620002A3FF4CCAE5A4B4FF4C060BC
:10E1C800996812F04BFC002384F83731FEF7C9BE7A
:10E1D800DCF8002012F020097FF4BBAE534A116826
:10E1E800090600F1EF85524A127B002A3FF4B1AECE
:10E1F80094F84911032900F26886DFE801F0322813
:10E2080019024C4B1B6859799A79DB7901F14071F5
:10E2180001EB022101EB0341002384F849314FF45B
:10E22800826012F01BFC002384F83731FEF799BE98
:10E23800414B1A68137A507992781B0403EB002338
:10E2480013444A1C84F8492103EB0161E7E73A4B80
:10E258001A68D379107952781B0403EB002313440E
:10E26800EFE7354B1A689379D07812781B0403EBE3
:10E2780000231344E5E7DCF8002051077FF569AE79
:10E288002E4B4FF48070196812F0E8FB002384F8D5
:10E298003731FEF766BE9EF80520002A3FF459AED6
:10E2A8009AF8001000293FF454AE214B5B7B002BF9
:10E2B80000F0B0851A4B1B8893FBF1F101EB81014B
:10E2C80049004FF4047012F0C9FB002384F8373179
:10E2D800FEF747BE4FF0010184F8361184F8383153
:10E2E800A4F84221E2E5B4F84221C2F1FF029342C8
:10E2F8007FF4D8AD4FF0010384F84531D2E54FF0F3
:10E30800010384F84431D1E50231AEE6012384F8F3
:10E31800483142F21071A2E6945300201C420020BA
:10E32800004F0020AC740020676666669466002083
:10E33800084F00204C7700203C420020B076002097
:10E348003B685E2098473B6802209847FF2012F000
:10E358008DF80378FF2B00F0328590F901304FEAF1
:10E36800E3785FFA88F8D8B21DF0E2FB40461DF06A
:10E37800DFFB3B685E2098473B6803209847FF20F7
:10E3880012F074F80378FF2B00F01485B0F9083008
:10E39800D8B2C3F30729DFF8B8821DF0C9FB484695
:10E3A8001DF0C6FB98F80530002B40F0D7820AA96B
:10E3B8009E481DF083FB3B685E2098473B6813200E
:10E3C8009847BDF928805FFA88F01DF0B1FBC8F3C3
:10E3D80007201DF0ADFB3B685E2098473B681B207B
:10E3E8009847BDF92A805FFA88F01DF0A1FBC8F3B1
:10E3F80007201DF09DFB3B685E2098473B68232063
:10E4080098474E201DF094FB00201DF091FB0AA9AF
:10E4180086481DF053FB3B685E2098473B681220F6
:10E428009847BDF928805FFA88F01DF081FBC8F392
:10E4380007201DF07DFB3B685E2098473B681A204B
:10E448009847BDF92A805FFA88F01DF071FBC8F380
:10E4580007201DF06DFB3B685E2098473B68222033
:10E46800984745201DF064FB00201DF061FB3B68C8
:10E478005E20984794F81431FEF7EBBCF9F722F9BF
:10E488006B4B1B68C01A40F6B833984200F286817D
:10E49800DFF8C0A19AF804303A2B00F0B1830023CA
:10E4A80088F80030FEF77ABD3868F4F761FF002875
:10E4B8007FF4F8AC4FF0010384F83731F6E4C4F880
:10E4C800283184F82031DFF890811DF0DFFA94F8C4
:10E4D8002C31FEF71BBD5749062012F0CBF800235C
:10E4E80084F8460184F83731FEF73BBD4FF0000849
:10E4F8003B68D6F8009084F814815E2098473B6802
:10E508004D4C1720984740461DF012FB4B4BA3FB80
:10E5180009239B0BA4FB03125209C2EB0212A3EBC3
:10E528008203D8B21DF004FB3B685E2098473B6825
:10E5380018209847424BA3FB09239B09A4FB03120D
:10E548005209C2EB0212A3EB8203D8B21DF0F0FA13
:10E5580040461DF0EDFA3B685E209847FEF77CBC0C
:10E568000AF1FF3A84F867A1FFF7B5BB0CF1FF3C4D
:10E5780084F866C1FFF76FB9013B84F85F31FFF794
:10E5880093B8013B84F85E31FEF76DBF2D493A2000
:10E5980012F070F82870FEF718BD2B4B32681B7804
:10E5A800C4F81C21013B012B3FF607AC10220223C3
:10E5B8008A700B7101E43B68DFF8A0905E209847F1
:10E5C8003B6810209847214AD9F8003082FB032A7B
:10E5D800DB17C3EB6A1A5FFA8AF01DF0A9FACAF3CF
:10E5E80007201DF0A5FA3B685E2098473B6821206C
:10E5F8009847D9F80030154AD81782FB0329C0EB91
:10E608006910642202FB10300028B8BF4042C0B233
:10E618001DF08EFA40461DF08BFAFEF7A6BD1DF0E0
:10E6280027FA01233B70FEF742BC00BF8096980092
:10E63800D06900205F0A02088988888873B2E74594
:10E64800D34D6210D5BB0208BC7600201F85EB5164
:10E6580094760020B8690020C0740020B0760020AD
:10E66800AA4B1B88DA0515D4D80600F11B84990635
:10E6780000F127845A0600F13384180700F13D841D
:10E68800D90700F1FA8413F0020F0CBF4FF0040809
:10E698004FF00C089E4B9F4A1B78D27803F0010379
:10E6A8000AB143F002035320029312F0A1F99A4AE7
:10E6B800128802EB820202EB8202900080B212F012
:10E6C8007DF9002012F07AF9944A95491288386841
:10E6D800C2EBC212520081FB023111444FEAE27AC6
:10E6E800CAEB612A5FFA8AFA5146F4F744FE8D4B69
:10E6F80038681A78029B48EA03088A4B8AEA020AB1
:10E70800002183F800A0F4F736FE41463868F4F794
:10E7180032FE844B834A1B78386888EA0303DBB2ED
:10E7280019461370F4F727FE94F85031002B7EF445
:10E7380078AD4F2012F05CF914F002FF14F000FFDE
:10E7480014F0FEFE01213868F4F715FE764A754B81
:10E7580092F800801B78734A386808F0010883F043
:10E76800010341461370F4F706FE6E4B6D4A1B78A1
:10E77800386888EA030319461370F4F7FCFD94F827
:10E788005031FEF74EBD694B9FED697AD3ED007AA3
:10E79800F8EEE77A67EE877AFFF76EB8654AB2F85F
:10E7A800523100210133A2F8523188F80010FEF7E7
:10E7B800F5BB614E614B00930024A6F13F01604B0D
:10E7C800604A089106F8404C5F4909960AA8F6F78E
:10E7D80065FB089E731C08933470089B2922591CFA
:10E7E80008911A70089BEA22591C08911A70089B14
:10E7F800C822591C08910AA81A701FF0ADFB471CC3
:10E808000AA93A46089820F02BFC089AD319013334
:10E818000893D455089B5A1C08921C70089B5A1CD4
:10E8280008921C70089B5A1C08921C70089B5A1C62
:10E8380008921C70089B5A1C08921C70089B5A1C52
:10E8480008921C70089B5A1C08921C70089B5A1C42
:10E8580008921C70089B5A1C08921C70089B5A1C32
:10E8680008921C70089B5A1C08921C70089BFF2277
:10E87800591C08911A70089B0122991812A808912E
:10E888001A7050F8283D9B1B33701DF06FF92C70DF
:10E89800FEF79BBB884689460846049105918E463B
:10E8A80006910391FEF712BE284A234B12680B9378
:10E8B800A3F1400500202121D70003F8400CA970DE
:10E8C80040F1CD8222490326104B1B88580500F1E0
:10E8D800C382DA0700F1F28203F002031D4A002B1B
:10E8E8001CBF032611461C4F3246384620F0B8FBA1
:10E8F800F31912A80133B91E40F8203D00225B1A13
:10E90800F2556B701DF032F9FEF71CBC0C4200206A
:10E9180068740020E0530020004F0020AA760020F1
:10E9280003082080F05F002090760020B076002059
:10E938000AD7233C582500200C75002045420020AA
:10E9480008490308104903081C490308C076002039
:10E95800F448030804490308CF7400209E4B93F839
:10E9680000A0BAF1000F3FF422AD9C4AB4F816E1BA
:10E9780011883B6802924FEA0E1E64201FFA8EFE31
:10E9880000FB01A14FEA4A00B1FBF0F14EEA012E6B
:10E998001FFA8EFEC1F303215E204EEA0109984753
:10E9A8003B68062098475FFA89F01DF0C1F84FEAE6
:10E9B80019201DF0BDF8B4F81631029A8849B2F84A
:10E9C80000904A7A01339BB2012A93FBFAF00AFBC2
:10E9D8001033A4F8163100F041836E2381484A7B36
:10E9E80003FB09F380FB03014FEAE379C9EBA109B3
:10E9F8002AB1794B1FFA89F91B7899FBF3F93B681F
:10EA0800DFF8F8A15E2098471FFA89F93B683A2099
:10EA18009847AAFB093A4FEA5A1A1FFA8AF3D8B25A
:10EA280002931DF085F8029B180A1DF081F83B68D7
:10EA38005E2098473B683B209847642303FB1A9362
:10EA48009BB26948053380FB0320DB17C3EBA000AA
:10EA5800C0B21DF06DF800201DF06AF83B68DFF8C1
:10EA680090A1DFF884915E2098473B68282098475A
:10EA7800DAF8003089FB0329DB17C3EBA9095FFA31
:10EA880089F01DF055F8C9F307201DF051F83B68CF
:10EA98005E2098473B6804209847B8F80830002B58
:10EAA80040F02282DAF8083083F310085FFA88F021
:10EAB8001DF03EF8C8F307201DF03AF877E4C4F8D3
:10EAC80024B187F80090FEF7F2B9484A434B0B92FD
:10EAD80012AEA2F13D0046F8200D1988444FA2F16C
:10EAE800400300204FF00A0E02F8400C082283F879
:10EAF80001E030469A70F6F7D6F83B683A49DA17DB
:10EB080081FB0313C2EBA30399B23046F6F7CBF8A7
:10EB180002F0F8FBBF680A9B3A0C591C0A911A705C
:10EB28000A9B3A0A591C0A911A700A9B5A1C0A92A3
:10EB38001F700A9B5A1C0A92187030461DF016F86E
:10EB4800FEF7FDBA2B4F9FED2C8AB7F90220274814
:10EB58000B9007EE902AF8EEE77A12AE67EE887A05
:10EB6800A0F13D01FDEEE77A46F8201D00F8403C93
:10EB78000823CDED027A00F83F3C1E23BDF80810AB
:10EB880000F83E3C3046F6F78EF8B7F9003007EE4D
:10EB9800903AF8EEE77A304667EE887AFDEEE77A43
:10EBA800CDED027ABDF80810F6F77DF8B7F9043014
:10EBB80007EE903AF8EEE77A304667EE887AFDEE8F
:10EBC800E77ACDED027ABDF80810F6F76CF8304612
:10EBD8001CF0CCFFFEF7B0BA164F0020004F002003
:10EBE800084F0020310CC330676666660C7500203C
:10EBF800AC7400201C42002058A08B411F85EB51AB
:10EC08009AF80240C4B1013CE4B20134544451467C
:10EC1800002211F8013B534083EA0313DBB2120AC6
:10EC2800DF0042EA03228C4287EA131382EA0302D6
:10EC3800EFD1002A7FF433ACB24AB34FB34B1288FA
:10EC4800B349B44CFA61DFF8F8921A6809689B680E
:10EC5800FA62B4F85221F866FB64D9F80000F96347
:10EC6800FA65F7F79BF8029000287EF492A9022132
:10EC7800D9F80000F4F770FB94F854319AF803209F
:10EC88000392642B4FF0040287F8742040F05C81F3
:10EC980094F85531072B04BF9DF8083084F8553196
:10ECA80094F85531069307EB031ADAF80410029129
:10ECB80008461FF051F9DAF8081005915FFA80FA52
:10ECC80008461FF049F9C0B204900AEB0002069BFF
:10ECD8009148029902900832C27123F00F028646C9
:10ECE8008272049803F00F0300EBCA008EF80D300F
:10ECF80052468EF80E000EF10F0020F0B1F9874B46
:10ED0800049A05990AF10900184420F0A9F9029813
:10ED1800C37903F1010ACBB1013B5FFA83FC0CF123
:10ED2800080CDFF820E284440023073010F8011BA8
:10ED380059408B00CA0883EA410302F018024B408D
:10ED48004EFA02F253408445DBB2EFD1734A03987E
:10ED58000AF8023014F0C2FB94F85531002201334E
:10ED680084F8553184F85421029BDDF808A09B787B
:10ED78005BB11AF80510D9F80000F4F7FCFA013570
:10ED88009AF80230EDB2AB42F3D894F8543103222A
:10ED9800013384F8543187F8742088F80020FFF78D
:10EDA80051B80221D8F80000F4F7D6FA94F82C31BB
:10EDB800FEF7ACB84FF000094846FFF7ECBA4046FA
:10EDC800FFF7D2BA1023042218460AA98DF82A9010
:10EDD8008DF82B908DF82C908DF82D908DF828308B
:10EDE8008DF8292011F01CFE84F83791FEF7B9B888
:10EDF8004B49881F11F0E2FC84F84601FFF79EB8E2
:10EE0800484AD278002A0CBF4FF0040C4FF0050C8A
:10EE1800FEF746BE3B4B1988FFF750BA0123D8F8D6
:10EE280000003B70F4F79EFA0746D8F80000F4F7A4
:10EE380099FA7F067EF43BA88E287EF438A894F8C9
:10EE48002031002B7EF450A8374BC4F828312D23ED
:10EE580084F82C31FEF732B80326344943E5344BA5
:10EE6800344A1B68344903F48003834216BF1146B1
:10EE78000426032628E523499A790B8803EB8303A4
:10EE880003EB83034FEA83081FFA88F8002A00F08F
:10EE980003811E4B1B680FFA83FA02F033FA40B263
:10EEA800FEF71CBA4FF03408FFF7F4BB98469946B2
:10EEB8001846049305930393FEF708BB1F490426DD
:10EEC80011E54FF02408FFF7E5BB4B1CDBB2042B20
:10EED80084F849314FEA01617FF4A1A9FFF79CB991
:10EEE8004FF01008FFF7D6BB02F00CFA1CF020FE1A
:10EEF80000201CF01DFEFFF75ABA4FF02008FFF75C
:10EF0800C9BB00BF004F002008000020AC740020DF
:10EF1800B076002058250020D05D0020D65D002066
:10EF280098260020E05300208C750020F84803083C
:10EF380094660020F4480308EC480308FC480308DA
:10EF4800506A00200007090E97F875A065490495D6
:10EF58001AF00F0F04BF0AF1010A5FFA8AFABAF130
:10EF6800070F28BF4FF0010A4FEA0A1C07EB0C03F2
:10EF7800187C5D4B02930A18002392F824105A4A11
:10EF880093725FFA8CF31A46584B964607EB0C02BD
:10EF98004EEA000001291870D26803F101000CD96B
:10EFA8000239C9B28D1C1D44034603F8012BAB423C
:10EFB8004FEA1222F9D101310844BC4422F060031F
:10EFC8000AF1010A9CF811205FFA8AFA1343BAF190
:10EFD800080F037000F101035AD04FEA0A1C07EB2F
:10EFE8000C01424A087C3F4901449A1A91F82410BE
:10EFF80055180EF1100E132D5FFA8EFEC6DD049D16
:10F008000298DFF8F4E0D1B28B1DDBB243F0400286
:10F01800C27103F1010CCBB14B1DDBB20833C3182D
:10F0280004930EF10100002310F8011B59408B00D6
:10F0380083EA4103CA084B402D4902F0180241FAFD
:10F0480002F25340049A8242DBB2EDD103980CF8E5
:10F058000E3087F875A014F041FA85E63B685E200B
:10F0680098473B68392098475FFA89F01CF060FDA3
:10F078004FEA19201CF05CFDF0E44FF00808FFF798
:10F0880009BB1C4B9046B3F900A06420FEF726B9D3
:10F09800164A049D9A1AB3E74FF0FF33FBE69846E9
:10F0A8009946184604930393FEF710BA9846994672
:10F0B8001846049305939E460393FEF707BA0393F5
:10F0C800FEF704BA98460393FEF700BA98469946A5
:10F0D8000393FEF7FBB99846994618460393FEF743
:10F0E800F5B900BF981F0308D05D0020DD5D002042
:10F0F8000007090EAC740020D65D00202DE9F04F02
:10F10800724B734A1C7893B000F59C4120318146BC
:10F1180007911160002C00F0E8846E4A1268904252
:10F1280040F221826C4A6D491768DFF8E8B1049211
:10F13800013C1C706A4C039107F48057002F40F083
:10F148001F82039B5B7D002B40F09B84049B1B6804
:10F158001E0400F1F286634B9945A37800F273838D
:10F16800002B40F07383604B0593049B1F6817F4D2
:10F17800805940F0FA83039BBBF906605B8B9E4283
:10F18800B4BF00260126594B1B6813F0805300F0CA
:10F198000182059A127812F0010200F002820398A7
:10F1A8005349408C91ED037A07EE900AF8EEE77A1E
:10F1B800B4EEE77AF1EE10FA80F2A587002E40F05F
:10F1C800F7814C4D95F8A010002940F0F1814A488C
:10F1D8004A49056895F82D50002008604860886005
:10F1E8004749002D40F0E5810D70002A40F0E68186
:10F1F800444B1A78002A50D10399BBF900E04F8B91
:10F20800898BBBF90200BE45CCBF8025002545F09F
:10F2180040038E45A8BF2B469B0843F08005B842A3
:10F22800C8BF2B4643F040058842A8BF1D46BBF91E
:10F2380004E0BBF90600AD0845F08003BE45C8BF31
:10F248001D4645F040038E45A8BF2B469B0843F05A
:10F25800800E284DB842C8BF734643F0400E95F85B
:10F26800A2708842B8BF73469F4201F0C180A5F8DA
:10F27800A42085F8A620244985F8A2300F78002F0D
:10F2880001F031805F2B01F099806F2B00F093879C
:10F29800059B1B78DE0740F15587049B1B4A1B68BA
:10F2A800069203F00403002B40F0D6840DF14008C9
:10F2B800174D0023C8F8043005F15009109340F6A3
:10F2C800330A192740F2833629E000BFD8400020CE
:10F2D800603C0020D4400020946600202068002074
:10F2E800E0530020404B4C0068740020C07600209A
:10F2F800184F0020242800203C4200201C33002006
:10F30800202500201C45002011210020C87600205F
:10F3180074350020485F002004354D4520D0AA7878
:10F32800EB789A4217FB0260F6D26978043117FB32
:10F3380003623BF911305345A8BF5346B3F5617FCB
:10F34800B8BF4FF461739842E6DA9A42E4DB297851
:10F358002429E1D840460435F5F7AEFE4D45DED107
:10F36800AD4B98E803001F78AC4B83E80300002FEF
:10F3780000F0FD830121A948F5F7ADFE002840F013
:10F388009A81E378002B40F09681A54C23881DB222
:10F3980025F00105AEB2B342268000F06186A14D8A
:10F3A80002270E204FF014094FF0FF082F7085F840
:10F3B800019085F8028018F05FFD39469748268845
:10F3C800F5F789FE002840F0A78726F002039BB2D4
:10F3D800B34223800AD0934B1421FF2202250E202A
:10F3E8001D7059709A7018F047FD26888E4B03934C
:10F3F8001978DFF880A2B30708BF81F00201DAF8B4
:10F408000400C1F34001F4F7BFFF24218348F5F756
:10F4180062FE30B9059A13785F0744BF23F00403EE
:10F428001370069B1B6813F00A0F1AD006217B483D
:10F43800F5F751FE002800F0348623885E0640F177
:10F448002C8707217548F5F746FE50B1774B784A67
:10F45800B3F90430774982FB0302DB17C3EBA2033D
:10F468000B800C216D48F5F736FE2288002800F045
:10F478003E8142F480739A42238009D0694B022569
:10F488001421FF220E201D7059709A7018F0F4FC98
:10F49800694B1B78082B00F036810E2B00F0338166
:10F4A800049B1B685D0544D5644B1B79002B00F059
:10F4B800E78014215948F5F70EFE002840F0E58052
:10F4C8001CF0C4FB012018F01FFC90B3DFF8A881E2
:10F4D80000254FF0CC0902E0DDB2022D29D809FB46
:10F4E80005F76B1C58F80760002EF5D1C378544A0D
:10F4F80090F9020052F8233001960322009201216C
:10F50800324618F089F8034605EB450000EB001079
:10F51800049353B1314608EB8000CC2222F0B5F8B1
:10F52800049B48F807300135EDB21AF0C7F90028F6
:10F53800D3D1059B1B78D80740F1F8804149424A4E
:10F5480001230B701370039BDAF80000197801F09F
:10F558000101F4F719FF069B1B685B0700F1568150
:10F5680013B0BDE8F08F394B394A1F68049307F48C
:10F5780080570392DFF804B1364C002F3FF4E1AD19
:10F5880000212648F5F7A7FD00287FF4DAAD15F02D
:10F598003BF8D6E57D023FF5FCAD059A127802F0FE
:10F5A80001022D4D002185F8A010002E3FF40FAE6A
:10F5B8002A4901200870002A3FF41AAEF8067FF5A0
:10F5C80017AE274A1278D1063FF512AEB9F1000FEF
:10F5D8007FF40EAE002B7FF40BAE7A023FF508AE37
:10F5E800204B1B78002B01F0E8821F4B9B78002EE4
:10F5F80041F0F3823BB11D4A1D4B12681B689B1AF0
:10F60800002BC1F290831020134D18F035FC012314
:10F6180085F8A130ECE500BF6A530020C0760020D1
:10F628000C420020C8490020105500201C42002030
:10F63800676666662424002070350020084F002085
:10F6480064470308697400205C2400209466002045
:10F6580020680020E05300202428002020250020D6
:10F6680090760020112100204C35002048550020BC
:10F67800F45F002014550020F0500020485F00205F
:10F68800059B1B78D9077FF51BAF3C2013F08EFD37
:10F6980000283FF44EAF02F0E3FF3C2013F032FDA8
:10F6A80000283FF446AF02F0DBFF3C2013F02AFDB0
:10F6B8000028F0D13DE7069B1B6898077FF565AEEB
:10F6C800BF4C2688F1073FF580AE46F001039E4205
:10F6D80023803FF47AAEBB4B1421FF2202250E2073
:10F6E8001D7059709A7018F0C7FB26886DE622F4D1
:10F6F80080739BB29A4223807FF4C0AEB24B1B78D2
:10F70800082B7FF4CAAE228822F040039BB29A42AB
:10F7180023803FF4C5AEAB4B02251421FF220E20F7
:10F728001D7059709A7018F0A7FBB9E6A74B93F8AB
:10F738000090B9F1000F5FD1DFF8E482A44F18F808
:10F74800030C3E784146A8F103051DF03FFD002853
:10F7580000F09C83002E40F0EE8305F108016879E3
:10F768001DF034FD002841F01D819A49A87A1DF04A
:10F778002DFD002800F09D83022E41F0308196492E
:10F78800E87B1DF023FD002841F02D819349287D59
:10F798001DF01CFD002800F09D83042E41F02781F8
:10F7A8008F49687E1DF012FD002841F024818D49A3
:10F7B800A87F1DF00BFD002800F09D83062E41F068
:10F7C8001E81894995F823001DF000FD002840F0AE
:10F7D800BA86864995F828001DF0F8FC002800F044
:10F7E8009D83082E40F09986814995F82D001DF0DB
:10F7F800EDFC002840F09D837E4B01221A701DF01D
:10F8080068FF069B1B685B077FF5AAAE03201DF007
:10F8180007FD002800F0E785238813F008047FF42B
:10F828009FAE082018F038FC7348744D7449754A27
:10F83800754BBBF8066000682E80086014601C6079
:10F8480013B0BDE8F08F0BB90123A3706F4B05937C
:10F858001B201F7894F821601DF0E2FC012E07F0B0
:10F868000109824600F0A68507F00203069394F882
:10F878002030DFF8B081664D052B69D8DFE813F03A
:10F888005B004F000600DC00FF008D00012E04BF66
:10F89800052384F82030B9F1000F00F01381039B91
:10F8A8005C4FB3F91810B8F80030002261F30F026A
:10F8B80063F31F42002361F30F0361F31F43CBF887
:10F8C800042039686269CBF800308A42C0F00284AB
:10F8D800012E41F0A081032294F820300692CBE754
:10F8E8001DF0CAFC012807D14A4FB8F802303A681F
:10F8F800642101FB03232361BAF1000F04D098F8B7
:10F908000630002B40F09080012E21D0414F226913
:10F918003B689A42C0F0B585012384F82030012E57
:10F928003BD098F80730012B00F0D5800EF042FE4E
:10F9380094F82030A0E7B9F1000FD1D14FF48060DE
:10F94800BAF1000F00F0AA8318F0A6FB0023236188
:10F95800069B002B3FF409AC069818F08DFA049B1F
:10F968001F6817F480593FF406AC1D212A48F5F7A3
:10F97800B2FB00287FF4FFAB284A039BD2881B8B7D
:10F98800BBF90660991A8E4240F3788513449E426B
:10F99800B4BF00260126FFF7F6BB1E4F3A68B8F839
:10F9A8000230642101FB03234FF4806000222361AD
:10F9B80084F82020E27018F057FB94F820305BE7B9
:10F9C8000C420020C84900207035002069740020CE
:10F9D8007E00002050480020554800205A4800204A
:10F9E8005F48002064480020694800206E480020D5
:10F9F800734800205C240020B076002030240020CA
:10FA08003C240020342400202C240020687400208A
:10FA1800CC76002048550020C0760020A44900205C
:10FA280046480020C04900200EF0C4FD03224FF4D0
:10FA38007A7384F82020E361994F2B8843F00203FE
:10FA48002B8014F0E1FD3A68E36913440422A361B2
:10FA580084F82020012E40F01E853B68A2699A4256
:10FA6800BFF476AF8F4B187820B91DF0D9FB00286A
:10FA78007FF46EAF2B8823F002032B808EE7884F2C
:10FA8800E8E7039A013BD27D3BF91330002A40F0A6
:10FA98001C83A3F57A73B3F57A7FA8BF4FF47A7302
:10FAA80023EAE37307EE903A9FED7F7AF8EEE77A60
:10FAB80067EE877A7D4AFCEEE77A17EE903A138074
:10FAC800FFF749BB764F3B6847F230520323E261A8
:10FAD80084F82030B1E70EF06DFD032240F6B8330C
:10FAE80084F82020E3616E4FA7E7714F3B78002B25
:10FAF80000F00D876F4BDFF8D481DFF8D4B1DFF861
:10FB0800D4A1039345465E46049099460EE019F841
:10FB180004109847032C28DC88B93B782AF8020F90
:10FB280001349C4205F1040580F2DA80072CE1B229
:10FB38003046DBF80430EADD984700B2EDE738F8E4
:10FB480024206B88801A4FF47A719B1A01FB00F00D
:10FB580040F6CA0290FBF3F00844904240F2EE23CC
:10FB6800A8BF10469842B8BF184600B2D5E7DFF8DC
:10FB780068A1DFF86881504D0AF15A064FF0010973
:10FB880051461AF8010C1DF021FBF8B19AF804004F
:10FB98009AF802309AF803E000EB400105EB810186
:10FBA800013BD1F8B42003EB4303434493420DD007
:10FBB80095F8E02081F8B0E009FA00F022EA0000A8
:10FBC800C1F8B430C1F8B87085F8E0000AF1060A47
:10FBD800B245D5D13949324A394B3A4D09681B7873
:10FBE800D2F8009008910793A5F1B00A00266B6837
:10FBF8005BB31F784FB3AA68A9EB0202002A0ADB9D
:10FC08009AF8E0200121B14022EA010209F5FA71CF
:10FC18008AF8E020A960079ABAB12A78597804329C
:10FC2800D2B2002940F0758203993BF91220098B62
:10FC380001F1C800824240F3F3839AF8E0109A7801
:10FC480041FA06F3D90740F163840136042E05F121
:10FC58000C05CCD1FFF78EBB174D95F8AA3053B1E0
:10FC6800059B1B78D80706D5039BBBF906205B8B41
:10FC78009A4200F3238411211348F5F72CFA00283F
:10FC880000F02F8295F8AE302BB995F8A83013B94B
:10FC98003223A5F8AC30012385F8AE30FFF706BB58
:10FCA8004855002011210020AAF1823FAA760020A1
:10FCB800546A002020680020242800204C77002067
:10FCC800E1410020D4280020C07600206C6A002082
:10FCD80030540020222800205D470020EC1F030834
:10FCE800DDF81090C44A04921146C44A0968A2FB80
:10FCF800092A42F201020A404FEA9A1A059200F0D4
:10FD0800EC81BF4DBF48C04CC04A95F800E0007870
:10FD180084F800E01070BEF1000F04D0BB4A92F8DE
:10FD280000E08EF0010EBA4D0F2085F82400002B5C
:10FD380000F0BB82B74B039E0C931B78B6F826C025
:10FD48000B931C463B78B78C039EB34A368B0E96B2
:10FD58002646A2FB0442520802EB4202B21AD2B271
:10FD6800CDF824C001F48051089295F82580DFF879
:10FD7800C0B2DFF8E8C20A900AF5967276460F918B
:10FD880005F1280400200692CDF83490AE46002EE6
:10FD980000F026823EF910201FFA82F9B9454FEA91
:10FDA800400103D3099DA94540F25D825CF82020FB
:10FDB800924580F01E823BF90120059D002D40F000
:10FDC8003182013098422BF8012004F10604DEDB71
:10FDD8000A98924ADDF834908EF825800F280CBFD7
:10FDE800012100218EF82400117000F065828C4CEE
:10FDF8008C4E8D4F35883868A1686268E06045F0A0
:10FE08000405401A90427F4F3580804D4FF0010124
:10FE180088BF00223970297088BF84F82120002B00
:10FE280000F05C82049A03991768804EB1F824C0E8
:10FE3800B1F818E07E4817F48057354640F07D82C7
:10FE480039460EE06A7802EB820202EB820202F285
:10FE5800EE2292B20131994220F8022B05F10205F7
:10FE68000ED016F81120002A00F00182022AE9D0EB
:10FE78000131028820F8022B994205F10205F0D1E0
:10FE88000C9A137801331370FFF758B908F105017C
:10FE980068791DF09BF900283FF467AC012E40F00B
:10FEA800818505F10D01A87A1DF090F9002840F030
:10FEB80096856049E87B1DF089F900283FF466AC17
:10FEC800032E40F090855C49287D1DF07FF90028BD
:10FED80040F08D855949687E1DF078F900283FF477
:10FEE80066AC052E40F087855549A87F1DF06EF950
:10FEF800002840F08485534995F823001DF066F9E1
:10FF080000283FF466AC072E40F01D834E4995F853
:10FF180028001DF05BF9002840F0FF824B4995F856
:10FF28002D001DF053F900283FF466AC092E3FF46C
:10FF380063AC4FF009094B46F2E2354DD5F88830ED
:10FF4800A9EB0303002BFFF606A9414A95F88C306C
:10FF5800517C079AC5F8882001333E4A039E32F83F
:10FF68001120B17D03F00F0385F88C302B4492B239
:10FF780092FBF1F283F8902095F8901095F8912073
:10FF880095F8923095F89C000A4495F8931013441C
:10FF980095F89420194495F895300A4495F89610E8
:10FFA800134495F89720194495F898300A4495F821
:10FFB8009910134495F89A20194495F89B300A44EF
:10FFC800134495F89D1095F89F20184495F89E3095
:10FFD80001440B441A4442F30B12642AF17DA8BF72
:10FFE800642213B209B1C2F1640307EE903A9FED9F
:08FFF8001A7AF8EEE77A5BE5E6
:020000040801F1
:1000000094660020D34D62103C3C0020CC000020C0
:10001000E1410020CD00002024280020016A0020BA
:10002000ABAAAAAA2E540020E0530020CC760020D0
:1000300048550020A06A0020485F00205548002055
:100040005A4800205F48002064480020694800208A
:100050006E48002073480020C4540020E054002063
:1000600014AE2341046A00200221C548F5F737F891
:1000700000283FF4AEA92580B2073FF5BBA946F0A2
:100080000203B34223803FF4B5A9BE4B02201421E2
:10009000FF2218700E2059709A7017F0F1FE268812
:1000A000FFF7A8B917F0E4FF54E4228822F04003D8
:1000B0009BB29A4223803FF4C8A9B24B0225142177
:1000C000FF220E201D7059709A7017F0D9FEFFF7AD
:1000D000BCB9C3F53B6308331BB2DEE403230693CC
:1000E000F6E4A94A92F800E019E695F8A830002B4A
:1000F0003FF4E0A8059B1B7813F001037FF4DAA816
:10010000012285F8A83085F8A920FFF7D3B89F4DC4
:10011000012185F8A010FFF74FBA012900F0B6833E
:100120009AF8E0200123B34001361343042E8AF8E5
:10013000E03005F10C057FF45EADFFF71FB9059BBC
:10014000934A1B781060DB0700F1CA8195F8A6106E
:1001500000297FF4A6A8B5F9A430322B7FF7A1A817
:1001600095F8A2200120572A85F8A60000F0038404
:10017000049B1B6813F0040302D05A2A00F00E857A
:100180005D2A00F086845B2A00F0A8845E2A00F0D5
:10019000B284562A00F0E784972A00F0F384A72A55
:1001A00040F03F847B49049B0A781B6842F00402BC
:1001B0000A70794A069203F00403FFF778B8B2F5A3
:1001C000FA7FFFF66EA895F8A620002A7FF469A8AA
:1001D000059B1B780121DF0785F8A61000F1178425
:1001E00013F058FDFFF75DB8002F3ED05CF82020DB
:1001F00092454FEA4001FFF4E2AD684A674D525C18
:1002000005EB0109002A7FD0022A47D199F8012085
:1002100002EB820202EB820202F2EE2292B2032889
:1002200033DD059D12B2002D3FF4CFAD089D24F8BB
:100230001520B8F1000F03D10B9D022D7FF6C5AD3F
:100240002288B4F80290B4F804804A449044544A96
:100250000FFA88F882FB0852524DA2EBE87225F89B
:10026000018012B24FF00108AFE53A464100069D09
:100270004CF82050A5E5CAB2022A04D9032A7FF41B
:10028000FBAD6246EAE57246E8E5012505FA00F9AC
:100290000A9D25EA090512B20A9592E53BF801206C
:1002A000BDE743F04002934222807FF406AFFFF7A0
:1002B000CCB83D493D4A0C91DFF8FCB001211170EA
:1002C0001B212F480593F4F70AFF059B00287FF4B4
:1002D00092AD374C374FE2683B68A3609B1AC82B3E
:1002E00000F23B83049B1F6807F48057CCE5394636
:1002F0002348F4F7F4FE00283FF421AF85F8A770F7
:1003000013F0C8FCFEF7C8BFC2B2022A40F2BC829A
:10031000032AC3D10E9A0F9D002D08BF3A467EE7EF
:1003200026F001039BB2B34223803FF4A5AE0E201A
:100330002F7085F8019085F8028017F0A1FD2688BE
:100340009AE600210FE06A7802EB820202EB820259
:1003500002F2EE2292B20131994220F8022B05F10D
:1003600002053FF491AD16F811201AB1022AEAD025
:100370000288F0E7CAB2032AFAD87246EBE700BF58
:10038000C0760020C8490020E14100202428002038
:10039000F85F002090760020C8760020A06A002038
:1003A0005655555594280020016A00202E540020EF
:1003B000E053002048550020485F002000230693AA
:1003C000FFF759BAB2F5FA7FFEF66BAF95F8A63093
:1003D000002B7EF466AF059B1B7801210B4085F84E
:1003E000A61000F09C8214F013F9FEF75ABF082003
:1003F00017F03EFEFFF7B8B8BB4ABC491068B5F924
:10040000A420C76981FB07018911FF17781A00F53D
:10041000FF407F3082423EF732AFC91B0A4412B21E
:10042000A5F8A420FEF72BBFC8398A423DDA9AF816
:10043000E0109A7841FA06F3DB073FF50AAC524226
:100440000120099217F0FCFD7B1E099A162B00F281
:10045000C280DFE813F0B101C7019801F001DD01AE
:10046000040283016E01570131011A01C000F0013D
:100470000501040283016E01EF00D900C300AE0044
:10048000960080000126FEF782BE0EF097F8032248
:1004900040F6B83384F82020E361FFF7D2BA3A6817
:1004A000E3691344A361FFF757BA9AF8E0300122D9
:1004B000B24023EA020309F5FA728AF8E030AA6032
:1004C000FFF7C7BB00218A48F4F709FE00287FF434
:1004D000D6AB322385F8AA00A5F8AC30FFF7CFBB26
:1004E000844B1B78002B3EF4DCAEE378002B7EF4CB
:1004F000D8AE95F8A7300133DBB2032B85F8A730CF
:100500007EF6CFAE7C4B5B7813B9002E7EF4C9AE7D
:1005100014F07EF8FEF7C0BE002A0CBF01200220B6
:100520008FE74FF008094B4603EB83031D4487F820
:100530000090A978687811F041F9059B6F4A1B7803
:1005400001211170DA077FF55EA9FFF700B84FF0BF
:1005500007094B46E8E7DAF8E400DFF8A48190F8F1
:10056000361098F8023011446429A8BF642121EAAA
:10057000E17180F83610002B40F08C830DF04AF9C1
:10058000CEE5DAF8E400DFF8788190F8371098F8D3
:1005900002301144FE29A8BFFE2121EAE17180F852
:1005A0003710002BEAD016201CF09CFEDAF8E4008D
:1005B000E4E70898DFF8488141781144B1F5967F67
:1005C000A8BF4FF4967121EAE171417098F80230AA
:1005D000002B40F05983DAF8E400CFE7DAF8E400C2
:1005E000DFF81C8181781144C829A8BFC82121EAFD
:1005F000E171817098F80230002BBFD014201CF0FC
:1006000071FEDAF8E400B9E7DAF8E400DFF8F08028
:1006100041781144C829A8BFC82121EAE17141707D
:1006200098F80230002BA9D013201CF05BFEDAF8FA
:10063000E400A3E7DAF8E400DFF8C48001781144AD
:10064000C829A8BFC82121EAE171017098F80230D9
:10065000002B93D012201CF045FEDAF8E4008DE761
:10066000DFF89C80089898F8023041791144642999
:10067000A8BF642121EAE1714171002BABD00E20AB
:100680001CF030FEDAF8E40078E7DAF8E400DFF88E
:100690007080017A98F802301144C829A8BFC82197
:1006A00021EAE1710172002B3FF468AF0B201CF0CE
:1006B00019FEDAF8E40061E7DAF8E400DFF84080D8
:1006C000C17998F802301144C829A8BFC82121EA8D
:1006D000E171C171002B3FF451AF0A201CF002FE02
:1006E000DAF8E4004AE700BF08760020D34D621034
:1006F000C0760020E14100204C3500205C24002021
:10070000A4760020DAF8E400DFF87885817998F89B
:1007100002301144C829A8BFC82121EAE1718171C2
:10072000002B3FF42BAF09201CF0DCFDDAF8E400CD
:1007300024E7DAF8E400DFF84C85417998F80230D4
:100740001144C829A8BFC82121EAE1714171002BD9
:1007500040F05282112F7FF445AF0FE7DAF8E40042
:10076000DFF82085017998F802301144C829A8BF24
:10077000C82121EAE1710171002B40F0D082102FD5
:100780007FF446AFFAE60899DFF8F8840F7917444A
:10079000642FA8BF642727EAE7770F711CF0BCFD20
:1007A00098F80230002B3FF416AF032039461CF0B6
:1007B00099FDDAF8E400E1E60898DFF8C8840178EA
:1007C0001144FA29A8BFFA2121EAE171017098F8D1
:1007D0000230002B3FF4FFAE01201CF083FDDAF85D
:1007E000E400CBE60898DFF89C8481781144642902
:1007F000A8BF642121EAE171817098F80230002BD2
:100800003FF4E9AE02201CF06DFDDAF8E400B5E635
:100810000898DFF87084C17998F80230114481F3A8
:100820000801C171002B3FF4D6AE05201CF05AFD23
:10083000DAF8E400A2E6089BDFF84884997998F892
:10084000020011446429A8BF642121EAE171997171
:10085000002840F0D9810D2F7FF404AFBBE6DAF811
:10086000E400DFF82084C17898F802301144C829E8
:10087000A8BFC82121EAE171C170002B40F05F825E
:100880000F2F7FF4DBAE79E60E9AC8E43BF9122015
:100890009978B2F5617F4FF4966393FBF1F331DB06
:1008A00040F633019142A8BF11460C2FA1F56171AA
:1008B00091FBF3F100F0F880182F7FF431ACC9B24E
:1008C000C8290B46A8BFC823DAF8E400C27DDFB20E
:1008D00097423FF425AC9A1ADFF8A883C77548BF42
:1008E0000732D71098F802300137FFB233B9002F22
:1008F0003FF416AC384617F0A3FB11E418201CF0A7
:10090000F1FCF4E70C2F00F0E680182F7FF408AC20
:1009100000210B46D8E7C44A0392FFF7E7B9C34961
:10092000096811F4003140F0EA800B46C048C65C0B
:100930000F2E03F10C033DD001311529F7D1049B93
:10094000BC491B680691FA3AA5F8A420002203F0DE
:10095000040385F8A620FEF7AABCB74A049B1F68CB
:10096000138823F004031380012307F4805784F8CD
:100970002130FFF789BAAF4AB04B069210461A6889
:10098000AF494FF47A73B3FBF2F3C3EB431203EBBB
:1009900082030268DB005507A1F8B43000F1A280A1
:1009A000049B1B6803F00403FEF781BC4FF00109B0
:1009B0004B46B9E5A34ED6F800E04B00BEF1000F60
:1009C00007D05F1800EB87079EF801E07F78774536
:1009D000B5D20B449C4F9D4900EB8300002330604F
:1009E0003B800B60ABE74FF002094B469CE54FF0B4
:1009F00003094B4698E54FF004094B4694E54FF048
:100A000005094B4690E54FF006094B468CE5049BE3
:100A10008F491B680A60874A069203F00403FEF7B9
:100A200046BC0021BB2A109100F09880B72A00F044
:100A30009180BE2A00F09580BD2A67D0792A00F007
:100A40005B817A2A00F051819E2A00F048819D2A1C
:100A500000F03E81AE2A00F03481AD2A00F02A81F8
:100A6000EF2A00F02181FD2A00F01881FB2A00F016
:100A70005081FE2A00F04781F72A00F068817B2A26
:100A80007EF40FAC4FF4FA6102201AF053F8FEF72F
:100A900008BC704B002201206F4D70492A700B601A
:100AA00017F0CEFAFEF7FDBBCFB26B4B09915B7826
:100AB000BB423FF435ABDFF8CC8138461AF014F96D
:100AC00098F8023009991BB1C9B20C201CF00AFC3D
:100AD0000137FFB20BE700273946E6E7604B0122FA
:100AE0000220D9E7049B5F4A1B680A21118003F0AA
:100AF0000403FEF7DCBB5C4B02220320CCE75B491E
:100B00000978032900F0868019460FE74FF6FE7337
:100B1000574A484896890690D089334401449381C6
:100B2000D18108F0E7FEF3F7A1FE08F0CBFEF6F75F
:100B3000EBFA012017F084FA049BB5F8A4201B6897
:100B4000FA3A0021A5F8A42003F0040385F8A610C2
:100B5000FEF7ADBB0B464FF6FE71D9E70B460221FF
:100B6000D6E70223D4E708F0C5FEF3F77FFE08F0CE
:100B7000A9FEF6F7C9FA012017F062FA95F8A2204B
:100B8000FFF70ABB049B3B4A1B684FF4C8711180F6
:100B9000284A069203F00403FEF789BB95F8A820C3
:100BA000002A40F0DF8095F8AA3083F0010385F831
:100BB000AA30002B40F0D1800C2017F061F9FEF72D
:100BC00070BB002E3EF423AD2B4D95F8A130002BC9
:100BD0003EF412AB17F038F9002385F8A130FEF788
:100BE0000BBB002BF0D02549254A09684FF47A70D9
:100BF00000FB03131360E7E7112009921CF072FB5E
:100C0000DAF8E400099AA5E50D2009921CF06AFBC8
:100C1000099A20E617F018F9B5F9A4208FE6032306
:100C20000693FEF79DBE00BF2068002050470020BD
:100C3000FC390308C8760020CC76002084660020AA
:100C400000640020F8240020482500204C250020C6
:100C5000F85F00207C430020404200203C420020FE
:100C6000CA4300206A77002018440020BC76002088
:100C7000303500206C7700202428002048550020C3
:100C8000F45F0020A476002015201CF02BFBDAF87E
:100C9000E40073E417201CF025FB9CE400210120F4
:100CA00019F048FFFEF7FDBA0021084619F042FF8F
:100CB000FEF7F7BAFF2100201EF08CF995F8A2206C
:100CC000CEE6012100201EF085F995F8A220C4E6A9
:100CD0000021FF201EF07EF995F8A220BAE601203F
:100CE0001EF078F995F8A220B1E6224A137A43F073
:100CF00001031372FEF7D5BA1E4A137A23F00103DB
:100D00001372FEF7CEBA0021032019F013FFFEF78D
:100D1000C8BA0021022019F00DFFFEF7C2BA102058
:100D200009921CF0DFFADAF8E400099A27E5124D7F
:100D300013F06EFC002385F8A130FEF75DBA0F209A
:100D400009921CF0CFFADAF8E400099A98E500213C
:100D5000042019F0EFFEFEF7A4BA0B2017F090F86C
:100D6000FEF79FBA054A85F8A81085F8A9000692F3
:100D7000FEF79DBA1454002024280020C8760020D5
:100D80002DE9F0478C4B1B78DB07074644D58B4B8E
:100D90008B4D1C788B4E012C59D01CD3022C07D1C3
:100DA00089498A4A09881288914201D901241C7014
:100DB000EB7AE3B12B89D3B1854B1B78BBB100F043
:100DC000A5FA002800F09B802B7B83422CBF0121D9
:100DD000002131700CE07C497E4A098810886A7BCA
:100DE000801A8842E2DAEB7A0024002BE2D13178D3
:100DF0002A79632A06D8022C774E00F0BA8033781D
:100E0000002B5DD1754AAB7A8C4238BF0C4614700A
:100E1000002B4CD1BDE8F0876B4B694D19885B887E
:100E2000E878CB1A83EAE3728142A2EBE3721DD326
:100E30002B788B421AD3614B1C78E01E012861D9B4
:100E40006749097802294FD0012C5E4EA5D15F4A2F
:100E50005D491288687B0988121A914239DD5D4A22
:100E600012888A42A4D200241C70A1E7B1EB400F83
:100E7000E1DC524B1C78E11E012940F29480022AE9
:100E8000DEDC57494F4E0878DFF84481DFF844C173
:100E9000DFF838E100210324022834701C7088F840
:100EA0000010ACF80010AEF8001081D11FE0012C4A
:100EB00071D0022C0BD10720BDE8F04716F0E0BF3F
:100EC0007068381A474B984258DD72709AE7BDE84F
:100ED000F08702241C706BE7022AD2DD40490978B2
:100EE00002294FF0040464D13949364E09783E484E
:100EF000022ACCBF00220122C28081804BE702215E
:100F0000317075E7022A9BDC95F800C091FBFCFC70
:100F10000CF1010CBCF1080FDFF8B4A0304EA8783A
:100F200095F801E096F800802A4CDFF8A090254E55
:100F3000A8BF4FF0080C8AF800C01FFA8CFA10FB0B
:100F40000AF01EFB0AFE80B2DFF88CA02080A9F810
:100F500000E000244FF0640EB8F1020F34701C70F2
:100F6000CAF804408AF801E07FF439AF0FFA8CF137
:100F7000BDE73078A0B9012377603370C2F1640215
:100F80001A4B00FB02F083FB0023C017A0EBA35019
:100F90006430707036E70820BDE8F04716F070BF87
:100FA0007368F81A8EE7032C96D10D490978022947
:100FB0009AD0044EFCE600BF68740020642900202B
:100FC000947600206A290020004F00206829002024
:100FD000164F0020662900201C240020BC7600202B
:100FE000384E00207F9698003C4E00206BCA5F6B05
:100FF000024B1A889B780280837070473420030864
:10100000084B196861B130B45D68074C642202FB7B
:1010100005F2B2FBF1F2228030BC0020186058606B
:10102000704700BF0C290020E8310020704700BF46
:10103000F0B53B4B5B79012B83B03AD0022B0FD03C
:10104000384B00221A805A80374B1B78022B05D16F
:10105000344A364B5188128819805A8003B0F0BD4B
:10106000334B1B681B01EFD5FF200FF003FA037809
:101070000A2B51D8B0F902202E49D31781FB021256
:10108000C3EBA2039BB207EE903AB8EE670A2A4C74
:1010900004F10C006381F1F743FDFCEEC07A214AB4
:1010A0006389CDED017A5380BDF80430238113802C
:1010B000CAE7224A224B92781F4D33F81240A4B25D
:1010C00007EE904A05F13400B8EE670AF1F728FD03
:1010D0001C4A1449107896785378FCEEC07A00EBDD
:1010E0004010CDED017ABDF8042044F6FB77C3EB48
:1010F000033300FB027200FB0474B2FBF3F2B4FB97
:10110000F3F3B2FBF6F2B3FBF6F392B29BB22A868C
:101110006B860A804B8097E79FED0B0A0023B6E7AA
:1011200094760020004F0020384E00203C4E0020D6
:1011300094660020676666660C290020C45400206F
:10114000E05400206743002000000000F8B5304D57
:10115000304C31496E79314B314A324F042008709E
:1011600084F8580000216420012EA4F85A10A4F835
:101170005C103970197059605870118051802DD0F1
:10118000022E0ED0A979284A00230229136084F880
:101190005E305360936034D004292DD001290ED0E5
:1011A000F8BD282204F1080020F073FA4CF2503107
:1011B0009FED1E0A04F10C00F3F734FFE2E71C4A2E
:1011C000236653609360D3609FED1A0A02F110000A
:1011D0004CF25031BDE8F840F3F724BF282204F167
:1011E000300020F056FA4CF250319FED100A04F115
:1011F0003400F3F717FFC5E70F4AC4F8A030536077
:10120000F8BD0E4AC4F8943053609360F8BD00BF37
:10121000947600200C290020BC7600201C2400209D
:10122000004F0020164F0020AC740020CDCCCC3DE8
:101230006C290020CDCCCC3EAC290020A029002078
:101240002DE9F0432F4DD5F8A83083B01BB195F8A8
:10125000AC30022B02D003B0BDE8F0834FF0200881
:101260004046294C05F1B009012655271BF0DCFF4B
:10127000A0B199F800300BB9217891B908F10108B3
:101280005FFA88F8B8F1230F04F1010409F10109AC
:10129000E1D040461BF0C8FF0028EAD189F80000E1
:1012A000ECE7D5F8A80050B30DF1080EAA220EF80D
:1012B000052D8DF802108DF800708DF801608DF805
:1012C0000430694655225340082213F0800F02F182
:1012D000FF324FEA430318BF83F0310312F0FF02DD
:1012E000DBB2F2D1714502D011F8012FEBE7AA224F
:1012F00069468DF803308DF8042011F0A3FE89F8BB
:101300000060BBE70C290020382003081F4B187829
:10131000002839D01E4A1389FBB11E4A9FED1E6A70
:10132000D2ED026A07EE903AF8EEE66AF8EE677AD6
:1013300007EE103A77EEE66AB8EEC77A66EE866A8E
:10134000C6EE877AFDEEE77A17EE900A6428A8BF0A
:10135000642020EAE070C0B2704710B40F4B54789C
:101360001B88117804FB1032091B642300FB01F079
:1013700003FB02F3B3FBF0F06428A8BF64205DF820
:10138000044B20EAE070C0B2704700BF164F002047
:1013900094760020AC7400200000C842004F00206A
:1013A0002DE9F04F794D81B0F6F790F9D5F8B840B6
:1013B0000022C5F8B420002C00F0A580237D052B69
:1013C000074617D9216A23690B44C31A9342B8BF51
:1013D00005F1B8010ADBD5E0137D052B0AD9136AA4
:1013E00012691344FB1A002B80F2CC8051F8042FB1
:1013F000002AF1D14FF0010B0023B9461E46C5F873
:10140000B43098469A46274623E07A6A39693B7D8C
:10141000A9EB0204B4FBF1F40134A4B213FB04F30E
:10142000013301369BB2B6B23C83FB82984506D2AB
:10143000BBF1000F01D1012C5FD99846BA46D5F80F
:10144000B430013305EB8302C5F8B430D2F8B8707C
:1014500047B3BB68C3B1FC8A002CD6D1396A484671
:10146000A9EB01019847D0B195F81431002B52D166
:101470003B7DC7F82490013601334FF00102B6B22C
:101480003A83FB820124D1E73B6A3A69A9EB030462
:10149000B4FBF2F4A4B23C8334BBFB8AC6E73C83C2
:1014A000FB8AC3E72B686A683949013316443C4616
:1014B00085E848004F46C1F800A0BAF1000F27D0D8
:1014C000DAF8203095F81421AAF81640FB1ACAF869
:1014D0001C30CAF82090002A35D1DAF80C30484682
:1014E00001B0BDE8F04F18473B7D13FB04F3013317
:1014F00001369BB2B6B2FB8298E73A7D062A04BF5A
:101500009846BA469BE72B68214A01332B6014604A
:1015100001B0BDE8F08FF6F7D9F81E4B1E4A1F4CFC
:1015200011681A68A0EB090002EB000E2268C3F8EC
:1015300000E09042A1EB5111014438BF1046164A19
:101540002060116094E7F6F7C1F8DAF80C30044631
:101550009847F6F7BBF8DAF82C20DAF82830DAF8F2
:101560003010001B9042A3EB53130344014438BFD7
:101570001046CAF82830CAF83010CAF82C0001B05A
:10158000BDE8F08F4FF0000B36E700BF0C290020BC
:1015900008760020EC310020F0310020F4310020EA
:1015A000F0B43423184F194A03FB00F3D2F8186142
:1015B000FC58FD18002E6B684B600C600DDDD2F8F6
:1015C000B8309D421DD0B832002303E052F8044FDA
:1015D000A54216D00133B342F8D10022342303FBD5
:1015E00000700A720369CB60037D4B72836AC56A1F
:1015F000046BC2690A615B094D618C61CB61F0BC0F
:1016000070470122EAE700BF981C00200C29002047
:101610002DE9F041244ED6F81851152D27DC002D68
:101620003DDDD6F8B830984221D005F1804106F171
:10163000B807013907EB81013B4603E053F8042F5B
:10164000904214D08B42F9D1D6F8B8409CB1237D9A
:10165000017D8B420ED3154A002405E052F8043F69
:101660004BB11B7D8B4206D30134A542F6DA002034
:10167000BDE8F08100248046601C80002A1B011F09
:1016800006EB840439443844920001351FF0E7FF2B
:10169000C4F8B880C6F818510120BDE8F081E6D141
:1016A00006F1B807D0E700BF0C290020C4290020AC
:1016B000172830D0152807D8184B342202FB0030E9
:1016C00019B1C3680BB1A3E7704770B5144DD5F8D5
:1016D0001841002C0FDDD5F8B83098420CD005F138
:1016E000B8063346002203E053F8041F884206D0B0
:1016F0000132A242F8D170BD002205F1B806900077
:10170000011DA21A920031443044013C1FF0A7FF92
:10171000C5F8184170BD034B1868D1E7981C00202C
:101720000C2900200876002010B54FF4804082B0CC
:1017300016F0EEFA00B30022032390F902000093A2
:1017400001924FF4E1334FF4804115F069FF0C4BE7
:10175000C3F8A80070B1012402221520214683F8A5
:10176000B04083F8B14083F8B24083F8AC20FFF773
:101770009FFF204602B010BD014BD3F8A800E9E757
:101780000C290020F0B50D4685B006460068F1F73B
:10179000C2FD95E81800E41A0023039324238DF872
:1017A00008304D238DF80930B5F90A30FF2C224658
:1017B000A8BFFF2201333DD02B7B002B0CBF3E2363
:1017C0003C238DF80A30FE2C2B898DF80B208DF8E8
:1017D0000C3031DD23128DF80D408DF80E300727C7
:1017E0003A4602A93068F1F79BFD02ABDA190DF118
:1017F0000B0100238A4221D1002C8DF807300CDD2B
:10180000224629683068F1F78BFD2B689DF8072088
:101810001919994216D18DF8072001220DF10701FF
:101820003068F1F77DFD3068F1F770FD04F10900D3
:1018300005B0F0BD2123C4E70527D1E711F8010B5E
:101840004340D7E713F8010B4240E2E72DE9FF4799
:101850000024104E07460D469846204601EB02092B
:10186000A246A159A31971B10A79142A0BD069466D
:1018700018468DE82002ADF80870ADF80AA08DF882
:101880000C80FFF77FFFCC34B4F5197FE9D104B0A9
:10189000BDE8F087F05000207C4B1B7893B12DE918
:1018A000F0417B4B7B4C9B79D4F81C51C4F81C0154
:1018B000013B82B0451B032B00F2B680DFE803F04A
:1018C00022709907744A1360536093607047D4F88C
:1018D0002C31C31A002B0ADD00F5C3350022A035D8
:1018E000114601236E20C4F82C51FFF7AFFF6A4B5D
:1018F000D4F8A420D4F8A01099605A601A6002B0FD
:10190000BDE8F081654A664BD279DFF8B48133F8DF
:101910001220B8F902306348B8F9001092B207EE0D
:10192000902A40F6E44707FB02F6C3EB1633B8EE05
:10193000670A4FF47A7606FB03F393FBF1F3E36651
:10194000F1F7EEF8E06ED4ED197ADFED576AB8F9E9
:101950000210514BB8F900E0586000FB05F207EEA9
:10196000102AB8EEC77ABCEEC06AE7EE267A8DED93
:10197000016ABDF80420C4ED197ABDEEE77A07FBD1
:1019800002F7C1EB173706FB07F683ED027A96FBE9
:10199000FEF684ED187AA6661E6002B0BDE8F081FE
:1019A0001BF06EFC002847D0404B414A1B78B4F82E
:1019B0002211D2ED037AC4F89C10DB0756D401FB48
:1019C00005F207EE902ADFED386A334BB8EEE77A7E
:1019D000D4ED267A5960E7EE267A1960BDEEE77AF3
:1019E000C4ED267A84ED257A83ED027A02B0BDE853
:1019F000F081304B1B68190181D5FF200EF03AFDB4
:101A000003780A2B88BF0021234B9CBFB0F9042028
:101A1000B0F90610C4F8241188BF0A46C4F828217A
:101A20005A601A6099606AE71B4B00221A605A607C
:101A30009A6002B0BDE8F0811E4B1B68DE06B3D58C
:101A40001A4BB4F822111B78C4F89C10DA07B6D5EB
:101A5000B4F92021184B00FB02F083FB0023C017D0
:101A6000C0EBA3100144C4F89C10A8E7FDEEE77A90
:101A7000124E17EE900AA0F57A7202FB02F386FB73
:101A80000306D817C0EB26101044E1E7164F0020DC
:101A9000947600200C290020AC740020C45400204F
:101AA000E05400207C2900202FE33E3168740020A0
:101AB000184F002094660020D34D62101F85EB5113
:101AC000203500202DE9F347012016F021F9174EAB
:101AD000DFF85CA00024CC2708B1022C02D902B0A8
:101AE000BDE8F08707FB04F856F8085015B101343B
:101AF000E4B2F1E7C37890F902005AF82330019577
:101B00000322009201212A4615F08AFD814648B140
:101B100004FB0760CC2229461FF0BBFD013446F8C8
:101B20000890E4B217F0CEFED6E700BFF0500020D8
:101B3000644703082DE9F04F2DED088BBD4CBE4BDB
:101B4000C4F8443887B00023C4F84838F3F702FDDE
:101B5000F1F7D4FFF2F754FE08B9F4F787FDF5F773
:101B6000D3FA0522B549B6481FF0DEFD08B1F4F7F7
:101B70007DFD94F84C38B34D43F0010384F84C38A4
:101B8000B14B9A78B14B1A70B14B1B682B6011F0B6
:101B9000B7F801210220F2F705FCF2F767FD2B6888
:101BA0001F070BD5AB4B1A7A0A2A07D8012393409B
:101BB00040F20342134201D010F034FF6420A64EDD
:101BC000F5F72AFEF4F742FEA44ADFF8C0E200234C
:101BD000B146985D03F10F0103F113073144374417
:101BE0000EEB000A11F8018FB8F1000F05D09AF83A
:101BF0000CC0C44508BF82F858C091F80480B8F101
